:020000020000FC
:100000000C940CF20C949B3A0C949C3A0C949D3AF0
:100010000C949E3A0C949F3A0C94A03A0C94A13AFA
:100020000C94A23A0C94A33A0C94173B0C94183BF2
:100030000C9488E30C94193B0C941A3B0C941B3BD6
:100040000C947C3B0C947D3B0C94A9E60C947E3B79
:100050000C947F3B0C94803B0C94913B0C94923B12
:100060000C94933B0C94943B0C943DE40C94953B82
:100070000C94963B0C94973B0C94FAE80C94983BA8
:100080000C94993B0C949A3B0C949B3BFFE30B54D0
:100090000200000010270000000000002530327828
:1000A0000025303478002575002530327500253064
:1000B0003375002530347500253035750025303511
:1000C0006C75002530386C7500253032752530325E
:1000D0007525303475002530327525303275002590
:1000E0003032752F253032752F253034752025306C
:1000F00032753A2530327500200025002A002F0085
:100100002D003D0000434F4D31202D2025732C251F
:10011000732C6E2C382C3100434F4D32202D20256E
:10012000732C25732C6E2C382C3100284329203257
:1001300030303420000A000C001B21001B25001B5E
:100140001C7001001B1C7081001B1C7010001B64C4
:100150003000425300584F4E2F584F464600393614
:100160003030003139323030003537363030003100
:100170003135323030008480928020253032752F26
:10018000253032752F253034750091204E202530D2
:100190003475208F8E204E20253034750091202517
:1001A0003032752F253032752F25303475208F8EE3
:1001B00020253032752F253032752F2530347500CB
:1001C000918C858D8020253034750080008D8325AD
:1001D00069200091858A96889F204E20257500848D
:1001E0008E8A938C858D92204E2530357520808D9A
:1001F0008D938B88908E82808D00848E8A938C85DF
:100200008D92204E25303575208D8584858991927B
:10021000828892858B858D2E00848E8A938C858D25
:1002200092204E20253035752087809085838891D7
:10023000929088908E82808D00848E8A938C858D9A
:100240009220008F8E82928E908D809F208F859736
:1002500080929C20848E8A938C858D928000828EE1
:10026000919192808D8E828B858D8E208887209DA6
:100270008A8B8700908583889192908096889F20B2
:100280008A8A8C204E202575008F8E918B85848DD7
:100290009F9F20918C858D80202575009085838877
:1002A000919290205A2D8E929785928E8200908501
:1002B0008388919290208D808B88978D9B95008D5F
:1002C0008090809192809E9988892088928E832048
:1002D0008F908E848086008E9192808B8E919C2050
:1002E00087808A909B92888920918C858D202575A6
:1002F0000091938C8C80208F908E848086005A2D64
:100300008E92978592204E20257500952D8E92977E
:100310008592204E2025750091828E848D9B8900C8
:100320008F8E208A8091918890808C008F8E209172
:10033000858A96889F8C008E9297859220918D9FBA
:100340008B20009488918A808B9C8D9B89208E9233
:10035000978592204E202575008F908E838E8D2E4E
:1003600020829B8F8E8B8D858D8E20257525252E49
:10037000208E9888818E8A2025752E008D808B8E08
:10038000838E82809F208390938F8F80202575009D
:1003900022888D8A8E92858A91220090AEE1E1A812
:1003A000EF2C20313035343834208CAEE1AAA2A0B5
:1003B0002C00E3AB2E2031362D8FA0E0AAAEA2A0F8
:1003C000EF2C2032362C20E22FE42028303935293A
:1003D0003734322D3031313900452D6D61696C3A39
:1003E00020696E636F746578406D61696C2E636E11
:1003F000742E7275001B2501202020202020202033
:10040000209488918A808B9C8D9B8920848E8A93EE
:100410008C858D9220FEFF0A1B25000020202020C5
:100420002020202020202020208A8E8F889F20843A
:100430008E8A938C858D9280202020202020202061
:10044000200A008F9085829B98858D8885208F90CB
:100450008E848E8B868892858B9C8D8E919288203F
:10046000918C858D9B008E928C858D80208F8597B9
:1004700080928820848E8A938C858D9280210020A2
:1004800020202020202020202020202080828090DA
:10049000889F208F8892808D889F210A008D859467
:1004A00088918A808B9C8D9B8920908586888C0082
:1004B0008082928E9285919288908E82808D88859E
:1004C000009285958D8E8B8E83889785918A8889F9
:1004D000209181908E91208A8A8C00939192808DB8
:1004E0008E828A80208780828E84918A8895208D52
:1004F000809192908E858A208A8A8C009280898C45
:100500008590202D200092859192204E56205241B8
:100510004D202D20009285919220948F202D200037
:1005200092859192209D8A8B87202D20008E98881D
:10053000818A80200020888B88208D85922087806A
:10054000838B93988A880087808F88918800979200
:10055000858D889F00888D948E908C8096888820C9
:100560008220948F0093918F85988D8E0092859133
:100570009220434F4D31202D2000928591922043AF
:100580004F4D32202D200084809297888A208485C8
:100590008D85868D8E838E209F99888A80202D2040
:1005A000009080878E8C8A8D93920087808C8A8DB4
:1005B0009392008A8E8D92908091928D8E91929CD2
:1005C000208F8597809288202825692D25692920EC
:1005D0002D2025692085842E008C8E84858B9C207F
:1005E0002D20008F908E8887828E848892858B9CA8
:1005F000202D200082859091889F208F8E202D2095
:10060000008A8A8C20818B8E8A88908E82808D8051
:10061000008D858F908082888B9C8D9B8920828223
:100620008E84208F80908E8B9F008D808B8E838E0A
:10063000828E838E20888D918F858A928E90800005
:100640008F8E8F9B928A802082828E848020818EE2
:100650008B85852090808D8D8589208480929B2C30
:100660000097858C2084809280208F8E918B85844A
:100670008D85892087808F889188208220948F00A3
:10068000838098858D8885208D85208F908E8285AA
:1006900084858D8E2E008A8E8D8596208082928E06
:1006A0009285919288908E82808D889F0094889107
:1006B0008A808B88878096889F208A8A8C0094887D
:1006C000918A808B88878096889F208F908E988BC8
:1006D000802093918F85988D8E009085838891924C
:1006E000908096889F208F908E988B802093918FFA
:1006F00085988D8E00838098858D8885008CA5E0F7
:10070000AAE3E0A8A9204D532D4B008E8E8E202207
:10071000888D8A8E92858A912200312E30204D5309
:100720004B2042332E3400938A8087808D8D9B89A5
:100730002082808C88208F8590888E8400829B9573
:100740008E848892208780208390808D88969B203D
:100750008F8590888E84802C00878094888A9188E9
:10076000908E82808D8D8E838E2082209488918AB7
:10077000808B9C8D8E89208F808C9F928821008D0C
:100780008520918E848590868892209488918A8095
:100790008B9C8D9B952087808F88918589210087F0
:1007A0008084808D208F8590888E8420918C858D8B
:1007B00000878084808D208F8590888E842084801F
:1007C0009200918E84859086888C8E852094889165
:1007D0008A808B9C8D8E89208F808C9F9288008749
:1007E0008094888A9188908E82808D208F859088D1
:1007F0008E842084809200878094888A9188908E4D
:1008000082808D208F8590888E8420918C858D00AC
:1008100094808A92889785918A8889208F8590888C
:100820008E8420918C858D0094808A928897859102
:100830008A8889208F8590888E8420848092008881
:10084000928E838E829B852091938C8C9B008D85CC
:100850008A8E9090858A928D9B852084808D8D9B39
:100860008521009D8A8B87208D85208E9282859799
:10087000808592208D802087808F908E919B009123
:10088000818E89208A90888F928E8F908E96859106
:10089000918E9080209D8A8B87008F8590858A8B92
:1008A0009E97889285208F8892808D88852094904D
:1008B000009D8A8B8720002023002530386C75200E
:1008C000232530366C75009D8A8B8720808A92881C
:1008D00082888788908E82808D80208220918E9160
:1008E0009280828520849093838E89208A8A8C00CE
:1008F0009D8A8B87208D8520808A92888288878830
:10090000908E82808D80009D8A8B8720818B888746
:100910008A80208A2087808F8E8B8D858D889E008F
:1009200080828090889F209D8A8B87008D8588910A
:100930008F908082888C809F208E9888818A8020EA
:100940009D8A8B87008090958882209D8A8B872046
:1009500087808A909B920080828090889F208A91D5
:10096000208220918E9192808285209D8A8B8700A3
:1009700088919785908F808D208290858C858D8D34
:100980008E89209085919390912088918F2E209D23
:100990008A8B87009D8A8B87208F8590858F8E8B91
:1009A0008D858D80009D8A8B872093868520808A07
:1009B000928882888788908E82808D8000808A923B
:1009C000888288878096889F209D8A8B87204E20EA
:1009D0002575009080878B88978D9B85208D8E8CC8
:1009E00085908020918C858D208220948F20882076
:1009F0009D8A8B87008D858A8E9090858A928D8EB8
:100A00008520918E91928E9F8D8885209D8A8B87DF
:100A1000008D85922087808F908E98858D8D9B95F7
:100A20002084808D8D9B952082209D8A8B87008ECF
:100A30009888818A802091829F87882091209D8A32
:100A40008B87008D8E8C859020918C858D9B20824C
:100A5000208A80919185204E202569008D8E8C857D
:100A60009020918C858D9B2082209D8A8B87204EA3
:100A7000202569008F908E828584889285208380CE
:100A800098858D8885208A8A8C00EB72F072F472CA
:100A9000F872FC720073047308730C731073147390
:100AA00018731C732073247328732C73307334737E
:100AB00038732E3030008A8A8C2000908D20008878
:100AC0008D8D20008D8420008D9720008A8091914B
:100AD000889020008F908E84808680200091848072
:100AE00097802000828E8782908092208F908E84C3
:100AF0002E208D808B2E2000828E878290809220E7
:100B00008F908E842E20818D2E2000808D8D938B52
:100B10002E208F908E842E208D808B2000808D8DB6
:100B2000938B2E208F908E842E20818D2E200091ED
:100B3000938C8C802000828D8591858D8885208D79
:100B4000808B88978D2E2000829B8F8B80928020B7
:100B50008D808B88978D2E20008F8E8A938F8A8030
:100B60002000828E8782908092208F8E8A2E208D08
:100B7000808B2E2000828E8782908092208F8E8A9A
:100B80002E20818D2E2000808D8D938B2E208F8E98
:100B90008A2E208D808B2E2000808D8D938B2E2091
:100BA0008F8E8A2E20818D2E20008E8F8B809280BA
:100BB000208D808B88978D9B8C8820008E8F8B80DA
:100BC00092802082208A908584889220008E8F8B4C
:100BD000809280208A8090928E8920008E8F8B80D8
:100BE0009280208D808B2F8A908584889220008E21
:100BF0008F8B809280208D808B2F8A809092802096
:100C0000008A8E8B8897859192828E0091938C8C2E
:100C100080008A8E8B2D828E208D808B88978D9B75
:100C20008C880091938C8C80208D808B88978D9BF5
:100C30008C88008A8E8B2D828E208185878D808B7B
:100C400088978D9B8C880091938C8C8020818587E0
:100C50008D808B88978D9B8C88008A8E8B8897855A
:100C60009192828E209280909B0091938C8C802018
:100C70009280909B008A8E8B8897859192828E209D
:100C800082208A90858488920091938C8C80208227
:100C9000208A9085848892008A8E8B88978591928D
:100CA000828E208A8090928E890091938C8C8020F5
:100CB0008A8090928E890091938C8C80208D808B7D
:100CC00088978D9B95008F908E848086008F8E8A6A
:100CD000938F8E8A008F2090208E20842080208603
:100CE0002088008F208E208A2093208F208A2088C1
:100CF00000828E87829080929B208F908E84808647
:100D00008800808D8D938B88908E82808D889F0047
:100D1000828E87829080929B208F8E8A938F8A8882
:100D200000808D8D938B88908E822E208F8E8A935B
:100D30008F8A8800918A88848A88008D8084818047
:100D4000828A8800828D8591858D8885208D808B13
:100D500088978D9B9500829B8F8B809280208D80C1
:100D60008B88978D9B95008D808B8E8388008D80DE
:100D700090809192809E9988892088928E83008DA0
:100D8000858485899192822E20848E8A938C858D8C
:100D9000929B0091938C8C80208D85208E818B2E50
:100DA000208D808B8E832E00828E87829080929BF6
:100DB00020918A88848E8A00828E87829080929B7E
:100DC000208D80848180828E8A00918A88848A80A6
:100DD00020008D80848180828A802000BBFFEEAA63
:100DE000BBFFEEAA20202020202020202020202031
:100DF000202020200708090A0B0C0D0D0E0E0F0FE6
:100E00000F101011111112121212121213131313C8
:100E1000131313131313131313131313141414149E
:100E200015151515161616171717181818191A1B51
:100E30001C1D1E1F00124080C0114080C000000019
:100E400000000000000000000000000000000000A2
:100E50000000000000000000000000000000000092
:100E60000000000000000000000000000000000082
:100E70000000000000000000000000000000000072
:100E80000000007000700030003000300030003092
:100E9000003000300000003000780030000000001A
:100EA0000000000000000000000000000000000042
:100EB0000000000000CC00CC00CC00CC00CC00CC6A
:100EC0000000000000000000000000000000000022
:100ED0000000000000000000000000000000000012
:100EE00000000000000000980198019801CC00FE6D
:100EF00001CC006600FF006600660033003300335B
:100F000000000000000000000000000000000000E1
:100F10000000000000180018007E00FE00DB001B2F
:100F2000001F001E003C007800F800D800DB007FA6
:100F3000007C001000100000000000000000000015
:100F40000000000000000000001E001B001B001B32
:100F5000001F03CF03F0003800EE01B701B301B06A
:100F600001F001F00000000000000000000000009F
:100F7000000000000000000000000000001E003F14
:100F800000330033001F001E009E01B201B301B305
:100F900001F300FF009E01000000000000000000BF
:100FA0000000000000000000000000000000003011
:100FB0000030003000300030003000000000000041
:100FC0000000000000000000000000000000000021
:100FD0000000000000000000000000000060007041
:100FE00000380018001C000C000C000C000C000C59
:100FF000000C000C001C001800380070006000009D
:1010000000000000000000000000000000000018C8
:1010100000380070006000E000C000C000C000C0E8
:1010200000C000C000C000E0006000700038001880
:1010300000000000000000000000000000000000B0
:10104000000000000000000000100010009301D715
:101050000138006C00C600C701000000000000005D
:101060000000000000000000000000000000000080
:10107000000000000000000000180018001800FF29
:1010800000FF001800180018000000000000000019
:101090000000000000000000000000000000000050
:1010A0000000000000000000000000000000000040
:1010B00000000000000000000000003000300030A0
:1010C00000180018000800000000000000000000E8
:1010D0000000000000000000000000000000000010
:1010E00000000000000000FC00FC00000000000008
:1010F00000000000000000000000000000000000F0
:1011000000000000000000000000000000000000DF
:1011100000000000000000000000000000000000CF
:1011200000300078003000000000000000000000E7
:1011300000000000000000000000000000000000AF
:101140000000000000000000008001C000600030CE
:101150000018000C00060003000000000000000062
:10116000000000000000000000000000000000007F
:10117000003C007E00E700C300C300C300C300C3FF
:1011800000C300C300E7007E003C00000000000038
:10119000000000000000000000000000000000004F
:1011A00000000018001E001E00180018001800188B
:1011B000001800180018001800FF00FF00000000D1
:1011C000000000000000000000000000000000001F
:1011D00000000000007E00FF00C300C300E00060CC
:1011E00000700038001C000E000700FF00FF000028
:1011F00000000000000000000000000000000000EF
:10120000000000000000007C007F00E300C000C080
:101210000078007800C000C000C000C3007F007CE0
:1012200000000000000000000000000000000000BE
:101230000000000000000000007000780078006CE2
:10124000006C00660066006300FF01FF0160006043
:10125000006000000000000000000000000000002E
:101260000000000000000000000000FE00FE00067C
:101270000003003B007F00E000C000C000C000E3AE
:10128000007F003E000000000000000000000000A1
:10129000000000000000000000000000007C00FED4
:1012A00000C700030003003B007F00E700C300C34A
:1012B00000E7007E003C000000000000000000008D
:1012C000000000000000000000000000000000FE20
:1012D00000FE00C000600060003000300018001800
:1012E000000C000C000600060000000000000000DA
:1012F00000000000000000000000000000000000EE
:10130000007E00FF00C300C300C300FF007E00C3D7
:1013100000C300C300C300FF007E00000000000007
:1013200000000000000000000000000000000000BD
:101330000000003C007E00E700C300C300E700FEA1
:1013400000FE00C000C000E3007F003E000000007F
:10135000000000000000000000000000000000008D
:1013600000000000000000000030007800300000A5
:101370000000000000000000003000780030000095
:10138000000000000000000000000000000000005D
:101390000000000000000000003000780030000075
:1013A0000000000000000000003000300030001895
:1013B000001800080000000000000000000000000D
:1013C000000000000000000000000000000000C05D
:1013D00001F00178000E0007000E007800F001C057
:1013E00001000000000000000000000000000000FC
:1013F00000000000000000000000000000000000ED
:101400000000000000FE00FE0000000000FE00FEE4
:1014100000000000000000000000000000000000CC
:1014200000000000000000000000000000000000BC
:1014300000000007001F007C00E000C001E0007C0D
:10144000001F000700000000000000000000000076
:101450000000000000000000000000000000007814
:1014600000CC0084008000C000600030001000103C
:101470000000003000780030000000000000000094
:101480000000000000000000000000000000003824
:1014900000CE00820003016101B1011101110111AF
:1014A000013101E301020006007C000000000000A1
:1014B000000000000000000000000000000000002C
:1014C000000000180018003C003C003C006600666C
:1014D000006600FF00C300C300C300C3000000009B
:1014E00000000000000000000000000000000000FC
:1014F00000000000007F00FF00C300C300C3007FA6
:10150000007F00C300C300C300C300FF007F0000D2
:1015100000000000000000000000000000000000CB
:10152000000000000000007E00FE00C70003000372
:101530000003000300030003000300C700FE007E59
:10154000000000000000000000000000000000009B
:101550000000000000000000007F007F00E300C3E7
:1015600000C300C300C300C300C300C300E3007F87
:10157000007F0000000000000000000000000000EC
:101580000000000000000000000000FF00FF00035A
:1015900000030003007F007F00030003000300033B
:1015A00000FF00FF0000000000000000000000003D
:1015B00000000000000000000000000000FF00FF2D
:1015C0000003000300030003007F007F000300030B
:1015D0000003000300030000000000000000000002
:1015E0000000000000000000000000000000007E7D
:1015F00000FE00C7000300030003007300F300C3F4
:1016000000C300C700FE007E0000000000000000D4
:1016100000000000000000000000000000000000CA
:1016200000C300C300C300C300C300FF00FF00C32A
:1016300000C300C300C300C300C3000000000000DB
:10164000000000000000000000000000000000009A
:101650000000007E007E0018001800180018001816
:101660000018001800180018007E007E000000001E
:10167000000000000000000000000000000000006A
:101680000000000000F000F000C000C000C000C07A
:1016900000C000C300C300C300E6007E003C0000A1
:1016A000000000000000000000000000000000003A
:1016B00000000000000000C3006300730033001B43
:1016C000000F000F001B003B0033006300E300C36A
:1016D0000100000000000000000000000000000009
:1016E00000000000000000000003000300030003EE
:1016F000000300030003000300030003000300FFD6
:1017000000FF0000000000000000000000000000DA
:101710000000000000000000000000C300C300FF44
:1017200000FF00DB00DB00DB00DB00C300C300C305
:1017300000C300C300000000000000000000000023
:10174000000000000000000000000000008301878E
:10175000018F019B019B01B301B301B301B301E30D
:1017600001C301C30183010000000000000000006C
:101770000000000000000000000000000000003C2D
:10178000007E00E700C300C300C300C300C300C362
:1017900000C300E7007E003C0000000000000000E5
:1017A0000000000000000000000000000000000039
:1017B000007F00FF00C300C300C300FF007F0003E1
:1017C000000300030003000300030000000000000A
:1017D0000000000000000000000000000000000009
:1017E000007E007E00E700C300C300C300C300C347
:1017F00000C300C300E7007E007E006000E000C080
:1018000000000000000000000000000000000000D8
:1018100000000000007F00E300C300C300C300FF1E
:10182000007F00330063006300C300C30083010036
:1018300000000000000000000000000000000000A8
:10184000000000000000007E00FF00C3000300074E
:10185000000E0038007000E000C000C300FF007EF2
:101860000000000000000000000000000000000078
:10187000000000000000000000FF00FF001800183A
:101880000018001800180018001800180018001898
:101890000018000000000000000000000000000030
:1018A0000000000000000000000000C300C300C3EF
:1018B00000C300C300C300C300C300C300C300E7EC
:1018C000007E003C0000000000000000000000005E
:1018D000000000000000000000000000008301C3C1
:1018E00001C600C600C6006C006C006C00380038F1
:1018F0000038001000100000000000000000000090
:101900000000000000000000000000000000008354
:1019100001830183018301D301D600D600EE00EEDE
:1019200000EE0044004400440000000000000000FD
:1019300000000000000000000000000000000000A7
:1019400000C300E70066003C003C0018003C003C7F
:1019500000660066006600C300C3000000000000CF
:101960000000000000000000000000000000000077
:10197000000000C300E7006600660066003C003C13
:10198000003C0018001800180018001800000000A3
:101990000000000000000000000000000000000047
:1019A0000000000000FE00FE00600060003000301B
:1019B00000180018000C000C000600FE00FE0000DD
:1019C0000000000000000000000000000000000017
:1019D000000000FC00FC000C000C000C000C000CD3
:1019E000000C000C000C000C000C000C000C000C97
:1019F00000FC00FC000000000000000000000000EF
:101A000000000000000000000000000000000000D6
:101A1000000000030006000C00180030006000C049
:101A20000080010000000000000000000000000035
:101A300000000000000000FC00FC00C000C000C06E
:101A400000C000C000C000C000C000C000C000C096
:101A500000C000C000FC00FC00000000000000000E
:101A60000000000000000000000000000000003046
:101A7000007800CC0086010000000000000000009B
:101A80000000000000000000000000000000000056
:101A90000000000000000000000000000000000046
:101AA0000000000000000000000000000000000036
:101AB000000000000000000000FF03FF0300000022
:101AC0000000000000000000000000000000000016
:101AD000001800180018003000300020000000003E
:101AE00000000000000000000000000000000000F6
:101AF00000000000000000000000000000000000E6
:101B00000000000000000000003C007E0066006055
:101B1000007E007F0063006300FF00DE0000000025
:101B200000000000000000000000000000000000B5
:101B300000000006000600060006007600FE00CE4B
:101B4000018601860186018601CE01FE0076000035
:101B50000000000000000000000000000000000085
:101B6000000000000000000000000000007C00FEFB
:101B700000C7000300030003000300C700FE007C51
:101B80000000000000000000000000000000000055
:101B900000000000000000C000C000C000C000FC49
:101BA00000FE00C700C300C300C300C300C700FE9F
:101BB00001BC010000000000000000000000000067
:101BC0000000000000000000000000000000000015
:101BD000003C007E00C300E7007F0003000300C755
:101BE00000FE007C0000000000000000000000007B
:101BF0000000000000000000000000F800FC018C64
:101C0000010C007F007F000C000C000C000C000C8D
:101C1000000C000C000C00000000000000000000A0
:101C200000000000000000000000000000000000B4
:101C300000BC01FE01C700C300C300C300C300C74E
:101C400000FE00FE00C000C600FE007C0000000098
:101C50000000000000000000000000000000000381
:101C6000000300030003007300FB00CF00C700C3A4
:101C700000C300C300C300C300C300000000000095
:101C80000000000000000000000000000000000054
:101C90000030003000000000003C003C003000300C
:101CA0000030003000300030003000300000000014
:101CB0000000000000000000000000000000000024
:101CC00000C000C00000000000F000F000C000C034
:101CD00000C000C000C000C000C000CC00CC00FCB0
:101CE000007800000000000000000000000000007C
:101CF00000000000000300030003000300C30063B2
:101D00000033001B000F001F0033006300C300837B
:101D100001000000000000000000000000000000C2
:101D2000000000000000003C003C003000300030AB
:101D30000030003000300030003000300030003023
:101D40000030000000000000000000000000000063
:101D50000000000000000000000000000000000083
:101D6000009B01FF03330333033303330333033394
:101D700003330333030000000000000000000000F4
:101D80000000000000000000000000000000000053
:101D9000000000E600F6019E0186018601860186AC
:101DA000018601860186010000000000000000009D
:101DB0000000000000000000000000000000000023
:101DC00000000000003C007E00E700C300C300C329
:101DD00000C300E7007E003C00000000000000009F
:101DE00000000000000000000000000000000000F3
:101DF0000000007700FF00CE018601860186018683
:101E000001CE01FE00760006000600060006000076
:101E100000000000000000000000000000000000C2
:101E20000000000000BC01FE01C700C300C300C3E6
:101E300000C300C700FE00FC00C000C000C000C01E
:101E40000000000000000000000000000000000092
:101E500000000000000000000000007300FF00CE42
:101E60000006000600060006000600060006000048
:101E70000000000000000000000000000000000062
:101E8000000000000000000000000000007E00FFD5
:101E900000C30007001E007800E000C300FF007EC2
:101EA0000000000000000000000000000000000032
:101EB00000000000000000000000000C000C007F8B
:101EC000007F000C000C000C000C000C00CC00FC8F
:101ED000007800000000000000000000000000008A
:101EE00000000000000000000000000000000000F2
:101EF00000C300C300C300C300C300C300E300F37A
:101F000000BF019E01000000000000000000000072
:101F100000000000000000000000000000000000C1
:101F2000000000C300C300C300660066003C003C24
:101F30000018001800180000000000000000000059
:101F40000000000000000000000000000000000091
:101F50000000000000C300C300DB00DB007E007E49
:101F600000660066006600660000000000000000D9
:101F70000000000000000000000000000000000061
:101F800000000000000000C300C30066003C001811
:101F90000018003C006600C300C300000000000001
:101FA0000000000000000000000000000000000031
:101FB0000000000000000086018601CE01CC00CCAC
:101FC00000780078003000300030001B001F000E49
:101FD0000000000000000000000000000000000001
:101FE0000000000000000000000000FE00FE006095
:101FF00000300018000C000C000600FF00FF00007D
:1020000000000000000000000000000000000000D0
:1020100000000000000000C0006000300030003010
:1020200000300030001C001C003000300030003058
:1020300000300060000000000000000000000030E0
:102040000030003000300030003000300030003010
:102050000030003000300030003000300030003000
:1020600000300030003000000000000000000000E0
:102070000000000000000000000C001800300030DC
:1020800000300030003000E000E000300030003070
:10209000003000300018000C0000000000000000BC
:1020A0000000000000000000000000000000000030
:1020B00000000000000000000000000C009F01F381
:1020C00001600000000000000000000000000000AF
:1020D0000000000000000000000000000000000000
:1020E00000000000000000000000000000000000F0
:1020F00000000000000000000000000000000000E0
:1021000000000000000000000000000000000000CF
:1021100000180018003C003C003C006600660066A9
:1021200000FF00C300C300C300C3000000000000A4
:10213000000000000000000000000000000000009F
:102140000000007F007F0003000300030003007F06
:1021500000FF00C300C300C300FF007F00000000B9
:10216000000000000000000000000000000000006F
:1021700000000000007F00FF00C300C300C3007F19
:10218000007F00C300C300C300C300FF007F000046
:10219000000000000000000000000000000000003F
:1021A00000000000000000FF00FF00030003000328
:1021B0000003000300030003000300030003000307
:1021C000000000000000000000000000000000000F
:1021D0000000000000000000007000F800CC00C605
:1021E00000C600C600C600C600C600C600C600FE87
:1021F00000FF0183018301000000000000000000D7
:102200000000000000000000000000FF00FF0003CD
:1022100000030003007F007F0003000300030003AE
:1022200000FF00FF000000000000000000000000B0
:1022300000000000000000000000000000DB00DBE8
:1022400000DB007E003C003C003C007E00DB00DB4D
:1022500000DB00DB00DB00000000000000000000ED
:102260000000000000000000000000000000007CF2
:1022700000FE00C600C000600070007000C000C01A
:1022800000C000C600FE007C00000000000000004E
:10229000000000000000000000000000000000003E
:1022A00000C300C300C300E300F300DB00DB00DB7E
:1022B00000CF00C700C300C300C30000000000003F
:1022C00000000000000000000000000000180018DE
:1022D000000000C300C300E300F300F300DB00DBF9
:1022E00000DB00CF00CF00C700C300C30000000028
:1022F00000000000000000000000000000000000DE
:102300000000000000C3006300330033001B000F17
:10231000000F001B001B0033006300C300C300005C
:1023200000000000000000000000000000000000AD
:1023300000000000000000180018003C003C003CB9
:1023400000660066006600C300C300C300C300C38C
:10235000000000000000000000000000000000007D
:10236000000000000000000000C300C300E700FF01
:1023700000DB00DB00DB00DB00C300C300C300C3E5
:1023800000C300000000000000000000000000008A
:102390000000000000000000000000C300C300C3F4
:1023A00000C300C300FF00FF00C300C300C300C39D
:1023B00000C300C300000000000000000000000097
:1023C000000000000000000000000000003C007E53
:1023D00000E700C300C300C300C300C300C300C3C1
:1023E00000E7007E003C000000000000000000004C
:1023F000000000000000000000000000000000FFDE
:1024000000FF00C300C300C300C300C300C300C378
:1024100000C300C300C300C30000000000000000B0
:1024200000000000000000000000000000000000AC
:10243000007F00FF00C300C300C300FF007F000354
:10244000000300030003000300030000000000007D
:10245000000000000000000000000000000000007C
:102460000000007C00FE00C700030003000300031F
:1024700000030003000300C700FE007C0000000012
:10248000000000000000000000000000000000004C
:102490000000000000FF00FF0018001800180018DE
:1024A0000018001800180018001800180018000084
:1024B000000000000000000000000000000000001C
:1024C00000000000000000C300C300C300C300C33D
:1024D00000C300C600FC00F800C000E3007F003E1F
:1024E00000000000000000000000000000000000EC
:1024F00000000000000000000018007E00FF00DB6C
:1025000000DB00DB00DB00FF007E00180018001875
:1025100000180000000000000000000000000000A3
:102520000000000000000000000000C300C30066BF
:10253000003C00180018003C003C0066006600E704
:1025400000C300C300000000000000000000000005
:1025500000000000000000000000000000C300C3F5
:1025600000C300C300C300C300C300C300C300C353
:1025700000C300FF00FF018001C000000000000058
:10258000000000000000000000000000000000C388
:1025900000C300C300C300C300C300FE00FC00C0B2
:1025A00000C000C000C000C000000000000000002B
:1025B000000000000000000000000000000000001B
:1025C00000C300C300DB00DB00DB00DB00DB00DB63
:1025D00000DB00DB00DB00FF00FF0000000000006C
:1025E00000000000000000000000000000000000EB
:1025F000000000C300C300DB00DB00DB00DB00DB0E
:1026000000DB00DB00DB00DB00FF01FF018001805D
:1026100001000000000000000000000000000000B9
:10262000000000000007000700060006000600FE8C
:1026300000FE018601860186018601FE01FE000082
:10264000000000000000000000000000000000008A
:1026500000000000000000830183018301830183E7
:10266000019F01BF01B101B101B101B101BF019FE2
:102670000100000000000000000000000000000059
:10268000000000000000000000030003000300033E
:102690000003007F00FF00C300C300C300C300FFAE
:1026A000007F0000000000000000000000000000AB
:1026B00000000000000000000000003E007F00E37A
:1026C00000C000C000F800F800C000C000C000E377
:1026D000007F003E0000000000000000000000003D
:1026E00000000000000000000000000000E300F314
:1026F00001BB031B031B031B031F031B031B031B48
:1027000003BB03F301E30000000000000000000031
:10271000000000000000000000000000000000FCBD
:1027200001FE01860186018601FE01FC0198018CF3
:10273000018C01860183018301000000000000007C
:102740000000000000000000000000000000000089
:10275000000000000000003C007E00660060007E7B
:10276000007F0063006300FF00DE00000000000047
:102770000000000000000000000000000000000059
:10278000007C00FE00C6000C003C007E00E700C399
:1027900000C300C300C300E7007E003C000000004F
:1027A0000000000000000000000000000000000029
:1027B0000000003E006600660036007E00FE0086D7
:1027C000018601860186018601C601FE007C0000AB
:1027D00000000000000000000000000000000000F9
:1027E000000000000000000000000000007E00FF6C
:1027F00000C300600038001C000600C300FF007E1C
:1028000000000000000000000000000000000000C8
:10281000000000000000003C007C00C000C000FC84
:1028200000FE00C700C300C300C300C300C700FE12
:10283000007C00000000000000000000000000001C
:102840000000000000000000000000000000000088
:10285000003C007E00C300FF007F0003000300C7B0
:1028600000FE007C000000000000000000000000EE
:102870000000000000000000000000000000000058
:10288000000000DB00DB00FF007E003C003C007E1F
:1028900000FF00DB00DB0000000000000000000083
:1028A0000000000000000000000000000000000028
:1028B00000000000007E00FF00C300C0007800F8A8
:1028C00000C000C300FF007E000000000000000008
:1028D00000000000000000000000000000000000F8
:1028E00000000000000000C300C300C300C300C319
:1028F00000C300C300E300FF019E010000000000D0
:1029000000000000000000000000000000000000C7
:10291000000000180018000000C300C300C300C37B
:1029200000C300C300C300E300BF019E010000001C
:102930000000000000000000000000000000000097
:102940000000000000000000000000C3006300332E
:10295000001B001B001F0033006300C30083010045
:102960000000000000000000000000000000000067
:1029700000000000000000000000000000E001F086
:10298000019801980198019801980198018C01869D
:102990000100000000000000000000000000000036
:1029A000000000000000000000000000000000C364
:1029B00000C300C300E700E700FF00DB00DB00C34B
:1029C00000C3000000000000000000000000000044
:1029D00000000000000000000000000000000000F7
:1029E00000C300C300C300FF00FF00C300C300C357
:1029F00000C300C300000000000000000000000051
:102A000000000000000000000000000000000000C6
:102A10000000003C007E00E700C300C300C300C309
:102A200000E7007E003C0000000000000000000005
:102A30000000000000000000000000000000000096
:102A40000000000000FE01FE01860186018601866D
:102A50000186018601860186010000000000000059
:102A60000000000000000000000000000000000066
:102A7000000000E700E700E700000000000000E7BA
:102A800000E700E7000000000000000000E7000091
:102A90000000000000000000000000000000000036
:102AA000000000E700E700E700180318031803E739
:102AB00000E700E7001803180318031803E700E70E
:102AC0000000000000000000000000000000000006
:102AD0000000000000FF03FF03FF036300630063C7
:102AE00000FF03FF03FF036300630063006300FF55
:102AF00003FF0300000000000000000000000000D1
:102B000000000000000000300030003000300030D5
:102B10000030003000300030003000300030003035
:102B20000030003000000000000000000000000045
:102B30000000000000000000002000200020002015
:102B4000002000200020002000200020003F002066
:102B50000020002000200000000000000000000015
:102B60000000000000000000000000200020002005
:102B700000200020002000200020003F0020002036
:102B8000003F0020002000200000000000000000A6
:102B900000000000000000000000000000480048A5
:102BA00000480048004800480048004800480048E5
:102BB000004F0048004800480048000000000000A6
:102BC0000000000000000000000000000000000005
:102BD00000000000000000000000000000000000F5
:102BE0000000007F00480048004800480000000046
:102BF00000000000000000000000000000000000D5
:102C000000000000000000000000000000000000C4
:102C1000003F00200020003F002000200020000096
:102C200000000000000000000000000000000000A4
:102C3000000000480048004800480048004800489C
:102C40000048004F00400040004F00480048004846
:102C50000000000000000000000000000000000074
:102C600000000000004800480048004800480048B4
:102C70000048004800480048004800480048004814
:102C800000480000000000000000000000000000FC
:102C90000000000000000000000000000000000034
:102CA000000000000000007F00400040004F00488E
:102CB0000048004800000000000000000000000084
:102CC00000000000000000000048004800480048E4
:102CD0000048004800480048004F00400040007F86
:102CE00000000000000000000000000000000000E4
:102CF00000000000000000000000004800480048FC
:102D00000048004800480048004800480048007F4C
:102D100000000000000000000000000000000000B3
:102D20000000000000000000000000000020002063
:102D3000002000200020002000200020003F002074
:102D40000020003F00000000000000000000000024
:102D50000000000000000000000000000000000073
:102D60000000000000000000000000000000000063
:102D70000000003F00200020002000200000000094
:102D80000000000000000000000000000000000043
:102D90000020002000200020002000200020002033
:102DA0000020002000E00300000000000000000000
:102DB0000000000000000000000000000000000013
:102DC0000000002000200020002000200020002023
:102DD00000200020002000FF030000000000000091
:102DE00000000000000000000000000000000000E3
:102DF00000000000000000000000000000000000D3
:102E0000000000000000000000FF03200020002060
:102E10000020000000000000000000000000000092
:102E20000000000000000020002000200020002002
:102E30000020002000200020002000E003200020CF
:102E40000020002000000000000000000000000042
:102E50000000000000000000000000000000000072
:102E600000000000000000000000000000FF030060
:102E70000000000000000000000000000000000052
:102E800000000000000000000000002000200020E2
:102E9000002000200020002000200020002000FF53
:102EA000032000200020002000000000000000009F
:102EB00000000000000000000000000000200020D2
:102EC00000200020002000200020002000E003203F
:102ED000002000E00320002000200000000000008F
:102EE000000000000000000000000000000000489A
:102EF0000048004800480048004800480048004892
:102F0000004800C80348004800480048000000008E
:102F100000000000000000000000000000000000B1
:102F20000048004800480048004800480048004861
:102F300000C80308000800F80300000000000000BB
:102F40000000000000000000000000000000000081
:102F50000000000000000000000000000000000071
:102F6000000000F80308000800C8034800480048B3
:102F70000000000000000000000000000000000051
:102F80000000000000480048004800480048004891
:102F90000048004800CF0300000000FF03000000CD
:102FA0000000000000000000000000000000000021
:102FB0000000000000000000000000000000000011
:102FC00000000000000000FF0300000000CF0348E5
:102FD0000048004800000000000000000000000061
:102FE00000000000000000000048004800480048C1
:102FF000004800480048004800C80308000800C80E
:1030000003480048004800000000000000000000E5
:1030100000000000000000000000000000000000B0
:103020000000000000000000000000FF030000009E
:1030300000FF03000000000000000000000000008E
:1030400000000000000000000000000000480048F0
:1030500000480048004800480048004800CF0300EE
:10306000000000CF034800480048000000000000B6
:103070000000000000000000000000000000002030
:10308000002000200020002000200020002000FF61
:103090000300000000FF030000000000000000002B
:1030A0000000000000000000000000000000000020
:1030B00000480048004800480048004800480048D0
:1030C0000048004800FF030000000000000000006E
:1030D00000000000000000000000000000000000F0
:1030E00000000000000000000000000000000000E0
:1030F000000000FF0300000000FF0320002000206C
:1031000000000000000000000000000000000000BF
:1031100000000000000000000000000000000000AF
:10312000000000000000000000FF034800480048C5
:103130000048000000000000000000000000000047
:103140000000000000000048004800480048004817
:103150000048004800480048004800F8030000000C
:10316000000000000000000000000000000000005F
:1031700000000000000000000020002000200020CF
:10318000002000200020002000E00320002000E0BC
:10319000030000000000000000000000000000002C
:1031A000000000000000000000000000000000001F
:1031B0000000000000000000000000E003200020EC
:1031C00000E00320002000200000000000000000BC
:1031D00000000000000000000000000000000000EF
:1031E00000000000000000000000000000000000DF
:1031F00000F80348004800480048000000000000B4
:103200000000000000000000000000000000004876
:10321000004800480048004800480048004800486E
:10322000004800FF03480048004800480000000034
:10323000000000000000000000000000000000008E
:10324000002000200020002000200020002000207E
:1032500000FF0320002000FF0320002000200000CA
:10326000000000000000000000000000000000005E
:10327000000000200020002000200020002000206E
:10328000002000200020003F00000000000000009F
:10329000000000000000000000000000000000002E
:1032A000000000000000000000000000000000001E
:1032B00000000000000000E00320002000200020AB
:1032C00000200000000000000000000000000000DE
:1032D00000000000000000FF03FF03FF03FF03FFE7
:1032E00003FF03FF03FF03FF03FF03FF03FF03FFCE
:1032F00003FF03FF030000000000000000000000C7
:1033000000000000000000000000000000000000BD
:1033100000000000000000000000000000FF03FFAC
:1033200003FF03FF03FF0300000000000000000094
:1033300000000000000000000000001F001F001F30
:10334000001F001F001F001F001F001F001F001F85
:10335000001F001F001F001F0000000000000000F1
:10336000000000E003E003E003E003E003E003E02B
:1033700003E003E003E003E003E003E003E003E035
:1033800003E003E003E003E003E0030000000000CB
:103390000000000000000000000000FF03FF03FF2A
:1033A00003FF03FF03FF03FF03FF03FF03FF03000C
:1033B000000000000000000000000000000000000D
:1033C00000000000000000000000000000000000FD
:1033D0000000007700FF00CE01860186018601868D
:1033E00001CE01FE00760006000600060006000081
:1033F00000000000000000000000000000000000CD
:103400000000000000000000007C00FE00C7000378
:1034100000030003000300C700FE007C0000000062
:10342000000000000000000000000000000000009C
:103430000000000000000000000000DB00FF01FEB3
:1034400001B601B601B601B601B601B601B601007A
:10345000000000000000000000000000000000006C
:10346000000000000000000000000086018601CE80
:1034700001CC00CC00D80078007000300030003360
:10348000001F000E0000000000000000000000000F
:103490000000000000000000000000000018007E96
:1034A00000FF00DB00DB00DB00FF007E00180018DF
:1034B00000180000000000000000000000000000F4
:1034C00000000000000000000000000000000000FC
:1034D00000C300E70066003C0018003C003C0066AA
:1034E00000E700C300000000000000000000000032
:1034F00000000000000000000000000000000000CC
:10350000000000C300C300C300C300C300C300C366
:1035100000F300BF00DE00C000000000000000005B
:10352000000000000000000000000000000000009B
:103530000000000000C300C300C300C300FF00FE82
:1035400000C000C000C000C000000000000000007B
:10355000000000000000000000000000000000006B
:1035600000000000000000DB00DB00DB00DB00DB14
:1035700000DB00DB00DB00FF00C6000000000000F5
:10358000000000000000000000000000000000003B
:10359000000000000000000000DB00DB00DB00DBBF
:1035A00000DB00DB00DB00DB00FF00E6018001C088
:1035B000000000000000000000000000000000000B
:1035C00000000000000000000000000700070006E7
:1035D0000006007E00FE00C600C600FE007E000061
:1035E00000000000000000000000000000000000DB
:1035F00000000000000000000000000000830183C4
:1036000001830183019F01BF01B301B301BF019F8A
:1036100001000000000000000000000000000000A9
:103620000000000000000000000000000000000694
:1036300000060006000600FE00FE0186018601FE6F
:1036400001FE00000000000000000000000000007B
:10365000000000000000000000000000000000006A
:10366000003C007E00E600C000F800F800C000E664
:10367000007E003C00000000000000000000000090
:10368000000000000000000000000000000000003A
:10369000000000E300F3011B031B031F031F031BB8
:1036A000031B03F301E30000000000000000000022
:1036B000000000000000000000000000000000000A
:1036C00000000000007E00FF00C300C300C300FF35
:1036D00000FE00CC00C600C3000000000000000097
:1036E00000000000000000000000006C006C000002
:1036F00000FF00FF000300030003007F007F0003C2
:1037000000030003000300FF00FF000000000000B2
:1037100000000000000000000000000000000000A9
:103720000000006C006C0000003C007E00C700FF41
:10373000007F0003000300C700FE007C00000000C3
:103740000000000000000000000000000000000079
:103750000000000000000000000000000000000069
:10376000008001C0006000300018000C000600005E
:103770000000000000000000000000000000000049
:103780000000000000000000000000000000000039
:1037900000000006000C00180030006000C000802F
:1037A0000100000000000000000000000000000018
:1037B0000000000000000000008001C00060003038
:1037C0000018000C000600000000000000000000CF
:1037D00000000000000000000000000000000000E9
:1037E000000000000000000000000006000C0018AF
:1037F0000030006000C000800100000000000000F8
:1038000000000000000000000000000000000000B8
:1038100000000000000000000000000000000000A8
:10382000000000000030006000C000FE01FE01C08A
:1038300000600030000000000000000000000000F8
:103840000000000000000000000000000000000078
:1038500000000000000000300018000C00FE01FE17
:10386000010C001800300000000000000000000003
:103870000000000000000000000000000018001818
:103880000018001800180018001800180018001878
:10389000001800DB007E003C00180018000000004B
:1038A0000000000000000000000000000000001800
:1038B0000018003C007E00DB0018001800180018FB
:1038C0000018001800180018001800180018000050
:1038D00000000000000000000000000000000000E8
:1038E0000000000000000000000000000030003078
:1038F000000000FE01FE010000300030000000006A
:1039000000000000000000000000000000000000B7
:103910000000000000000000000000000018001877
:10392000001800FF00FF00180018000000FF00FF53
:103930000000000000000000000000000000000087
:1039400000000000000000000063036303670367DA
:10395000006F007B007B00730073007300630063E3
:1039600000630000000000000000000000000000F4
:103970000000000000000000000000000000000047
:103980000000008301FE007C00C600C600C6007C6B
:1039900000FE0083010000000000000000000000A5
:1039A0000000000000000000000000000000000017
:1039B000000000000000000000000000000000FC0B
:1039C00000FC00FC00FC0000000000000000000003
:1039D00000000000000000000000000000000000E7
:1039E00000000000000000000000000000000000D7
:1039F00000000000000000000000000000000000C7
:103A000000000000000000000000000000000000B6
:103A1000003C007E00FF00E700E700E700E700E76A
:103A200000E700E700FF007E003C0000000000000F
:103A30000000000000000000000000000000000086
:103A40000000001E001F001F001C001C001C001CAA
:103A5000001C001C001C007F007F007F0000000095
:103A60000000000000000000000000000000000056
:103A700000000000007E00FF00FF00E70070007003
:103A80000038001C000E000700FF00FF00FF0000D0
:103A90000000000000000000000000000000000026
:103AA000000000000000007C00FF00FF00E300E0D9
:103AB0000078007800F800E000E300FF00FF007CE1
:103AC00000000000000000000000000000000000F6
:103AD00000000000000000000078007C007C007EF8
:103AE000007E0077007700FF01FF01FF017000708A
:103AF0000070000000000000000000000000000056
:103B00000000000000000000000000FE00FE00FEBB
:103B10000007003B007F00E700E000E000E700FF57
:103B2000007F003E000000000000000000000000D8
:103B3000000000000000000000000000007C00FE0B
:103B400000FF00C70007003F007F00FF00E700E71D
:103B500000FF007E003C00000000000000000000AC
:103B6000000000000000000000000000000000FF56
:103B700000FF00FF0070007000380038001C001CBF
:103B8000000E000E0007000700000000000000000B
:103B90000000000000000000000000000000000025
:103BA000007E00FF00E700E700FF00FF007E00FF4F
:103BB00000E700E700FF00FF007E000000000000BB
:103BC00000000000000000000000000000000000F5
:103BD0000000003C007E00FF00E700E700FF00FE61
:103BE00000FC00E000E000FF007F003E000000005D
:103BF00000000000000000000000000000000000C5
:103C00000000000000E003F803FC039C039C039CFD
:103C100003FC03F803F003800380038003800300A8
:103C20000000000000000000000000000000000094
:103C30000000000000000007001F003F00390039AD
:103C40000039003F001F000F0001000100010001CA
:103C500000000000003D0E3D0E3D0E3D0E3D0E3DB0
:103C60000E3D0E3D0E3D0E3D0E3D0E3D0E3D0E3DFC
:103C70000E3D0E3D0E3D0E3D0E3D0E3D0E3D0E3DEC
:103C80000E3D0E3D0E3D0E3D0E3D0E3D0E3D0E3DDC
:103C90000E3D0E3D0E3D0E6F0EA10ED30E050F37DD
:103CA0000F690F9B0FCD0FFF0F311063109510C7D9
:103CB00010F9102B115D118F11C111F3112512573D
:103CC000128912BB12ED121F1351138313B513E7A0
:103CD0001319144B147D14AF14E114131545157703
:103CE00015A915DB150D163F167116A316D5160767
:103CF0001739176B179D17CF1701183318651897C9
:103D000018C918FB182D195F199119C319F519272E
:103D10001A591A8B1ABD1AEF1A211B531B851BB790
:103D20001BE91B1B1C4D1C7F1CB11CE31C151D47F4
:103D30001D791DAB1DDD1D0F1E411E731EA51ED757
:103D40001E091F3B1F6D1F9F1FD11F0320352067BA
:103D5000209920CB20FD202F2161219321C521F71F
:103D60002129225B228D22BF22F122232355238782
:103D700023B923EB231D244F248124B324E52417E6
:103D80002549257B25AD25DF25752643261126A748
:103D900026D9260B273D276F27A127D327052837AC
:103DA0002869289B28CD28FF28312963299529C710
:103DB00029F9292B2A5D2A8F2AC12AF32A252B5774
:103DC0002B892BBB2BED2B1F2C512C832CB52CE7D7
:103DD0002C192D4B2D7D2DAF2D452E132EE12D773A
:103DE0002EA92EDB2E0D2F3F2F712FA32FD52F079E
:103DF0003039306B309D30CF300131333165319700
:103E000031C931FB312D325F329132C332F5322765
:103E10003359338B33BD33EF33213453348534B7C7
:103E200034E9341B354D357F35B135E3351536472B
:103E3000367936AB36DD360F3741377337A537D78E
:103E40003709383B386D389F38D1380339353967F1
:103E5000399939CB393D0E3D0E3D0E3D0E3D0E3D9F
:103E60000E3D0E3D0E3D0E3D0E3D0E3D0E3D0E3DFA
:103E70000E3D0E3D0E3D0E3D0E3D0E3D0E3D0E3DEA
:103E80000E3D0E3D0E3D0E3D0E3D0E3D0E3D0E3DDA
:103E90000E3D0E3D0E3D0E6F0EA10ED30E050F37DB
:103EA0000F690F9B0FCD0FFF0F311063109510C7D7
:103EB00010F9102B11FD392F3A613A933AC53AF7B0
:103EC0003A293B5B3B8D3BBF3B51138313B513E753
:103ED0001319144B147D14AF14E114131545157701
:103EE00015A915DB150D163F167116A316D5160765
:103EF0001739176B179D17CF1701183318651897C7
:103F000018C918FB182D195F199119C319F519272C
:103F10001A591A8B1ABD1AEF1A211B531B851BB78E
:103F20001BE91B1B1C4D1C7F1CB11CE31C151D47F2
:103F30001D791DAB1DDD1D0F1E411E731EA51ED755
:103F40001E091F3B1F6D1F9F1FD11F0320352067B8
:103F5000209920CB20FD202F2161219321C521F71D
:103F60002129225B228D22BF22F122232355238780
:103F700023B923EB231D244F248124B324E52417E4
:103F80002549257B25AD25DF25752643261126A746
:103F900026D9260B273D276F27A127D327052837AA
:103FA0002869289B28CD28FF28312963299529C70E
:103FB00029F9292B2A5D2A8F2AC12AF32A252B5772
:103FC0002B892BBB2BED2B1F2C512C832CB52CE7D5
:103FD0002C192D4B2D7D2DAF2D452E132EE12D7738
:103FE0002EA92EDB2E0D2F3F2F712FA32FD52F079C
:103FF0003039306B309D30CF3001313331653197FE
:1040000031C931FB312D325F329132C332F5322763
:104010003359338B33BD33EF33213453348534B7C5
:1040200034E9341B354D357F35B135E33515364729
:10403000367936AB36DD360F3741377337A537D78C
:104040003709383B386D389F38D1380339353967EF
:1040500039F13B233C00000000000000000000009C
:104060000000000000000000000000000000000050
:104070000000000000000000000000000000000040
:10408000000000000000000000000000000E000E14
:10409000000E000E000E00060006000600060006D8
:1040A000000600060006000600000000000E001FCB
:1040B000001F000E00000000000000000000006370
:1040C00000630063006300630063006300630063D8
:1040D00000000000000000000000000000000000E0
:1040E00000000000000000000000000000000000D0
:1040F00000300630061002180318030801FE07FE00
:104100000708018C018400FF03FF038400C600C67A
:1041100000420042006300630000000000300030F5
:1041200000F800FE01B60337013300330036003ECD
:10413000003C00F000F001B00330033006300630E0
:10414000063203B703FE01FC0030003000300000EF
:1041500000000000001E003F007300630063006366
:1041600008730C3F078E03E00070003C078E0FC7FA
:104170000C610C600C600CE00CC00E8007000000AD
:10418000000000000000007800FC008E018601861F
:10419000018601C6006C003C0038006E0C660CC73E
:1041A0000CC30D830D030703068E0FFE0D780C0064
:1041B00000000000000000000003000300030003F3
:1041C00000030003000300030003000000000000E0
:1041D00000000000000000000000000000000000DF
:1041E00000000000000000000018000C000C000699
:1041F000000600060006000300030003000300039E
:10420000000300030006000600060006000C000C78
:1042100000180000000000000000000C001800184A
:10422000003000300030003000600060006000604E
:104230000060006000600030003000300030001886
:104240000018000C0000000000000000000000004A
:10425000000000000060006000600062046F0FFC5E
:10426000036000F00098010C030E07040200000038
:10427000000000000000000000000000000000003E
:10428000000000000000006000600060006000604E
:1042900000FF0FFF0F600060006000600060000022
:1042A000000000000000000000000000000000000E
:1042B00000000000000000000000000000000000FE
:1042C00000000000000000000000000000000000EE
:1042D00000000000003C003C001C001C000E000020
:1042E00000000000000000000000000000000000CE
:1042F0000000000000FF01FF0100000000000000BE
:1043000000000000000000000000000000000000AD
:10431000000000000000000000000000000000009D
:10432000000000000000000000000000000000008D
:104330000000000000000000000E001F001F000E23
:104340000000000000000000000003000380018066
:1043500001C000C00060006000300030001800188C
:104360000018000C000C0006000600030003000308
:1043700000000000000000000000007000FC018E42
:1043800003060307070306030603060306030603E3
:10439000060306030603060306070706038E01FC51
:1043A0000170000000000000000000000038003F25
:1043B0000037003000300030003000300030003076
:1043C000003000300030003000300030003000306D
:1043D00000FF01FF0100000000000000000000F8E5
:1043E00000FE030E03070603060306000600038013
:1043F00003C001E000700038001C000E000600033E
:10440000000300FF07FF070000000000000000009D
:1044100000F800FC030E0304070006000600070076
:10442000038003F000F0038003000700060006028B
:104430000607078603FE03F80000000000000000E6
:10444000000000C001E001A001B0019001980198B6
:10445000018C018C018601860183018301FF0FFF1E
:104460000F800180018001800180010000000000B8
:104470000000000000FC03FC030C000C000400061C
:1044800000F600FE038E0306070006000600060085
:10449000060006020607078603FE01F8000000007A
:1044A00000000000000000F801FC070E02060006F4
:1044B000000300F300FF038F03070703060306034F
:1044C0000603060306030606038E03FC01F800003C
:1044D000000000000000000000FF03FF0300038055
:1044E000018001C000C0006000600060003000304A
:1044F000001800180018000C000C000C0006000644
:104500000000000000000000000000F800FE0306AC
:1045100003070703060306030607070603FC01FC5F
:10452000010603070703060306030607070603FE43
:1045300003F80000000000000000000000F800FC8C
:10454000018E0306030306030603060306030603A0
:104550000607078E07FE06780600060003000382A2
:1045600003FF017C000000000000000000000000CC
:1045700000000000000E001F001F000E00000000E1
:1045800000000000000000000000000E001F001FDF
:10459000000E00000000000000000000000000000D
:1045A000000000000000001C003E003E001C000057
:1045B000000000000000000000000000003C003C83
:1045C000001C001C000E000E00060007000000008A
:1045D0000000000000000000000008000E800FF046
:1045E000017C000F0003000F007C00F001800F0031
:1045F0000E000800000000000000000000000000A5
:1046000000000000000000000000000000FF07FFA5
:10461000070000000000000000FF07FF0700000087
:10462000000000000000000000000000000000008A
:104630000000000000000000000000000001000772
:10464000001F00F800E003000F000C000FE003F86B
:10465000001F000700010000000000000000000033
:10466000000000000000007C00FE00C70182018005
:104670000180018001C0006000300018001800189F
:1046800000180000000000000038007C007C0038AA
:10469000000000000000000000F000FC030C070612
:1046A00006060C030CC30DE30F630C330C330C3301
:1046B0000C330C330CE30EC307060006000E00FC9F
:1046C00000F0010000000000000000000070007019
:1046D000007000D800D800D8008C018C018C018CAF
:1046E0000106030603FE03FE030306030603060397
:1046F0000603060306000000000000000000007F23
:1047000000FF018301030303030303030383038304
:1047100001FF00FF018303030703060306030603EB
:10472000068303FF03FF00000000000000000000FC
:1047300000F801FC030E0306060706030603000348
:104740000003000300030003000300030003060747
:104750000606060E03FC03F801000000000000003E
:104760000000007F00FF0183030303030703060328
:1047700006030603060306030603060306030603F1
:1047800006030703038303FF017F0000000000000E
:104790000000000000FF07FF070300030003000301
:1047A00000030003000300FF01FF010300030003F7
:1047B000000300030003000300FF07FF07000000E1
:1047C00000000000000000FF07FF070300030003D4
:1047D000000300030003000300FF01FF01030003C7
:1047E00000030003000300030003000300030000B4
:1047F000000000000000000000F801FC030E0306AA
:1048000006070603000300030003000300C307C3F9
:1048100007030603060306070606070E07FC05F84E
:10482000040000000000000000000003060306036F
:1048300006030603060306030603060306FF07FF37
:10484000070306030603060306030603060306031F
:1048500006030600000000000000000000FF00FF4B
:104860000018001800180018001800180018001888
:104870000018001800180018001800180018001878
:1048800000FF00FF0000000000000000000000E04A
:1048900007E0070006000600060006000600060006
:1048A00006000600060006030603060306030607C5
:1048B000070603FE03F800000000000000000000EF
:1048C000000302030783038301C300630073003303
:1048D000001B000F001B003B0073006300C300C3FC
:1048E0000183030307030E030C0000000000000017
:1048F00000000003000300030003000300030003A3
:10490000000300030003000300030003000300038F
:1049100000030003000300FF07FF07000000000082
:104920000000000000030C030C070E0F0F0F0F9B7D
:104930000D9B0DF30CF30C630C630C630C030C0365
:104940000C030C030C030C030C030C030C00000001
:104950000000000000000003060306070607060F1C
:10496000060F061B061B063306330663066306C3E3
:1049700006C306830783070307030703060306002E
:10498000000000000000000000F800FC018E03069B
:1049900003070703060306030603060306030603CD
:1049A00006030603060306070706038E03FC01F849
:1049B0000000000000000000000000FF00FF0303F3
:1049C000070306030603060306030603060307FFA1
:1049D00003FF0003000300030003000300030003C0
:1049E00000030000000000000000000000F800FCD0
:1049F000018E0306030707030603060306030603E7
:104A00000603060306030603060306070706038ECE
:104A100003FC01F80180030003000000000000FF18
:104A200000FF0383030306030603060306030603CE
:104A300003C303FF017F00E300C300C3018301033D
:104A40000303070306030E0000000000000000003F
:104A500000F800FE01860307010300070006001EA0
:104A6000003800F000E001800300030007000600AA
:104A70000602078703FE03FC0000000000000000A0
:104A8000000000FF0FFF0F6000600060006000602A
:104A90000060006000600060006000600060006016
:104AA0000060006000600060006000000000000026
:104AB00000000000000306030603060306030603C6
:104AC000060306030603060306030603060306039E
:104AD000060306070706038E03FC01F8000000002A
:104AE00000000000000000030C030C030C06060687
:104AF0000606060C030C030C030C0398019801989E
:104B0000019801F000F000F000600060006000001B
:104B1000000000000000000000030C030C030C0365
:104B20000C030C630C660666066606660666066679
:104B3000066606F6069606960696069C030C030C79
:104B400003000000000000000000000E070C030C32
:104B50000398019801F00060006000600060006050
:104B600000F000F000980198010C030C0306060603
:104B700006070E00000000000000000000070E06FF
:104B80000606060C030C030C03980198019000F034
:104B900000F0006000600060006000600060006085
:104BA000006000600000000000000000000000FF46
:104BB00007FF07000380038001C000C000E0006021
:104BC0000030003000380018000C000C000E000609
:104BD000000300FF07FF07000000000000000000C6
:104BE00000FF00FF000300030003000300030003B5
:104BF000000300030003000300030003000300039D
:104C00000003000300FF00FF0000000000000000A0
:104C1000000000030003000300060006000C000C67
:104C2000001800180018003000300060006000C05C
:104C300000C00080018001000300030000000000AC
:104C40000000000000FF00FF00C000C000C000C066
:104C500000C000C000C000C000C000C000C000C054
:104C600000C000C000C000C000FF00FF0000000046
:104C70000000000000000060006000F00098010CDF
:104C8000030606030C0108000000000000000000FD
:104C90000000000000000000000000000000000014
:104CA0000000000000000000000000000000000004
:104CB00000000000000000000000000000000000F4
:104CC00000000000000000000000000000000000E4
:104CD00000FF7FFF7F00000000000006001F007C37
:104CE00000E00000000000000000000000000000E4
:104CF00000000000000000000000000000000000B4
:104D000000000000000000000000000000000000A3
:104D100000000000000000FC00FE0184030003000E
:104D2000037C03FE03060303030303030303038758
:104D300007FE0E7C0C0000000000000000060006CC
:104D4000000600060006000600E600F6019E030EBF
:104D500003060606060606060606060606060606F6
:104D6000039E03F701E300000000000000000000C4
:104D70000000000000000000000000F801FC030E2D
:104D80000306030302030003000300030003000300
:104D90000006020E07FC03F80100000000000000FE
:104DA0000000030003000300030003000338037C3A
:104DB00003CE038603030303030303030303030375
:104DC00003030306038E03FC063806000000000000
:104DD000000000000000000000000000000000F8DB
:104DE00000FC018E03060303060306FF07FF07030B
:104DF000000300030006000E02FC07F8010000009B
:104E000000000000000000C003E00F70043000301C
:104E1000003000FF03FF033000300030003000306E
:104E20000030003000300030003000300030000032
:104E3000000000000000000000000038067C07CEE3
:104E4000030603030303030303030303030303032F
:104E5000030603CE037C03380300030003800384AE
:104E600001FE0178000000000000000300030003C1
:104E70000003000300F300FB018B030F0307030390
:104E800003030303030303030303030303030303F2
:104E90000303030000000000000000000038003899
:104EA000000000000000003F003F003000300030F4
:104EB0000030003000300030003000300030003072
:104EC000003000300000000000000000000000C0C2
:104ED00001C0010000F801F801800180018001801B
:104EE00001800180018001800180018001800183B7
:104EF000018301C301C600FE007C00000000000029
:104F00000003000300030003000300030E030783F4
:104F100003C301C300630033003F0077006300C395
:104F200000830183030307030E000000000000005C
:104F30000000003F003F0030003000300030003003
:104F400000300030003000300030003000300030E1
:104F50000030003000300030003000000000000061
:104F6000000000000000000000000000000000330E
:104F7000063B0FEF0D630C630C630C630C630C6357
:104F80000C630C630C630C630C630C630C0000007B
:104F90000000000000000000000000000000000011
:104FA00000E301F70336071E060E06060606060690
:104FB0000606060606060606060606060606060097
:104FC00000000000000000000000000000000000E1
:104FD000000000F800FC018E03060303060306032D
:104FE00006030603060306030606038E03FC01F808
:104FF00000000000000000000000000000000000B1
:1050000000E300F7019E03060306060606060606F1
:10501000060606060606060E039E03F601E60006D1
:10502000000600060006000000000000000000006E
:1050300000000038067C07CE0306030303030303C6
:105040000303030303030303038603CE037C033834
:105050000300030003000300030000000000000041
:10506000000000000000000000C703E607760E1CE9
:105070000C1C0C1C000C000C000C000C000C000C98
:10508000000C000C000C00000000000000000000FC
:105090000000000000000000000000FC00FE01878E
:1050A000000300030006003E00FC00E00180030056
:1050B0000300038603FF01FC000000000000000065
:1050C00000000000001800180018001800FF03FF7F
:1050D000031800180018001800180018001800180D
:1050E00000180018023807F003E00100000000007B
:1050F00000000000000000000000000000000003AD
:10510000030303030303030303030303030303036F
:105110000303038303C30347037E073C0600000029
:10512000000000000000000000000000000000007F
:1051300000030607070603060306038C018C018C97
:10514000018C01D800D800D8005000700070000019
:10515000000000000000000000000000000000004F
:10516000000000034C034C034C630C630C630C63A2
:105170000C630CF606F606960696069C030C030CCA
:10518000030000000000000000000000000000001C
:1051900000000000000E070C0398019801F000F0D9
:1051A0000060006000F000F000980198010C030618
:1051B00006070E00000000000000000000000000D4
:1051C00000030C030C0606060606030C030C038CF6
:1051D000019801D800D800D800700060006000601D
:1051E00000600033003F000E0000000000000000DF
:1051F000000000000000000000FF07FF0700038020
:1052000001C001C00060007000300018001C000CDC
:10521000000600FF07FF070000000000000000007C
:1052200000E000700030003000300030003000300E
:105230000018000F000F0018003000300030003060
:1052400000300030007000E00000000000000000AE
:105250000000000300030003000300030003000339
:105260000003000300030003000300030003000326
:105270000003000300030003000300030003000019
:1052800000000000000E001C001800180018001894
:1052900000180018003000E001E00130001800188C
:1052A0000018001800180018001C000E0000000074
:1052B000000000000000003C087F0CC30F810700C5
:1052C00000000000000000000000000000000000DE
:1052D00000000000000000000000000000000000CE
:1052E00000000000000000000000000000000000BE
:1052F00000000000000000000000000000000000AE
:10530000000000000000000000000000000000009D
:10531000000000000000000000000060006000606D
:1053200000F000F000F00098019801980198010C3D
:10533000030C03FC03FC03060606060606030C0327
:105340000C030C00000000000000000000FF07FF3D
:1053500007030603040300030003000300FF00FF2C
:1053600001830303070306030603060306030683FC
:1053700003FF03FF00000000000000000000007FAA
:1053800000FF018301030303030303030383038378
:1053900001FF00FF0183030307030603060306035F
:1053A000068303FF03FF0000000000000000000070
:1053B00000FF07FF070306030403000300030003C5
:1053C00000030003000300030003000300030003C5
:1053D00000030003000300030000000000000000C1
:1053E0000000008003C003600360036003700330AB
:1053F000033003300338031803180318031C030C8D
:10540000030C030C030C03FF0FFF0F030C0204003B
:105410000000000000FF07FF070300030003000374
:1054200000030003000300FF01FF0103000300036A
:10543000000300030003000300FF07FF0700000054
:1054400000000000000000630C630C630C6606663D
:105450000666066C036C03F801F000F000F8016CBE
:10546000036C03660666066606630C630C630C0039
:105470000000000000000000007000FC018C03062A
:105480000302030003000300038001F000F80100A1
:1054900003000600060006020603060707FE03FCDB
:1054A00001000000000000000000000306030603E6
:1054B00007030783078307C306C306630663063330
:1054C00006330633061B061B060F060706070603F0
:1054D00006030600000000000070007000030603D1
:1054E00006030783078307C306C306C30663066371
:1054F000063306330633061B061B060F0607060790
:105500000603060306000000000000000000000380
:1055100003030383018301C300C300630063007FAF
:10552000007F00C300C3008301830103030303035F
:10553000060306030C030C0000000000000000003E
:1055400000C007F007300638061806180618061CB3
:10555000060C060C060C060E0606060606060606D1
:105560000603060306030603060000000000000011
:10557000000000030C030C070E0F0F0F0F9B0D9B79
:105580000DF30CF30C630C630C630C030C030C03A2
:105590000C030C030C030C030C030C0000000000B4
:1055A00000000000000306030603060306030603CB
:1055B00006030603060306FF07FF070306030603A9
:1055C000060306030603060306030603060000009F
:1055D00000000000000000F800FC018E0306030735
:1055E0000703060306030603060306030603060372
:1055F0000603060306070706038E03FC01F80000F6
:10560000000000000000000000FF07FF0703060382
:105610000603060306030603060306030603060342
:105620000603060306030603060306030603060332
:105630000600000000000000000000FF00FF030360
:10564000070306030603060306030603060307FF14
:1056500003FF000300030003000300030003000333
:1056600000030000000000000000000000F801FC42
:10567000030E0306060706030603000300030003E8
:105680000003000300030003000306070606060EDE
:1056900003FC03F80100000000000000000000FF10
:1056A0000FFF0F600060006000600060006000603D
:1056B00000600060006000600060006000600060EA
:1056C00000600060006000000000000000000000BA
:1056D0000003060306030603060306030603060388
:1056E0000603060706FE07F8070006000600060187
:1056F0000603060707FE03FC01000000000000008F
:10570000000000FC03FE07670E630C630C630C6370
:105710000C630C630C630C670EFE07FC03600060F7
:105720000060006000600060006000000000000099
:105730000000000000030C030C060606060C030C18
:105740000398019801F00060006000F00098019853
:10575000010C030C0306060606030C030C000000F4
:10576000000000000000000303030303030303031E
:1057700003030303030303030303030303030303F9
:105780000303030303030303030303FF0FFF0F00DC
:105790000C000400000000000003060306030603DB
:1057A000060306030603060306030603060706FEB2
:1057B00007F80700060006000600060006000600BF
:1057C0000600000000000000000000030C030C6352
:1057D0000C630C630C630C630C630C630C630C6351
:1057E0000C630C630C630C630C630C630C630CFFA5
:1057F0000FFF0F0000000000000000000003030383
:1058000003330333033303330333033303330333E8
:1058100003330333033303330333033303330333D8
:1058200003FF0FFF0F000C00040000000000000346
:10583000000300030003000300030003000300FF54
:1058400000FF03030703060306030603060306031C
:10585000060307FF03FF0000000000000000000037
:105860000003180318031803180318031803180378
:10587000187F18FF188319831983198319831983D3
:105880001983198319FF187F180000000000000019
:105890000000001F001F0019001800180018001851
:1058A000001800F803F807180E180C180C180C183C
:1058B0000C180C180C180EF807F803000000000074
:1058C0000000000000FC00FE018603030303070341
:1058D00006000600060006F007F0070006000600B6
:1058E000060306030703038603FE01FC0000000015
:1058F000000000000000008303C307E30E630C7385
:105900005C33583358335833583F583F5833583323
:105910005833583358735C630CE30EC3078303009A
:10592000000000000000000000F00FFC0F0E0C064D
:105930000C060C060C060C060C0C0C3C0CF80FE0CC
:105940000F700C300C380C180C0C0C0E0C060C07DD
:105950000C0000000000000000000000000000003B
:105960000000000000FC00FE018403000300037C33
:1059700003FE03860303030303030303038707FEF6
:105980000E7C0C00000000000000008601CF01FB2F
:105990000003000E001C007000FC00CE0186010315
:1059A000030303030303030303030303038701CE7A
:1059B00001FC00780000000000000000003C007EB8
:1059C00000630033001B000F007700FB00C7018756
:1059D0000103030303030303030303030303038616
:1059E00001CE01FC00780000000000000000000073
:1059F00000000000000000000000007E00FF00C268
:105A000001800180018001F001FC001E00070003FD
:105A10000003008701FE03FC0000000000000000FE
:105A20000000003C00F800C0018001000338037C46
:105A300003CE0386030303030303030303030303E8
:105A40000303038601CE01FC007800000000000083
:105A5000000000000000000000000000000000F84E
:105A600000FC018E03060303060306FF07FF07037E
:105A7000000300030006000E02FC07F8010000000E
:105A80000000000000000000000000000000000016
:105A900000630C66066606FC03F0006000F000FC84
:105AA000036606660666066606670E630C630C00F0
:105AB00000000000000000000000000000000000E6
:105AC000000000F800FC018E03060304038001F0CF
:105AD00000F00100030006000601078303FE01FC3D
:105AE00000000000000000000000000000000000B6
:105AF0000000000000030303030303030303030385
:105B00000303030303030303038303830347037EA6
:105B1000073C06000000000000000000000000003C
:105B200000000078003000030303030303030303B2
:105B300003030303030303030303038303C30347B1
:105B4000037E063C0600000000000000000000008C
:105B500000000000000000000003078303C301E30E
:105B600000630033001B003F0077006300C3008325
:105B70000183030307030E00000000000000000083
:105B80000000000000000000000000E007F007181F
:105B9000061806180618060C060C060C060406065F
:105BA00006060606060306030600000000000000C5
:105BB00000000000000000000000000000030C07CF
:105BC0000E0F0F9B0D9B0DF30CF30C630C630C037A
:105BD0000C030C030C030C030C030C00000000006E
:105BE00000000000000000000000000000000003B2
:105BF0000603060306030603060306FF07FF070363
:105C00000603060306030603060306030600000058
:105C10000000000000000000000000000000000084
:105C200000F800FC018E03060303060306030603C7
:105C30000603060306030606038E03FC01F80000B4
:105C40000000000000000000000000000000000054
:105C5000000000FF07FF0703060306030603060311
:105C600006030603060306030603060306030603EC
:105C700006000000000F0F0F0F0F0F0F0F0F0F0088
:105C80000000000000000000000F0F0F0F0F0F0FAB
:105C90000F0F0F000000000000000000000F0F0FAA
:105CA0000F0F0F0F0F0F0F0F0F0F0F0F0F0F0F0F04
:105CB0000FF0F0F0F0F0F0F0F0F0F00F0F0F0F0F2A
:105CC0000F0F0F0F0FF0F0F0F0F0F0F0F0F0F00F1A
:105CD0000F0F0F0F0F0F0F0F0FFFFFFFFFFFFFFF44
:105CE000FF0F0F0F0F0F0F0F0F0F0F0F0FFFFFFF04
:105CF000FFFFFFFFFF0F0F0F0F0F0F0F0F0F0F0F04
:105D00000FFFFFFFFFFFFFFFFF0F0F8001800180EC
:105D1000018001800180018001800180018001807B
:105D2000018001800180018001800180018001806B
:105D3000018001800180018001800180018001805B
:105D4000018001800180018001800180018001804B
:105D5000018001800180018001FF01FF018001803D
:105D6000018001800180018001800180018001802B
:105D7000018001800180018001800180018001801B
:105D80000180018001FF01FF01800180018001FF8E
:105D900001FF01800180018001800180018001807C
:105DA0000130063006300630063006300630063048
:105DB000063006300630063006300630063F063F15
:105DC0000630063006300630063006300630063023
:105DD0000630060000000000000000000000000087
:105DE000000000000000000000000000000000FFB4
:105DF00007FF073006300630063006300630063022
:105E00000630063006000000000000000000000020
:105E10000000000000000000000000FF01FF018002
:105E20000180018001FF01FF01800180018001806C
:105E300001800180018001300630063006300630D6
:105E4000063006300630063006300630063F063F84
:105E5000060006000600063F063F06300630063004
:105E60000630063006300630063006300630063082
:105E70000630063006300630063006300630063072
:105E80000630063006300630063006300630063062
:105E900006300630063006300630060000000000EE
:105EA00000000000000000000000000000000000F2
:105EB00000FF07FF070006000600063F063F06300A
:105EC0000630063006300630063006300630063022
:105ED0000630063006300630063006300630063012
:105EE0000630063F063F06000600060006FF07FFD5
:105EF000070000000000000000000000000000306B
:105F000006300630063006300630063006300630E1
:105F10000630063006300630063006FF07FF070061
:105F20000000000000000000000000000000000071
:105F3000008001800180018001800180018001805A
:105F400001800180018001FF01FF0180018001804B
:105F500001FF01FF01000000000000000000000040
:105F60000000000000000000000000000000000031
:105F700000000000000000000000000000FF01FF22
:105F80000180018001800180018001800180018009
:105F900001800180018001800180018001800180F9
:105FA00001800180018001800180018001800180E9
:105FB0000180FF80FF0000000000000000000000E2
:105FC000000000000000008001800180018001804D
:105FD00001800180018001800180018001800180B9
:105FE000018001FFFFFFFF00000000000000000033
:105FF00000000000000000000000000000000000A1
:106000000000000000000000000000000000000090
:106010000000000000FFFFFFFF8001800180018081
:106020000180018001800180018001800180018068
:106030000180018001800180018001800180018058
:106040000180018001800180FF80FF80018001804C
:106050000180018001800180018001800100000039
:106060000000000000000000000000000000000030
:10607000000000000000000000FFFFFFFF00000024
:106080000000000000000000000000000000008090
:1060900001800180018001800180018001800180F8
:1060A0000180018001800180018001FFFFFFFF80EE
:1060B00001800180018001800180018001800180D8
:1060C00001800180018001800180018001800180C8
:1060D0000180018001800180FF80FF8001800180BC
:1060E0000180FF80FF8001800180018001800180AC
:1060F00001800130063006300630063006300630AA
:1061000006300630063006300630063006300630DF
:10611000FE30FE30063006300630063006300630DF
:1061200006300630063006300630063006300630BF
:10613000063006300630063006300630FE30FE30BF
:106140000030003000F0FFF0FF0000000000000011
:10615000000000000000000000000000000000003F
:1061600000000000000000000000000000F0FFF050
:10617000FF30003000300030FE30FE300630063098
:10618000063006300630063006300630063006305F
:106190000630063006300630063006300630063F40
:1061A000FE3FFE000000000000FFFFFFFF000000B8
:1061B00000000000000000000000000000000000DF
:1061C00000000000000000000000000000000000CF
:1061D00000FFFFFFFF0000000000003FFE3FFE3019
:1061E00006300630063006300630063006300630FF
:1061F00006300630063006300630063006300630EF
:1062000006300630FE30FE30003000300030FE3008
:10621000FE30063006300630063006300630060006
:10622000000000000000000000000000000000006E
:106230000000000000FFFFFFFF000000000000FF63
:10624000FFFFFF0000000000000000000000000051
:106250000030063006300630063006300630063094
:10626000063006300630063FFE3FFE00000000000C
:10627000003FFE3FFE300630063006300630063066
:10628000063006800180018001800180018001804C
:10629000018001800180018001FFFFFFFF000000FD
:1062A000000000FFFFFFFF000000000000000000F2
:1062B00000000000003006300630063006300630A0
:1062C000063006300630063006300630063006301E
:1062D00006FFFFFFFF0000000000000000000000BC
:1062E00000000000000000000000000000000000AE
:1062F00000000000000000000000000000FFFFFFA1
:10630000FF000000000000FFFFFFFF800180018010
:106310000180018001800180010000000000000078
:10632000000000000000000000000000000000006D
:106330000000000000FFFFFFFF300630063006308F
:10634000063006300630063006300630063006309D
:10635000063006300630063006300630063006308D
:1063600006300630063006F0FFF0FF0000000000A7
:10637000000000000000000000000000008001801C
:106380000180018001800180018001800180018005
:1063900001800180FF80FF80018001800180FF80FB
:1063A000FF000000000000000000000000000000EE
:1063B00000000000000000000000000000000000DD
:1063C000000000000080FF80FF80018001800180CC
:1063D000FF80FF80018001800180018001800180B9
:1063E00001000000000000000000000000000000AC
:1063F00000000000000000000000000000F0FFF0BE
:10640000FF300630063006300630063006300630E3
:1064100006300630063006300630063006300630CC
:10642000063006300630063006300630063006FFED
:10643000FFFFFF30063006300630063006300630EB
:1064400006300630068001800180018001800180D5
:106450000180018001800180018001FFFFFFFF803A
:106460000180018001FFFFFFFF800180018001802A
:106470000180018001800180018001800180018014
:106480000180018001800180018001800180018004
:10649000018001FF01FF010000000000000000007A
:1064A00000000000000000000000000000000000EC
:1064B00000000000000000000000000000000000DC
:1064C00000000080FF80FF8001800180018001804A
:1064D0000180018001800180018001FFFFFFFFFF3B
:1064E000FFFFFFFFFFFFFFFFFFFFFFFFFFFFFFFFBC
:1064F000FFFFFFFFFFFFFFFFFFFFFFFFFFFFFFFFAC
:10650000FFFFFFFFFFFFFFFFFFFFFFFFFF00000098
:10651000000000000000000000000000000000007B
:106520000000000000000000000000FFFFFFFFFF70
:10653000FFFFFFFFFFFFFFFFFFFFFFFFFFFFFFFF6B
:1065400000FF00FF00FF00FF00FF00FF00FF00FF53
:1065500000FF00FF00FF00FF00FF00FF00FF00FF43
:1065600000FF00FF00FF00FF00FF00FF00FF00FF33
:106570000000C000C000C080FF80FF80FF80FF805F
:10658000FF80FF80FF80FF80FF80FF80FF80FF8013
:10659000FF80FF80FF80FF80FF80FF80FF80FF8003
:1065A000FF80FF000000000000000000000000006D
:1065B00000000000000000000000000000000000DB
:1065C00000FF7FFF7FFF7FFF7FFF7FFF7FFF7FFF5A
:1065D0007FFF7FFF7F000000000000000000000040
:1065E00000F300FB030F0707060306030603060379
:1065F0000603060306030603060707FF03FB000363
:106600000003000300030000000000000000000081
:1066100000000000000000F801FC030E0306030365
:106620000203000300030003000300030006020E40
:1066300007FC03F80100000000000000000000005B
:10664000000000000000000000FF0FFF0F630C625D
:106650000460006000600060006000600060006036
:10666000006000600060000000000000000000000A
:106670000000000000000000000000030603060305
:106680000603060306030603078707FE07FC06004A
:106690000601060307FE03FC0100000000000000E5
:1066A000000000000000000000000000006000F892
:1066B00001FE07670E630C630C630C630C670EFE30
:1066C00007F801600060006000600000000000004A
:1066D0000000000000000000000000000000000EAC
:1066E0000E0C061C071803B001B001E000E000B07A
:1066F00001B00118031C070C06060C071C00000063
:106700000000000000000000000000000000000089
:106710000003060306030603060306030603060337
:106720000603060306030603078707FE1E781E00FE
:106730001800080000000000000000000000000039
:106740000000000306030603060306030603060310
:10675000060706FE07F8070006000600060006000A
:106760000600000000000000000000000000000023
:106770000000000000630C630C630C630C630C638B
:106780000C630C630C630C630C630C630C730EEFF3
:106790004DC64C000000000000000000000000009A
:1067A00000000000000000630C630C630C630C63CA
:1067B0000C630C630C630C630C630C630C630C7351
:1067C0000EEF0DC65C0058005800000000000000ED
:1067D0000000000000000000000F000F000C000C83
:1067E000000C000C00CC03EC073C0E1C0C0C0C0C39
:1067F0000C0C0EFC07F80300000000000000000075
:1068000000000000000000000000000358035803CF
:1068100058035803580358F358FB598F5B075B0321
:106820005B035B835BFF59FE580000000000000023
:106830000000000000000000000000000003000352
:10684000000300030003000300F300FB030F07072E
:1068500006030603060307FF03FE01000000000015
:106860000000000000000000000000000000007CAC
:1068700000FE00C701830101030003C803FC0338C5
:1068800003000300038301C701FE007C0000000039
:1068900000000000000000000000000000000000F8
:1068A000008301C30363066306334C334C3F4C3F04
:1068B0004C334C334C334C63066306C303830100F3
:1068C00000000000000000000000000000000000C8
:1068D000000000F807FC0706060306030603060788
:1068E00006FE07F8076006300618060C06060603C3
:1068F0000600000000000000000000980198010060
:1069000000FF07FF0703000300030003000300FF6D
:1069100000FF00030003000300030003000300FF67
:1069200007FF07000000000000000000000000005A
:1069300000980198010000F800FC018E0306030393
:106940000603060306FF07FF070300030006020E07
:1069500007FC03F801000000000000000000000038
:106960000000000000000000000000000000000027
:10697000000000000000038001C00060003000182B
:10698000000C0006000300000000000000000000F2
:1069900000000000000000000000000000000000F7
:1069A0000000000000030006000C0018003000602A
:1069B00000C000800100030006000000000000008D
:1069C000000000000600038001C0006000300018D5
:1069D000000C0006000300000000000000000000A2
:1069E00000000000000000000000000000000000A7
:1069F0000000000000030006000C001800300060DA
:106A000000C000800100030006000000000000003C
:106A10000000000000000000000000000000000076
:106A20000000000000000000000000000000000066
:106A300000C00080010003FF07FF0700038001C0C2
:106A40000000000000000000000000000000000046
:106A50000000000000000000000000000000000036
:106A600000000018000C000600FF07FF0706000CDE
:106A700000180000000000000000000000000000FE
:106A80000000000000000000000000000000000006
:106A90000000000000000030003000300030003006
:106AA0000031023303B601FC007800300000000022
:106AB00000000000000000000000000000000000D6
:106AC00000000000000000000030007800FC00B66C
:106AD000013303310230003000300030003000005C
:106AE00000000000000000000000000000000000A6
:106AF000000000000000003000300000000000FF37
:106B000007FF070000000030003000000000000018
:106B10000000000000000000000000000000000075
:106B200000600060006000600060006000FF0FFF18
:106B30000F60006000600060006000600000000006
:106B400000FE0FFE0F00000000000000000000002B
:106B5000000000835D835583558755875D87018FCE
:106B6000018F019B019B019B01B301B301E301E391
:106B700001C301C301830183018301000000000000
:106B8000000000000000000000000000000318F3F7
:106B900019FC070E0E060C060C060C060C0E0EFC5D
:106BA00007F31903180000000000000000000000B7
:106BB00000000000000000000000000000000000D5
:106BC000000000000000007F007F007F0000000048
:106BD00000000000000000000000000000000000B5
:106BE00000000000000000000000000000000000A5
:106BF0000000000000000000000000000000000095
:106C00000000000000000000000000000000000084
:106C100000000000000000000000007000FC01FE09
:106C2000038E038F070707070707070707070707ED
:106C30000707070707070707078F078E03FE01FCF3
:106C40000170000000000000000000000038003F5C
:106C5000003F003B0038003800380038003800386A
:106C6000003800380038003800380038003800FF9D
:106C700001FF01FF0100000000000000000000F81B
:106C800000FE03FE030F070707070700078003C086
:106C900003E001F00078003C001E000F0007000731
:106CA00000FF07FF07FF07000000000000000000D2
:106CB00000F800FC03FE038C0700070007000780B4
:106CC00003C003F001F003E003800700070007069C
:106CD000078F07FE03FE03F800000000000000001D
:106CE000000000C001E001E001F001F001F801D86E
:106CF00001DC01DC01CE01CE01C701FF0FFF0FFF58
:106D00000FC001C001C001C001C0010000000000AF
:106D10000000000000FC03FC03FC031C000C000E40
:106D200000FE00FE01FE038E0700070007000700BB
:106D300007000706078F07FE03FE01F800000000AA
:106D400000000000000000F801FC079E070E000E86
:106D5000000700F700FF03FF038F07070707070778
:106D6000070707070707078E03FE03FC01F800006B
:106D7000000000000000000000FF03FF03FF03C04D
:106D800001C001E000E000700070007000380038C1
:106D9000001C001C001C000E000E000E0007000767
:106DA0000000000000000000000000F800FE03FEEC
:106DB000038F070707070707078F07FE03FC01FC80
:106DC00001FE038F070707070707078F07FE03FE6C
:106DD00003F80000000000000000000000F800FCC4
:106DE00001FE038E030707070707070707070707C3
:106DF000078F07FE07FE077807000780038003FE62
:106E000003FF017C00000000000000000000000003
:106E1000F000F0C0FFE0FFF0FFF8F878F078F078CD
:106E2000F078F078F0F0F8E0FFC0FF80FF00F000AD
:106E3000F000F000F000F000F000F00000000000B2
:106E40000003000300FF00FF01FF03C70783078360
:106E500007830783078307C703FF01FF007F000342
:106E60000003000300030003000300030055405526
:106E7000405540554055405540554055405540556A
:106E8000405540554055405540554055405540555A
:106E9000405540554055405540554055405540554A
:106EA0004055405540554055405540554055408708
:106EB00040B940EB401D414F418141B341E541178D
:106EC0004249427B42AD42DF42114343437543A7EF
:106ED00043D9430B443D446F44A144D34405453753
:106EE0004569459B45CD45FF45314663469546C7B7
:106EF00046F9462B475D478F47C147F3472548571B
:106F0000488948BB48ED481F4951498349B549E77D
:106F100049194A4B4A7D4AAF4AE14A134B454B77E0
:106F20004BA94BDB4B0D4C3F4C714CA34CD54C0744
:106F30004D394D6B4D9D4DCF4D014E334E654E97A6
:106F40004EC94EFB4E2D4F5F4F914FC34FF54F270C
:106F50005059508B50BD50EF50215153518551B76E
:106F600051E9511B524D527F52B152E352155347D2
:106F7000537953AB53DD530F5441547354A554D735
:106F80005409553B556D559F55D155035635566798
:106F9000569956CB56FD562F5761579357C557F7FD
:106FA000578D585B582958BF58F158235955598760
:106FB00059B959EB591D5A4F5A815AB35AE55A17C4
:106FC0005B495B7B5BAD5BDF5B115C435C755CA726
:106FD0005CD95C0B5D3D5D6F5DA15DD35D055E378A
:106FE0005E695E9B5ECD5EFF5E315F635F955FC7EE
:106FF0005F5D602B60F95F8F60C160F36025615752
:10700000618961BB61ED611F6251628362B562E7B4
:107010006219634B637D63AF63E163136445647717
:1070200064A964DB640D653F657165A365D565077B
:107030006639666B669D66CF6601673367656797DD
:1070400067C967FB672D685F689168C368F5682743
:107050006959698B69BD69EF69216A536A856AB7A5
:107060006AE96A1B6B4D6B7F6BB16BE36B554055E7
:107070004055405540554055405540554055405568
:107080004055405540554055405540554055405558
:107090004055405540554055405540554055405548
:1070A0004055405540554055405540554055408706
:1070B00040B940EB401D414F418141B341E541178B
:1070C0004249427B42AD42DF4211434343156C4784
:1070D0006C796CAB6CDD6C0F6D416D736DA56DD70C
:1070E0006D69459B45CD45FF45314663469546C78D
:1070F00046F9462B475D478F47C147F34725485719
:10710000488948BB48ED481F4951498349B549E77B
:1071100049194A4B4A7D4AAF4AE14A134B454B77DE
:107120004BA94BDB4B0D4C3F4C714CA34CD54C0742
:107130004D394D6B4D9D4DCF4D014E334E654E97A4
:107140004EC94EFB4E2D4F5F4F914FC34FF54F270A
:107150005059508B50BD50EF50215153518551B76C
:1071600051E9511B524D527F52B152E352155347D0
:10717000537953AB53DD530F5441547354A554D733
:107180005409553B556D559F55D155035635566796
:10719000569956CB56FD562F5761579357C557F7FB
:1071A000578D585B582958BF58F15823595559875E
:1071B00059B959EB591D5A4F5A815AB35AE55A17C2
:1071C0005B495B7B5BAD5BDF5B115C435C755CA724
:1071D0005CD95C0B5D3D5D6F5DA15DD35D055E3788
:1071E0005E695E9B5ECD5EFF5E315F635F955FC7EC
:1071F0005F5D602B60F95F8F60C160F36025615750
:10720000618961BB61ED611F6251628362B562E7B2
:107210006219634B637D63AF63E163136445647715
:1072200064A964DB640D653F657165A365D5650779
:107230006639666B669D66CF6601673367656797DB
:1072400067C967FB672D685F689168C368F5682741
:107250006959698B69BD69EF69216A536A856AB7A3
:107260006AE96A1B6B4D6B7F6B096E3B6E30313286
:10727000333435363738394142434445460030319E
:1072800032333435363738396162636465660028D5
:107290006E756C6C20706F696E74657229003F3F6B
:1072A0003F00464C4F4154533F2077726F6E67202A
:1072B000666F726D617474657220696E7374616C4F
:1072C0006C65642100000020202020202020202048
:1072D0002828282828202020202020202020202086
:1072E00020202020202020881010101010101010B6
:1072F00010101010101010040404040404040404FA
:107300000410101010101010414141414141010181
:10731000010101010101010101010101010101015D
:10732000010110101010101042424242424202026B
:10733000020202020202020202020202020202022D
:107340000202101010102000000000EB511A00EC97
:107350004E114F334F554F6E4F884FA34FCB4FECCD
:107360004F0D502A50EB5164508550A650C750E83D
:107370005009512A5151516751EB518851A151BBCC
:1073800051D65100000001E659AB5701C25701D94F
:107390005701F057010758011E58013558014C5844
:1073A000016358017A5801915801A85801B0580159
:1073B000C55801EB580B02590219590130590147C0
:1073C00059015E59017559028C5901A15901B859E9
:1073D00001CF59FB3000A36D0800D76CD96CF66C57
:1073E000F66C3D6D3D6D726D886D3101AAAEC2AD1A
:1073F00005F6AD01DCAD01F1AD01E1AD08E6AD0191
:1074000051AE01D5AD0138AE012FAE018EAE01E90E
:10741000AD01EEAD013BAE014DAE0393AE0254AEF5
:107420000343AE01CAAD0157AE013EAE0148AE0105
:107430005AAE0198AE019BAE019EAE025FAE0164F2
:10744000AE0169AE01C7AD01A1AE01A4AE01A7AE08
:10745000FB00012C008CB82F0023B62BB633B63BB3
:10746000B643B653B663B669B68CB88CB873B68BF0
:10747000B6A3B6B6B6C8B6D5B637B744B7FAB64DA2
:10748000B78CB88CB88CB85AB78CB867B774B7815A
:10749000B78EB79BB7A8B7B5B7C2B78CB88CB8CF03
:1074A000B7DFB7EFB7FBB70AB817B88CB84DB85C01
:1074B000B869B875B87DB800300036E50800B2E4A8
:1074C000C0E4CEE4DCE4EAE4FDE410E523E50001F9
:1074D0006BEE68EE455BEE025BEE11C2ED0B88EDE4
:1074E00001DFED015BEE015BEE015BEE02DFED051E
:1074F0007BED01B5ED01C2ED038FED02C2ED03BEE0
:10750000EDFB0001D3F0CDF045C8F002C8F0112426
:10751000F00BE8EF0144F001C8F001C8F001C8F039
:107520000244F005CCEF0118F00124F003F1EF0262
:1075300024F00321F0FB18951895189518951895C7
:107540001895189518951E9AC698009325110FB78F
:107550000093261100922711E0932811F09329112E
:10756000C6981E9A30FD09C0C6981E9A00910C114B
:107570000395077000930C1108C0C6981E9A0091DD
:107580000B110395077000930B111A9509F421C094
:10759000ECEDFDE030FD05C0C6981E9A00910C117F
:1075A00004C0C6981E9A00910B11E00F00E0F01F76
:1075B000C895002D30FF1EC00F70C69AC79A009361
:1075C000FCFFC7981C981E9AC6980E94A5400C9470
:1075D000ED3A0E94A54008E005BD1E9AF0912911E0
:1075E000E091281100902711009126110FBF009102
:1075F00025111895007FC69AC79A0093FCFFC7987B
:107600001E9AC698E4EEFDE000910C11E00F00E038
:10761000F01FC895002DC69AC79A0093FFFFC79820
:107620001C981D98C6981E9A0E94A540D6CF189502
:107630001895189518951E9A00932A110FB7009364
:107640002B1100922C11E0932D11F0932E11C6985E
:107650001E9A08E003BF38C000911011003029F4D1
:107660000395009310110DEF17C0013029F4039515
:10767000009310110BEF10C0023031F1063029F4E5
:107680000395009310110FED07C00730E9F403953F
:10769000009310110FEB00C0C69AC79A0093FEFF2B
:1076A000C798C6981E9A00910D1101BF0DE003BF47
:1076B000F0912E11E0912D1100902C1100912B11C1
:1076C0000FBF00912A111895C4980FEFC69AC79A58
:1076D0000093FEFFC798C6981E9A00E00093101111
:1076E000F0912E11E0912D1100902C1100912B1191
:1076F0000FBF00912A11189518951895189518958F
:1077000000932F110FB70093301104B100930511AE
:1077100005B100930611009130110FBF00912F1198
:1077200018951895189518951895189518951895F1
:1077300018951895189518950FEF0BBB07EF07BB19
:107740000FEE08BB00E005BB0FEE01BB0FEF02BB65
:107750000EE702B90FEF03B905B7689407F906F908
:1077600005BF0EE000936D0000E007B9C6980E94C7
:10777000C73F00E00093031100E00093FCFF00E826
:1077800003BD0FEF0093051101E00093061100E126
:107790000093091103E100930A1100E1009307111E
:1077A00003E10093081107B702680E7B07BF309111
:1077B00037113C7031603093A8010E94843E00E094
:1077C00000930F110093111100931011C69AC79ADC
:1077D00000E00093FCFF00E00093FFFF0FEF009339
:1077E000FEFF0FE1202F2093A6012093FDFFC798F5
:1077F000C6981E9A0E949D3E0E94D744C6981E9A23
:10780000789407B702680E7B07BF1C9A1D9A0E94E6
:10781000C93F0895F89487D3C6980E94C73F209324
:10782000A60181D3C6980E94C73F0091A601021706
:1078300091F7C69AC79A2093FDFFC798C6980E94F1
:10784000C93F789408950E940A3C022F07700730C0
:1078500011F001E0089500E0089500E00093AA010E
:107860000E94C73F069B14D3049B27D3059B3AD3A2
:107870000E94C93F08950E94C73F0AD30E94C93F92
:1078800008950E94C73F0E94563D789400E803BDCA
:1078900007B702680E7B07BF3091A801C09039116D
:1078A000E894C6F817C00E94C73F0E94563D7894DE
:1078B00000E803BD07B702680E7B07BF3091A8013F
:1078C00000E10093091103E100930A11C0903911FE
:1078D000E894C6F8E0ECF2E1E0933211F093331152
:1078E00009E2102EE0E4F1E1A0910911B0910A1132
:1078F0000D91A0930911B0930A1165C05EC00D30BF
:1079000099F30A3069F10C3051F11A94B9F330FD52
:1079100006C0C7FE02C000E002C06894C6F801932A
:1079200000E0016037FD01C00E7F0260C0FC01C0B5
:107930000D7F0460C1FC01C00B7F0860C2FC01C068
:10794000077FEF93FF93E0913211F0913311019390
:10795000E0933211F0933311FF91EF91C5CF86C0C0
:107960000E94A1400E940A3C0E94C73FC698022F75
:1079700007700730E9F00E94A1403093A801C0923F
:1079800029110E948C3E1C9A1D9A00E803BD0E949A
:10799000C93F0E94C2AE0E94C73FC698C09029113D
:1079A0003091A8010091A7010030D1F20C94363D2E
:1079B0000E94C73F0E94CB3F8DCF1197A093091122
:1079C000B0930A11CDCF0B3109F099CF0D91043648
:1079D00079F10532D1F10C31B9F40D910037A9F7E5
:1079E0000D91A0930911B0930A11EF93FF930E9498
:1079F00044420091A701003021F0FF91EF910C94D7
:107A0000363DFF91EF9170CF013261F40D9100FB93
:107A1000C0F805FBC1F804FBC2F807FBC7F8C09229
:107A2000391166CF033389F60D910093381160CF79
:107A30000D91003309F05CCFA0930911B0930A11A6
:107A40000E94E93E0E94C73F4FCF0D91003039F0B0
:107A500034FD05C0689437F93093A80149CFE89404
:107A600037F93093A80144CF0E94CB3F0E94D744FE
:107A70000E94A1401D9A0E94723E0E94723E0E9486
:107A8000723E0E94723E0E94723E0E94723E30938D
:107A9000A8011C9A00E803BD0E94A1400E94B33DCA
:107AA0000E94813D0E94C93FC69808950E94C73F29
:107AB000C6980FB7009331114092131150921411D0
:107AC00060921511709216118092171190921811F0
:107AD000A0921911B0921A11C0921B11D0921C11D0
:107AE000E0921D11F0921E1180931F1190932011AE
:107AF000A0932111B0932211C0932311D09324118C
:107B000008950E94C73FC698009131110FBF409061
:107B100013115090141160901511709016118090EF
:107B2000171190901811A0901911B0901A11C090CF
:107B30001B11D0901C11E0901D11F0901E1180912E
:107B40001F1190912011A0912111B0912211C0918B
:107B50002311D09124110895C6980FEF0093A70127
:107B60000E94A140089500E00093A7010E94A14057
:107B700008950E94C73FC6983091A801E89434F94F
:107B80003093A8010E94C93F08950E94C73FC6983C
:107B90003091A801689434F93093A8010E94C93F3C
:107BA00008950E94C73FC6983091A801E89430F923
:107BB0003093A80100E803BD0E94C93F08950E94C8
:107BC000C73FC6983091A801689430F93093A80156
:107BD00000E803BD0E94C93F08950E94C73F0E946C
:107BE000E93E0E94C93F08950E94C73F00913611A7
:107BF000003009F024C0C6981D98009111116894B6
:107C000000F9C69AC79A0093FFFFC798C6980090DC
:107C100034110E945D3E00911111E89400F9C69A5A
:107C2000C79A0093FFFFC798C698009035110E942D
:107C30005D3EC798C6981D9A0E94C93F0895C69890
:107C40001D9800911111689401F9C69AC79A009382
:107C5000FFFFC798C698009034110E945D3E0091C6
:107C60001111E89401F9C69AC79A0093FFFFC798CB
:107C7000C698009035110E945D3EC7981D9A0E94DB
:107C8000C93F08950E94563D789407B702680E7B5D
:107C900007BF3091A801C6980E94C73F1C980EE10B
:107CA000102F0E9446400E94A1401C9A3093A801C8
:107CB0000E94813D0E94C93F08950E94673E0A9438
:107CC000E1F708950FEF102E0CE1202E04C00FEF06
:107CD000102E0CE8202E1A940000E9F72A940000D8
:107CE000D1F708950FEF102E202E1A940000E9F717
:107CF0002A940000D1F708950E94723E0E94723EBD
:107D00000E94723E0E94723E0E94723E0E94723E2B
:107D10000E94723E0E94723E0E94723E0E94723E1B
:107D20000E94723E0E94723E0E94723E0E94723E0B
:107D30000E94723E0E94723E089533FD0895C69AD5
:107D4000C79A0091FCFF04FD2BC0C798C698089500
:107D500002E3002E0A9419F10E94723E0091FCFF8A
:107D600004FFF8CF0E94723E04FFF4CF089502E3AF
:107D7000002E0A94A1F00E94723E0091FCFF04FDC7
:107D8000F8CF0E94723E0091FCFF04FDF2CFC79A2B
:107D90001D9800E40093FFFF0E94723E089510C0FA
:107DA000C79A1D9800EC0093FFFF0091FCFF04FDB3
:107DB00005C00E94A83E0E94B73E02C00E94B73E86
:107DC00000E00093FFFFC798C6981D9A0E94C93F24
:107DD000089533FD08951D98C79A00EC0093FFFFA6
:107DE0000E94A83E0E94B73EEBCF0E94C73FC698B4
:107DF0003091A801E89433F93093A80130933711FA
:107E00000E94C93F08950E94C73FC6983091A801BB
:107E1000689433F93093A801309337110E94C93F19
:107E200008950E94C73FC69800933F110E94C93F22
:107E300008950E94C73FC69800913F110E94C93F14
:107E400008950E94C73FC6983091A801689432F9FE
:107E50003093A801309337110E94C93F08950E94C2
:107E6000C73FC6983091A801E89432F93093A80131
:107E7000309337110E94C93F08950E94C73FC698AA
:107E800000913711047002FDC6980E94C93F089501
:107E90000E94C73F1C98E89430F900E4102F0E941C
:107EA0005F400E94A1400E94C73F3091A8011C9AE8
:107EB0001D9A04E00093AA0108950E94C73F1C98F0
:107EC000689430F900E4102F0E945F400E94A140A6
:107ED0000E94C73F3091A8011C9A1D9A02E00093AE
:107EE000AA01089501E00093AA0108950895C69A91
:107EF000C79A0091FCFFC798C69800780E94C93FB6
:107F00000895C69AC79A0091FCFFC798C698027058
:107F10000E94C93F0895C6980091A8010870C698AC
:107F20000E94C93F089500E0102EC69AC79A00919A
:107F3000FCFFC798002E6894029BE89413F868949D
:107F4000039BE89414F8002D009502FB10F805FB44
:107F500011F806FB12F8002D1092A901E8940470A4
:107F600009F4689410F820F9E894029B689421F9C8
:107F7000002D007211F0E89421F9E894039B6894B5
:107F800022F9002D007411F0E89422F908951E9A48
:107F900008951E98089507B70F930F7E07BF30FF0F
:107FA00003C000E007B90DC0C6FC09C0C7FE07C08A
:107FB0000F9107BF0E94D744E89431F9089501E07A
:107FC00007B90FEC06B990E00BE0E02EE89436F923
:107FD00002E100930211D02E0FE0602E30FD04C0AC
:107FE00000913F1100FF06C000913811003011F0E0
:107FF000102F4CD0A6D002E0102F48D00FEC06B9BD
:10800000A0D001E0102F42D0CCD001D431FD08C067
:1080100000910211039503950093021131FF20C0D6
:108020000E2D003031F40091021103950395009359
:1080300002110FEC06B985D001E0102F27D0B1D086
:10804000E6D3D394D3940E2D003031F40091021175
:1080500003950395009302110E2D003009F0EA9468
:108060006A9461F600E4A02F01E1B02F07E006B9A1
:108070000F9107BF0E94D744E89431F962D0E89489
:10808000C6F8E89436F9C092391108950D9B17C0CF
:1080900030FD15C004EEE02F0DE0F02F00910C1123
:1080A000E00F00E0F01FC895002DC69AC79A009314
:1080B000FFFFC7981D98C6981E9A0E948C3E0E948A
:1080C000A140C6980E94C73F0CEDE02F0DE0F02FB5
:1080D00030FF03C000910B1102C000910C11E00FA2
:1080E00000E0F01FC895002D30FF0CC00F70C69A3D
:1080F000C79A0093FCFFC798C6981E9A1C980CE07C
:1081000005BD0895007FC69AC79A0093FCFFC798E3
:10811000C6981E9A04EEE02F0DE0F02F00910C118E
:10812000E00F00E0F01FC895002DC69AC79A009393
:10813000FFFFC798C6981E9A1C981D980CE005BDB5
:10814000089505B50770E9F7089503B5085418F0C8
:1081500003B5085003BD089503B50156E0F3F8CF09
:1081600010FA80F881F811FA82F883F812FA84F88C
:1081700085F813FA86F887F814FA90F891F815FA4A
:1081800092F893F816FA94F895F817FA96F897F883
:1081900008950E94B040282C392C102C0E94B04029
:1081A0000895E0ECF2E1E0ECF2E1A0E4B1E102E0FC
:1081B000A02E00E3702E32FF04C001E0A02E00E9E3
:1081C000702E00E0102E0E948541D7D2F7FC0CC023
:1081D00030FD06C0E89431F900913F1100FF04C062
:1081E000F3FE02C0689431F9F1FE20C0F2FE12C025
:1081F00004E10E946041C8F00E94C9400E9472419F
:10820000122C0E948541132C0E948541082C0E944B
:10821000E9413CC00AE00E94604138F00E9472418E
:108220000E9485410E94064231C038C0F7FC0DC053
:1082300036FD0BC004E0D02E0093021106E1602E43
:10824000689436F902910E9198D2F2FE15C00CE1B5
:108250000E94604150F30E94C9400E947241122C5A
:108260000E948541132C0E948541182C0E94854153
:10827000092C0E94E9410AC00EE00E946041A8F268
:108280000E9472410E9485410E94BE410A2D003029
:1082900021F4072D003009F401C097CF32FD0DC045
:1082A00000E0102E0E948541B499FECFC5980000D1
:1082B000000000000000C59A08950E941542F4CF06
:1082C000202E701A00E0A00A08F0089570947394AC
:1082D000022D0719702EC19AC298C1987A94D9F7C5
:1082E0000894089531FF0CC0F3FC0AC00E2D003035
:1082F00041F000E0002E102E202E302E802E902EE9
:1083000008950EE20D19E0F7F4CF1694C19A10F01B
:10831000C29801C0C29AC1981694C19A10F0C2982E
:1083200001C0C29AC1981694C19A10F0C29801C0B7
:10833000C29AC1981694C19A10F0C29801C0C29A0C
:10834000C1981694C19A10F0C29801C0C29AC198FF
:108350001694C19A10F0C29801C0C29AC19816949E
:10836000C19A10F0C29801C0C29AC1981694C19ADD
:1083700010F0C29801C0C29AC19808950694C19A9B
:1083800010F0C29801C0C29AC1980694C19A10F028
:10839000C29801C0C29AC1980694C19A10F0C298BE
:1083A00001C0C29AC1980694C19A10F0C29801C047
:1083B000C29AC1980694C19A10F0C29801C0C29A9C
:1083C000C1980694C19A10F0C29801C0C29AC1988F
:1083D00008950694C19A10F0C29801C0C29AC1983B
:1083E0000694C19A10F0C29801C0C29AC19806942E
:1083F000C19A10F0C29801C0C29AC1980694C19A5D
:1084000010F0C29801C0C29AC19808950694C19A0A
:1084100010F0C29801C0C29AC1980694C19A10F097
:10842000C29801C0C29AC198089505E1202E00E0CB
:10843000102E0E9485412A94D1F708950E940A3C8B
:108440000E94C73FC698022F07700730D9F00E94DC
:10845000A1401C9A1D9A3093A801C0922A111C9A1F
:108460001D9A0E94C93F0E94C2AE0E94C73FC69893
:10847000C0902A113091A8010091A7010030F1F2BB
:108480000FEF089500E0089540E004FF03C00E944C
:108490006744089530FD03C007FF01C008951E9A88
:1084A000C69A959807700E94E442A0E0BF2FFD9005
:1084B000BD901D900B2D095710F008E7B02E06E473
:1084C000A02EDF2C32FF14C00D2D025388F0602F38
:1084D00002E3D02E00E0102E0E9485411D900E94E4
:1084E0008541AA94DA94D1F70D906A95E9F74CC0CA
:1084F00000E0102E0E9485411D900E948541AA94A3
:10850000DA94D1F741C000E0102E0E948541959A7F
:10851000C6981E9A0E945441C6981E9AB0923A116B
:10852000D0923B11F0923C11A0933D11B0933E11BB
:108530000E941E42C6981E9AB0903A11D0903B11EC
:10854000F0903C11A0913D11B0913E11003041F0EE
:10855000C698959A1E9A0E94A1400FEF0895AFCF3A
:108560000E94A7430E94A1401E9A4F3F11F0C69A55
:108570009598BA94A1F7C698959A1E9A0E94A14020
:1085800000E008950C9483420A2D0030D9F300E0F6
:10859000102E0E948541AA94E1F7B5CF202E0E94AB
:1085A000563DC69A95981E9A022D07700E94E44285
:1085B000BF2FA0E02D902D902C90959AC6980E94E8
:1085C000813D1E98022D0895E4E3FEE0E00F00E0F7
:1085D000F01FC895F02D08951E9AC6980E94563D2A
:1085E0003091A801A0E1B3E1689430F94FEF0E9407
:1085F00057420C94363D1E9A0E94563D3091A80178
:10860000A0E1B3E14D904D904D901E980E944F43D4
:108610001E9AC698042D07700E94E442E0E0A0E193
:10862000B3E14D90342C0E942A434D90B42C0E940B
:108630002A434D900E942A43A32C4D900E942A4326
:10864000AA94D9F7BA94C1F70E94813D1E98C698A2
:1086500000E0089501E800936C0000E005BB1E985F
:10866000C69A0AEA959800935585959A05E59598D6
:108670000093AA82959A00EA959800935585959A59
:1086800000E800936C001E9A000095984192959A1C
:1086900006E9102E1A94F1F71E9AC698089501E87B
:1086A00000936C0000E005BBC69A0AEA9598009317
:1086B0005585959A05E595980093AA82959A00E8C4
:1086C000959800935585959A0AEA95980093558553
:1086D000959A05E595980093AA82959A042D0F70B6
:1086E000013011F4F0E819C0023011F4F0E427C0B1
:1086F000033011F4F0E823C0043011F4F0EC1FC093
:10870000053011F4F4E01BC0063011F4F5E017C099
:10871000073011F4F6E013C0F7E000E3E0E01E9A42
:1087200095980083959A000095984081959A47FF07
:10873000FBCF959AC69800E800936C000895959A2F
:10874000C69800E800936C009598C69AE6CF07B7E4
:108750000F930F7E07BF30FF03C001E007B902C0CF
:1087600000E007B90FEC06B9ECDC01E0102F8EDC5D
:108770004ED0E8940F9107BF0895008101FF13C008
:108780000191F02EEF93FF930170003031F0E5E599
:10879000FEE30D91902E00E018C0E5E5FCE30D919D
:1087A000902E00E012C00191F02EEF93FF93017024
:1087B000003031F0EDE6F0E70D91902E00E005C0BD
:1087C000EDE6FEE60D91902E00E0990CF01FE90D0C
:1087D000F01FC895102C3196C895F02DE12D30FD75
:1087E00004C010903F1110FE07C0F3FE05C000E06A
:1087F0001D2CE10DF01F04C010900211E10DF01FBF
:10880000C895102C3196C895FF91EF910895B499B1
:10881000FECF04EFE02F0DE0F02F00910511009046
:108820000611069407950694079506950695E00FA0
:1088300000E0F01FC895009104110F70039590306F
:1088400029F49395039503950C942B44913019F4D6
:10885000939503950395923019F493950395039599
:10886000933019F4939503950395943019F49395E7
:1088700003950395953019F493950395039500306E
:1088800009F40395102E002D06940694000D1A94F9
:108890000000E1F700930D1130FF06C006E00093E1
:1088A00010110FEE0FE805C000E0009310110EEF5D
:1088B00008EFC69AC79A0093FEFFC798C6981E9AFB
:1088C000C49A00910D1101BF0DE003BF08951E9AD7
:1088D000C69806E1602E59E462E974E20E94AA4457
:1088E00053E262E372E20E94AA4455E464E574E450
:1088F0000E94AA4459E868E978E80E94AA4451E134
:1089000061E171E10E94AA4453E262E372E20E94D3
:10891000AA4455E464E574E40E94AA4459E868E96D
:1089200078E80E94AA4451E161E171E10E94AA4401
:1089300053E262E372E20E94AA4455E464E574E4FF
:108940000E94AA4459E868E978E80E94AA446A9417
:1089500011F6089500E132FD01C007E1A02E00E00C
:10896000102E0E948541152E0E948541162E0E94D0
:108970008541172E0E948541AA94A9F7152E0E94C1
:10898000854100E0102E0E94854132FF02C00E9406
:108990001542B499FECFC598000000000000000009
:1089A000C59ACFDB01E0102F71DB31DF08950E9403
:1089B000C73FE0E4F1E100E0002E08E30E94E84454
:1089C000E0ECF2E100E8002E08E30E94E84408959C
:1089D00001920A95E9F708950E9461F32A9780E0D1
:1089E0000FEF10E00E946AF4A0E0A53048F40E9466
:1089F000BCF3FE01B0E0EA0FFB1F0083A395F5CFA7
:108A000040E050E863E070E09E0105E010E00E9465
:108A10009572002309F0816040E050E863E070E067
:108A20009E012B5F3F4F05E010E00E948072002303
:108A300011F082600BC045E050E09E012B5F3F4F7C
:108A40008E010E947FF3012B09F08260082F2A9685
:108A5000E4E00C9472F30E945DF3EF97219780E2BB
:108A6000A0E0B0E0482F50E02FEF30E08E010E94F0
:108A7000B3F300E000938A1100918A11053008F0E9
:108A800052C090E040918A1150E060E0959F9001C3
:108A9000849F8001949F100D211D361F589F100D3B
:108AA000211D361F065F1F4F2F4F3F4F28013901F1
:108AB000A201B3019E01205E3F4F082F10E00E94EB
:108AC0008072482F50E09E01205E3F4F8E010E9431
:108AD0007FF3012B99F4A201B3019E01205E3F4F69
:108AE000082F10E00E948072482F50E09E01205E07
:108AF0003F4F8E010E947FF3012BA9F04FAD282F2D
:108B000030E0215030408E01005E1F4F0E94834DA7
:108B1000002319F0A1E0B0E006C0EAE8F1E100812D
:108B200003950083A9CF8D01EF962196E8E00C9480
:108B30006EF30E945DF3A29781E1A0E0B0E0482FC0
:108B400050E02FEF30E08E010F5E1F4F0E94B3F315
:108B500000E000938B1100918B11043108F04CC0A0
:108B600090E040918B1150E060E0959F9001849FD0
:108B70008001949F100D211D361F589F100D211D3F
:108B8000361F065511412D4F3F4F28013901A201D3
:108B9000B3019E01082F10E00E948072482F50E020
:108BA0009E018E010F5E1F4F0E947FF3012B89F4FF
:108BB000A201B3019E01082F10E00E948072482F8D
:108BC00050E09E018E010F5E1F4F0E947FF3012B2C
:108BD00099F04889282F30E0215030408E010E94C2
:108BE000834D002319F0A1E0B0E006C0EBE8F1E10D
:108BF000008103950083AFCF8D01A296E8E00C942D
:108C00006EF30E945DF3EF97219780E4A0E0B0E05F
:108C1000482F50E02FEF30E08E010E94B3F300E0C8
:108C200010E0ECE8F1E100831183ECE8F1E1008170
:108C30001181083B2BE0120708F05CC090E0ECE8E3
:108C4000F1E14081518160E0959F9001849F800116
:108C5000949F100D211D361F589F100D211D361F8A
:108C600006551F4F2F4F3F4F28013901A201B30175
:108C70002BE331E1082F10E00E948072482F50E072
:108C80002BE331E18E010E947FF3012B89F4A201D5
:108C9000B3012BE331E1082F10E00E948072482FCE
:108CA00050E02BE331E18E010E947FF3012B11F1A3
:108CB00040917A11282F30E0215030400BE311E130
:108CC0000E94834D002319F0A1E0B0E00AC028EC17
:108CD0003EE16BE371E18901FB0140E450E00E9459
:108CE0003FF3ECE8F1E1008111810F5F1F4F00833A
:108CF00011839BCF8D01EF962196E8E00C946EF3E3
:108D00002A9705E50093741D0AEA0093881D05E57E
:108D10000093DB1D0AEA0093871E05E50093DC69DA
:108D20000AEA0093FB6905E500932C6A0AEA0093BE
:108D3000556A05E50093746A0AEA0093A8850091D4
:108D4000741D08830091881D09830091DB1D0A832F
:108D50000091871E0B830091DC690C830091FB69F5
:108D60000D8300912C6A0E830091556A0F83009148
:108D7000746A08870091A885098740E02AE030E0FE
:108D80008E010E94834D0093FC9F2A9608950091C6
:108D9000741D0093C7010091881D0093C8010091C4
:108DA000DB1D0093C9010091871E0093CA01009149
:108DB000DC690093CB010091FB690093CC01009129
:108DC0002C6A0093CD010091556A0093CE01009169
:108DD000746A0093CF010091A8850093D00140915F
:108DE000FC9F2AE030E007EC11E00E94834D002355
:108DF00011F001E0089500E008950E9460F32197CA
:108E000005E50883442480E090E0843600E0900784
:108E100010F5442001F540E021E030E08E010E9491
:108E200059E5A0E0B0E0A03107E2B00720F45F9977
:108E300002C01196F8CF5F9B07C00CB118810117D3
:108E400029F04424439402C04424439408810095AB
:108E500008830196DACF042D2196E5E00C9471F396
:108E6000AC0115E500E080E090E0843620E0920758
:108E700028F5002319F520919B00322F35FFFBCFF9
:108E800010939C00E0E0F0E0E03127E2F20738F4D4
:108E900020919B00322F37FD02C03196F5CF2091F3
:108EA0009B00322F37FF06C020919C00211719F03C
:108EB00001E001C001E010950196D7CF969824E714
:108EC00037E121503040E9F700C00000849B02C028
:108ED00001E00AC0969A24E737E121503040E9F7D3
:108EE00000C00000849B01E0969ACA0108950E9488
:108EF0005CF3269780E000E010E0EEE7F1E100830C
:108F000011830E944F4D01E00E94638600E00093B0
:108F1000791D62DD402E442019F001E00093791D97
:108F200055240091791D0023E9F403DE012B11F093
:108F30005524539490DD012B11F055245394E3EC08
:108F4000F1E000811181012B29F05BDEE1E0F1E12C
:108F500000831183E1E0F1E100811181012B11F027
:108F60005524539466249E018E010E5F1F4F0E946C
:108F70007EB9012B29F06624639401E00093791DEA
:108F800006DF702EE4ECFDE1018100FD03C00E94CC
:108F9000AA67802F01E00093B9010AE11AE60E9456
:108FA000B788E1EDFDE100811181E3EDFDE1008392
:108FB00011830E940C7841E030E200EB14E020E0E5
:108FC0000E94A7AB0E94E4A2003139F441E031E0F5
:108FD00001EC14E020E00E94A7AB0E94E4A2013063
:108FE00039F441E031E00BED14E020E00E94A7AB42
:108FF000E3ECF1E000811181012B09F452C0FDDEA8
:10900000902F2EDF802E20E006E311E10E94EB710D
:109010000E94F43D21E006E311E10E94EB710E9401
:10902000F43D042D10E0252D30E0200F311F062DDA
:1090300010E0020F131F292F30E0200F311F082DE1
:1090400010E0020F131F272D30E0200F311FE5EC39
:10905000F1E000811181020F131F00831183E5EC01
:10906000F1E0008111811A930A93E3ECF1E0408171
:10907000518104E610E00E9446F240EE51E00E9469
:1090800060F21A930A9349E553E060E00DE012E0C4
:109090000E944AF4249631E021E00DE012E00E94A3
:1090A00010AC4CEF54E060E007EC11E00E944AF491
:1090B000662059F0EDE2F5E030E0A7ECB1E00E9467
:1090C00084F401E00093791D22C0088110E01A9316
:1090D0000A930B8110E01A930A930E811F811A9351
:1090E0000A930B8510E01A930A930C8510E01A93EB
:1090F0000A934FED50E060E00DE012E00E944AF468
:109100002A962DE032E007EC11E00E9472F40E94F2
:1091100074AC46E055E060E007EC11E00E944AF4D0
:10912000772059F0EDE2F5E030E0A7ECB1E00E94E5
:1091300084F401E00093791D07C0E5E6F5E030E036
:10914000A7ECB1E00E9484F40E9474AC45E155E0C4
:1091500060E007EC11E00E944AF4442011F455202D
:1091600041F101E00093791DEDE2F5E030E0A7EC7C
:10917000B1E00E9484F441FA46F4EEE4F5E030E018
:10918000A7ECB1E00E9484F41BC040FA46F4E7E487
:10919000F5E030E0A7ECB1E00E9484F411C0552066
:1091A00079F0E5E5F5E030E0A7ECB1E00E9484F469
:1091B00007C0E5E6F5E030E0A7ECB1E00E9484F4FA
:1091C0000E9474AC0E94E4A20131F9F0E4ECFDE1EC
:1091D000018100FD1AC040E255E060E007EC11E0BB
:1091E0000E944AF4882341F0EDE2F5E030E0A7EC7C
:1091F000B1E00E9484F407C0E5E6F5E030E0A7ECBA
:10920000B1E00E9484F40E9474ACE3ECF1E00081D0
:109210001181012B09F44BC10E949A610023B1F422
:1092200045E027E130EA0DE012E00E949190E1EB89
:10923000F8E030E0A7ECB1E00E94A5F42DE032E0C8
:1092400007EC11E00E9472F40E9474AC4DE655E008
:1092500060E007EC11E00E944AF4992379F0EDE216
:10926000F5E030E0A7ECB1E00E9484F4E5E3F5E03E
:1092700030E0A7ECB1E00E9484F407C0E5E6F5E039
:1092800030E0A7ECB1E00E9484F40E9474AC4AE79D
:1092900055E060E007EC11E00E944AF4882079F084
:1092A000EDE2F5E030E0A7ECB1E00E9484F4E5E304
:1092B000F5E030E0A7ECB1E00E9484F407C0E5E6F9
:1092C000F5E030E0A7ECB1E00E9484F40E9474ACB9
:1092D00047E855E060E007EC11E00E944AF40E9484
:1092E000813F002341F0E1EAF5E030E0A7ECB1E096
:1092F0000E9484F407C0EBEAF5E030E0A7ECB1E0AF
:109300000E9484F40E9474ACE2ECFDE14081518142
:10931000440F40E050E0441F03E010E00E9446F29A
:10932000F801E050FF4F008111812281F801322FB6
:10933000A3E5B2E00E94A5F44091841D50E003E053
:1093400010E00E9446F2F801EA58FF4F00811181B7
:109350002281F801322FADE0B2E00E94A5F40DE0C9
:1093600012E01A930A9303E512E01A930A9345E078
:1093700051E060E007EC11E00E944AF424960E945C
:1093800074ACE2ECFDE140815181440F40E050E0DB
:10939000441F03E010E00E9446F2F801E050FF4F46
:1093A000008111812281F801322FA3E5B2E00E94F1
:1093B000A5F44091851D50E003E010E00E9446F2C4
:1093C000F801E659FF4F008111812281F801322F07
:1093D000ADE0B2E00E94A5F40DE012E01A930A930A
:1093E00003E512E01A930A9348E151E060E007ECCC
:1093F00011E00E944AF424960E9474AC04E011E14A
:109400000E94F77110E0025010401A930A9301E095
:1094100010E01A930A9300E010E01A930A9343EBCA
:1094200055E060E007EC11E00E944AF426960E94A5
:1094300074ACE9E4F1E030E0A7ECB1E00E94A5F4FF
:1094400040E024E030E007EC11E00E94EFA7E3EEFB
:10945000F5E030E0A7ECB1E00E94A5F4EBE0F7E026
:1094600030E0A7ECB1E00E9484F40E9474ACE9ED16
:10947000F5E030E0A7ECB1E00E94A5F4EDEFF6E0F6
:1094800030E0A7ECB1E00E9484F40E9474ACE4EFF9
:10949000F5E030E0A7ECB1E00E94A5F4EAE1F7E0E6
:1094A00030E0A7ECB1E00E9484F40E9474AC882301
:1094B00019F40E941767802F0091791D002361F431
:1094C0000091771D002341F40091781D002321F4C1
:1094D000772011F4882339F041E031E001E016E013
:1094E00020E00E94A7AB0091771D002371F041E0BE
:1094F00031E001E116E020E00E94A7AB41E031E05D
:109500000AE216E020E00E94A7AB0091781D00233C
:1095100071F041E031E000E416E020E00E94A7ABEA
:1095200041E031E001E616E020E00E94A7AB89347B
:1095300039F441E031E007EC18E020E00E94A7ABED
:109540008A3439F441E031E000EF18E020E00E9475
:10955000A7AB833339F441E031E000E219E020E0C9
:109560000E94A7AB843339F441E031E007E519E00C
:1095700020E00E94A7AB853339F441E031E000E7F9
:1095800019E020E00E94A7AB863339F441E031E0D6
:1095900004E919E020E00E94A7AB8B3439F441E0E4
:1095A00031E00CE219E020E00E94A7AB8F34A1F477
:1095B000E6E2FFE1008103FD08C041E031E000EF99
:1095C00018E020E00E94A7AB07C041E031E005E4CD
:1095D00019E020E00E94A7AB8D3439F441E031E07E
:1095E00005EA19E020E00E94A7AB803509F055C0DC
:1095F00041E031E003ED19E020E00E94A7ABE8E88C
:10960000FEE1048115810F5F1F4F1A930A9343E413
:109610005AE060E00DE012E00E944AF4229631E048
:1096200021E00DE012E00E9410ACE0E2FFE10081D9
:1096300011811A930A934CE55AE060E00DE012E0C4
:109640000E944AF4229631E021E00DE012E00E94EF
:1096500010ACE8E8FEE1048115810F5F1F4FE0E2E6
:10966000FFE12081318102171307B8F4E0E2FFE146
:1096700000811181E8E8FEE124813581021B130B92
:1096800001501040013020E0120739F441E031E090
:1096900004E71AE020E00E94A7AB823339F441E0EE
:1096A00031E005EF19E020E00E94A7AB883339F4E0
:1096B00041E031E001E11AE020E00E94A7AB8033F5
:1096C00031F0863421F0873411F0883439F441E0E8
:1096D00031E00FE21AE020E00E94A7AB41E031E068
:1096E00006E916E020E00E94A7ABE2ECFDE1008174
:1096F000118101FF05C010E000E10E9421A904C012
:1097000010E000E00E9421A9E3ECF1E0008111816A
:10971000012BA9F00091831D002389F090E00091B6
:10972000831D901760F40E94E93E0E94423E0E9411
:10973000423E0E94423E0E94423E9395F0CF01E09D
:109740000E94D3A802E000937F1D0E9465A800E05C
:1097500000937F1DE1EDFDE1008111810F5F1F4F3F
:109760000083118300E010E0E3EDFDE1008311834D
:109770000E94DBAC00E00093B9012696E9E00C946E
:109780006DF340E953E060E00DED1DE10E944AF405
:109790004BE953E060E006E01EE10E944AF442EB30
:1097A00053E060E00FE21EE10E944AF449ED53E00D
:1097B00060E008E51EE10E944AF40FE00093DC1D22
:1097C00008959A938A93C80100E010E0EEE7F1E172
:1097D000008311830091771D002339F001E110E02F
:1097E000EEE7F1E10083118398C00091781D00231A
:1097F00039F009E010E0EEE7F1E1008311838DC05C
:10980000E2ECFDE10081118100FF07C002E010E001
:10981000EEE7F1E10083118380C028E230E08C01A3
:109820000E94B0EAEEE7F1E100831183EEE7F1E197
:1098300000811181012B09F070C028E230E08C0119
:10984000075D1F4F0E94B0EAEEE7F1E1008311834C
:10985000EEE7F1E100811181012B09F05EC028E201
:1098600030E08C010E5A1F4F0E94B0EAEEE7F1E1A2
:1098700000831183EEE7F1E100811181012B09F0F2
:109880004CC028E230E08C0105581F4F0E94B0EA1E
:10989000EEE7F1E100831183EEE7F1E10081118150
:1098A000012BD9F58C010E94ACF4012BE1F48C0161
:1098B000075D1F4F0E94ACF4012BA9F48C010E5AD6
:1098C0001F4F0E94ACF4012B71F48C0105581F4FFF
:1098D0000E94ACF4012B39F408E110E0EEE7F1E16D
:1098E000008311831AC09C010DED1DE10E949AF4C2
:1098F0009C01275D3F4F06E01EE10E949AF49C0107
:109900002E5A3F4F0FE21EE10E949AF49C01255807
:109910003F4F08E51EE10E949AF4EEE7F1E1208155
:10992000318109E30E9461AD89919991089500E028
:1099300010E0EEE7F1E1008311830E945EA801E0F0
:109940000E940DA90E944F4DE2ECFDE100811181C2
:1099500001FF05C010E000E90E9421A904C010E049
:1099600000E80E9421A90DED1DE10E94ACF4012B3D
:10997000D1F0ECEDFDE1008100FD15C0E4ECFDE16E
:10998000008100FF05C00DED1DE10E9486AC06C000
:1099900030E020E80DED1DE10E9410ACECEDFDE1A2
:1099A00000810061008306E01EE10E94ACF4012BFF
:1099B000D1F0ECEDFDE1008101FD15C0E4ECFDE12D
:1099C000008100FF05C006E01EE10E9486AC06C0D3
:1099D00030E020E806E01EE10E9410ACECEDFDE175
:1099E0000081006200830FE21EE10E94ACF4012BB3
:1099F000D1F0ECEDFDE1008102FD15C0E4ECFDE1EC
:109A0000008100FF05C00FE21EE10E9486AC06C087
:109A100030E020E80FE21EE10E9410ACECEDFDE129
:109A200000810064008308E51EE10E94ACF4012B74
:109A3000D1F0ECEDFDE1008103FD15C0E4ECFDE1AA
:109A4000008100FF05C008E51EE10E9486AC06C04B
:109A500030E020E808E51EE10E9410ACECEDFDE1ED
:109A60000081006800830E9465A8EEE7F1E1208193
:109A7000318101E60E9461AD0895E2ECFDE10081D3
:109A800011810179107800831183E2ECFDE10081FE
:109A9000118100601C670083118301D008950E942A
:109AA000A04EE2ECFDE100811181077F118300836C
:109AB000E2ECFDE10081118104FF1EC0ECE8F1E160
:109AC000008111810B392BE0120738F0E2ECFDE147
:109AD00000811181006211830083ECE8F1E10081D3
:109AE0001181083B2BE0120738F0E2ECFDE1008128
:109AF00011810064118300830E94085EE2ECFDE1A5
:109B00000081118108951C012297B80155E880E079
:109B100090E0FB01E80FF91F00810983019682178D
:109B2000930730F4FB01E80FF91F0081088301C09F
:109B3000488310E01830A8F4098107FF0AC00880A4
:109B40001980000C111C08821982098105270983DC
:109B500006C008801980000C111C08821982139518
:109B6000E9CF0196F90131968E179F07C0F209815E
:109B70002296C101089540E04830A8F4502F51705A
:109B8000622F61706527662341F016950795B8012D
:109B900001E010EA0627172702C0169507953695AB
:109BA00027954395E9CF08950E945BF32801390179
:109BB000842F4201A0E0A81758F4B0E0F301EA0FA7
:109BC000FB1F208130E08401D6DF4801A395F3CF4D
:109BD0008401EAE00C946CF39A938A9380E090E01D
:109BE00047E023E031E18C01DFDFC8014CE02BE1ED
:109BF00031E18C01D9DFC80142E024E931E18C0177
:109C0000D3DFC80144E02EE831E18C01CDDFC8018B
:109C100042E022E931E18C01C7DFC80141E028E2DE
:109C20003FE18C01C1DFC80148E024E232E18C0150
:109C3000BBDFC80145E02EE231E18C01B5DFC80190
:109C400044E022E23FE18C01AFDFC8018C01899141
:109C500099910895E2ECFDE1008111810F77118364
:109C6000008308E813E120E030E0E8ECFDE1008348
:109C700011832283338308E813E120E030E0ECEC29
:109C8000FDE1008311832283338300E00093D01D24
:109C900022E004E011E10E94EB7125E008E311E10C
:109CA0000E94EB710E94F53E0E942F3F01E00E944E
:109CB000113FE4ECFDE100810E7F0083E4ECFDE167
:109CC00000810D7F0083E4ECFDE1008104600083EE
:109CD000E4ECFDE10081077F008301E00093801D3B
:109CE000E4ECFDE100810F770083E4ECFDE100810D
:109CF0000F7E00830091C51D097F02600093C51D82
:109D0000E4ECFDE101810E7F0183E4ECFDE10081E3
:109D100002FB00E000F9E6ECFDE100FB008102F946
:109D2000008344E050E020E330E003E81EE10E94BD
:109D3000B3F300E30E94A9E404E30E94A9E40895B8
:109D40008A930E943D3F802F882341F0E2ECFDE1A1
:109D50000081118102601183008307C0E2ECFDE104
:109D6000008111810D7F11830083899108950E94E4
:109D70005BF3D801FD0104810E941C90802EFD013F
:109D800005810E941C90702EFD0106810E941C908E
:109D9000982C8824990C990C990C990C372D20E05B
:109DA0002829392910E044E00E944EF24801822A15
:109DB000932AFD0107810E941C9010E008291929AF
:109DC00028018D010E9482F1C8018201E8E4F0E0DF
:109DD000FBBFF3E70C94FEF241E050E020E030E0FE
:109DE0008C010E94D3EAEEE7F1E100831183EEE7F4
:109DF000F1E100811181012B09F0F3C2082F092B39
:109E000041F0E2ECFDE100811181006811830083E3
:109E1000E8C2E2ECFDE1008111810F77118300833C
:109E2000E0C244E853E020E030E08C010E94D3EA35
:109E3000EEE7F1E100831183EEE7F1E100811181AA
:109E4000012B09F0CEC2AC0160E070E008EE13E037
:109E500020E030E00E948CF2E8ECFDE10083118309
:109E600022833383BEC244E853E020E030E08C011B
:109E70000E94D3EAEEE7F1E100831183EEE7F1E11E
:109E800000811181012B09F0ACC2AC0160E070E0EF
:109E900008EE13E020E030E00E948CF2ECECFDE1F3
:109EA00000831183228333839CC241E050E020E091
:109EB00030E08C010E94D3EAEEE7F1E100831183E8
:109EC000EEE7F1E100811181012B09F08AC2282F10
:109ED0002E5F04E011E10E94EB7183C24FEF50E06E
:109EE00020E030E08C010E94D3EAEEE7F1E100834C
:109EF0001183EEE7F1E100811181012B09F071C2BC
:109F0000082F602E262D08E311E10E94EB7169C233
:109F100041E050E020E030E08C010E94D3EAEEE71F
:109F2000F1E100831183EEE7F1E100811181012B62
:109F300009F057C2082F092B19F00E94033F51C2A4
:109F40000E94F53E4EC2E2ECFDE10081118100FF6E
:109F500007C002E010E0EEE7F1E10083118341C2A7
:109F600041E050E020E030E08C010E94D3EAEEE7CF
:109F7000F1E100831183EEE7F1E100811181012B12
:109F800009F02FC2082F092B19F00E94213F29C286
:109F90000E942F3F26C241E050E020E030E08C01DB
:109FA0000E94D3EAEEE7F1E100831183EEE7F1E1ED
:109FB00000811181012B09F014C2082F092B31F007
:109FC000E4ECFDE10081016000830BC2E4ECFDE103
:109FD00000810E7F008305C241E050E020E030E0C8
:109FE0008C010E94D3EAEEE7F1E100831183EEE7F2
:109FF000F1E100811181012B09F0F3C1082F092B38
:10A0000031F0E4ECFDE1008102600083EAC1E4ECA0
:10A01000FDE100810D7F0083E4C141E050E020E0DC
:10A0200030E08C010E94D3EAEEE7F1E10083118376
:10A03000EEE7F1E100811181012B09F0D2C1082F77
:10A04000092B21F001E00E94113FCBC100E00E94EA
:10A05000113FC7C1E2ECFDE10081118100FF07C0A3
:10A0600002E010E0EEE7F1E100831183BAC141E0C4
:10A0700050E020E030E08C010E94D3EAEEE7F1E10D
:10A0800000831183EEE7F1E100811181012B09F0DA
:10A09000A8C1082F092B31F0E4ECFDE10081046038
:10A0A000008305C0E4ECFDE100810B7F0083E4EC5C
:10A0B000FDE1008102FB00E000F9E6ECFDE100FBC0
:10A0C000008102F900838DC141E050E020E030E0E2
:10A0D0008C010E94D3EAEEE7F1E100831183EEE701
:10A0E000F1E100811181012B09F07BC1082F092BBF
:10A0F00031F0E4ECFDE100810860008372C1E4EC22
:10A10000FDE10081077F00836CC141E050E020E069
:10A1100030E08C010E94D3EAEEE7F1E10083118385
:10A12000EEE7F1E100811181012B09F05AC1082FFE
:10A13000092B31F0ECEDFDE100810160008351C19C
:10A14000ECEDFDE100810E7F00834BC141E050E06A
:10A1500020E030E08C010E94D3EAEEE7F1E10083D9
:10A160001183EEE7F1E100811181012B09F039C182
:10A17000082F092B31F0ECEDFDE100810260008336
:10A1800030C1ECEDFDE100810D7F00832AC141E08B
:10A1900050E020E030E08C010E94D3EAEEE7F1E1EC
:10A1A00000831183EEE7F1E100811181012B09F0B9
:10A1B00018C1082F092B31F0ECEDFDE1008104609E
:10A1C00000830FC1ECEDFDE100810B7F008309C12D
:10A1D00041E050E020E030E08C010E94D3EAEEE75D
:10A1E000F1E100831183EEE7F1E100811181012BA0
:10A1F00009F0F7C0082F092B31F0ECEDFDE10081EB
:10A2000008600083EEC0ECEDFDE10081077F008374
:10A21000E8C041E050E020E030E08C010E94D3EA49
:10A22000EEE7F1E100831183EEE7F1E100811181B6
:10A23000012B09F0D6C0082F092B31F0ECEDFDE120
:10A2400000810F600083CDC0ECEDFDE10081007F57
:10A250000083C7C041E050E020E030E08C010E9464
:10A26000D3EAEEE7F1E100831183EEE7F1E100814B
:10A270001181012B09F0B5C0082F092B71F0E4EC16
:10A28000FDE100810F7D0083E4ECFDE100810F7BA7
:10A29000008301E00093801DA4C000E00093801DB6
:10A2A000A0C04FEF50E020E030E08C010E94D3EAE4
:10A2B000EEE7F1E100831183EEE7F1E10081118126
:10A2C000012B09F08EC0082F0093871D8AC041E042
:10A2D00050E020E030E08C010E94D3EAEEE7F1E1AB
:10A2E00000831183EEE7F1E100811181012B09F078
:10A2F00078C0082F092B31F0E4ECFDE1008100610A
:10A3000000836FC0E4ECFDE100810F7E008369C033
:10A310008D010E9482F1C801843100E0900738F07D
:10A3200005E110E0EEE7F1E1008311835AC000E09F
:10A3300010E0EEE7F1E100831183082F0093D01DB8
:10A3400050C041E050E020E030E08C010E94D3EAB0
:10A35000EEE7F1E100831183EEE7F1E10081118185
:10A36000012BF9F5082F0170E4ECFDE100FB018100
:10A3700000F9018336C042E050E020E030E08C017B
:10A380000E94D3EAEEE7F1E100831183EEE7F1E109
:10A3900000811181012B29F51091C51D197F082F0E
:10A3A000000F0670012B0093C51D1BC048EC50E048
:10A3B00020E030E08C010E94D3EAEEE7F1E1008377
:10A3C0001183EEE7F1E100811181012B51F4082F97
:10A3D0000093831D06C005E110E0EEE7F1E1008384
:10A3E0001183EEE7F1E12081318107E50E9461AD43
:10A3F000EAE00C946CF30E9461F301E010E0E5EDFB
:10A40000FDE1008311830E9427BAE4ECFDE10081A5
:10A4100003FD04C004ED19E60E94B78800E010E0D7
:10A42000E2EDF9E6008311830FE81EE10E94B78890
:10A4300007E91EE10E94B78800E010E0EDEDF9E6C3
:10A44000008311830FED19E60E94B78800E010E049
:10A45000E7EEF9E60083118309EE19E60E94B7885A
:10A4600000E010E0E1EFF9E60083118303EF19E665
:10A470000E94B78800E010E0E0E1FAE60083118373
:10A4800002E11AE60E94B78800E010E0E2E2FAE694
:10A490000083118304E21AE60E94B78800E010E00E
:10A4A000EDE2FAE6008311830FE21AE60E94B78814
:10A4B00000E010E0E7E3FAE60083118309E31AE61F
:10A4C0000E94B78800E010E0E9E4FAE60083118317
:10A4D00001E41AE60E94B78800E010E0E3E5FAE63E
:10A4E000008311830BE41AE60E94B78800E010E0B5
:10A4F000EEE5FAE60083118306E51AE60E94B788C6
:10A5000000E010E0E8E6FAE60083118300E61AE6D0
:10A510000E94B78800E010E0ECEFF9E600831183B9
:10A520000EEF19E60E94B78800E010E0E6E0FAE6D8
:10A530000083118308E01AE60E94B78800E010E06B
:10A54000E2E7FAE6008311830AE61AE60E94B7887A
:10A5500000E010E0EDE7FAE60083118305E71AE674
:10A560000E94B78880E090E0853000E0900774F4A6
:10A57000ACECBFE9AC0108E010E00E9446F2A00F8D
:10A58000B11F8D010E94B7880196EECF04EF1FE93D
:10A590000E94B7880FE91EE10E94B78807EA1EE112
:10A5A0000E94B7880FEA1EE10E94B78807EB1EE100
:10A5B0000E94B7880FEB1EE10E94B788E4E00C947C
:10A5C00072F30E9460F34FB6F89400919811005016
:10A5D00069F00A9509F48CC20A9509F47FC30A95BB
:10A5E00009F4B3C3095009F483C2E5C3009199117A
:10A5F000005069F00A9509F441C00A9509F43DC17B
:10A600000A9509F46CC00A9509F4D0C066C124E229
:10A6100032E104ED19E60E94138A24E232E109E3F3
:10A620001AE60E94138AE7E3FAE6008111810F5FC0
:10A630001F4F0083118324E232E1C901ACE4BFE182
:10A640004091281F50E00FEB10E00E9446F2A00F4F
:10A65000B11F8D019C010E94138A4091281F50E078
:10A660000FEB10E00E9446F2F801EA5CF04E04891C
:10A6700015890F5F1F4F048B158B2FC124E232E128
:10A680000FE21AE60E94138AEDE2FAE600811181D8
:10A690000F5F1F4F0083118324E232E1C901A6E559
:10A6A000BFE14091281F50E00FEB10E00E9446F2FE
:10A6B000A00FB11F8D019C010E94138A4091281F99
:10A6C00050E00FEB10E00E9446F2F801EA5CF04E19
:10A6D000068D178D0F5F1F4F068F178FFEC02CE260
:10A6E00032E104ED19E60E94138A2CE232E109E31B
:10A6F0001AE60E94138AE7E3FAE6008111810F5FF0
:10A700001F4F0083118324E332E10FE21AE60E9417
:10A71000138AEDE2FAE6008111810F5F1F4F00837B
:10A7200011832CE232E1C901ACE4BFE14091281F62
:10A7300050E00FEB10E00E9446F2A00FB11F8D0118
:10A740009C010E94138A4091281F50E00FEB10E0FB
:10A750000E9446F2F801EA5CF04E048915890F5F09
:10A760001F4F048B158B24E332E1C901A6E5BFE13D
:10A770004091281F50E00FEB10E00E9446F2A00F1E
:10A78000B11F8D019C010E94138A4091281F50E047
:10A790000FEB10E00E9446F2F801EA5CF04E068DE5
:10A7A000178D0F5F1F4F068F178F97C02CE232E176
:10A7B00004ED19E60E94138A2CE232E109E31AE65D
:10A7C0000E94138AE7E3FAE6008111810F5F1F4FB1
:10A7D0000083118324E332E105E71AE60E94138A1D
:10A7E000EDE7FAE6008111810F5F1F4F00831183AF
:10A7F0002CE232E1C901ACE4BFE14091281F50E0F6
:10A800000FEB10E00E9446F2A00FB11F8D019C01DA
:10A810000E94138A4091281F50E00FEB10E00E9425
:10A8200046F2F801EA5CF04E048915890F5F1F4F6C
:10A83000048B158B24E332E1C901A0E6BFE140910E
:10A84000281F50E00FEB10E00E9446F2A00FB11F4E
:10A850008D019C010E94138A4091281F50E00FEB4C
:10A8600010E00E9446F2F801EA5CF04E00A511A546
:10A870000F5F1F4F00A711A730C024E232E105E7A8
:10A880001AE60E94138AEDE7FAE6008111810F5F54
:10A890001F4F0083118324E232E1C901A0E6BFE12A
:10A8A0004091281F50E00FEB10E00E9446F2A00FED
:10A8B000B11F8D019C010E94138A4091281F50E016
:10A8C0000FEB10E00E9446F2F801EA5CF04E00A5A2
:10A8D00011A50F5F1F4F00A711A724E232E10FE877
:10A8E0001EE10E94138AEEE8F1E104851585E2ED90
:10A8F000F9E620813181200F311F2083318324E24A
:10A9000032E1C901A8E3BFE14091281F50E00FEBFD
:10A9100010E00E9446F2A00FB11F8D019C010E9421
:10A92000138AEEE8F1E1848595854091281F50E077
:10A930000FEB10E00E9446F2F801EA5CF04E008155
:10A940001181080F191F0083118324E232E10FE700
:10A950001AE60E94138A002351F00FE71AE60E94BC
:10A96000B78824E232E10FE71AE60E94138A24E254
:10A9700032E107E81AE60E94138A002351F007E843
:10A980001AE60E94B78824E232E107E81AE60E943C
:10A99000138A24EA31E106E51AE60E94138AEEE8FA
:10A9A000F1E106851785EEE5FAE620813181200F79
:10A9B000311F2083318324EA31E1C901AAE6BFE1D6
:10A9C0004091281F50E00FEB10E00E9446F2A00FCC
:10A9D000B11F8D019C010E94138AEEE8F1E186858A
:10A9E00097854091281F50E00FEB10E00E9446F23F
:10A9F000F801EA5CF04E02A913A9080F191F02AB77
:10AA000013AB2CEA31E100E61AE60E94138AEEE865
:10AA1000F1E100891189E8E6FAE620813181200F11
:10AA2000311F208331832CEA31E1C901A4E7BFE162
:10AA30004091281F50E00FEB10E00E9446F2A00F5B
:10AA4000B11F8D019C010E94138AEEE8F1E180891B
:10AA500091894091281F50E00FEB10E00E9446F2D0
:10AA6000F801EE58F04E00811181080F191F008384
:10AA7000118324EB31E10AE61AE60E94138AEEE81C
:10AA8000F1E102891389E2E7FAE620813181200FA2
:10AA9000311F2083318324EB31E1C901A2E4BFE1FE
:10AAA0004091281F50E00FEB10E00E9446F2A00FEB
:10AAB000B11F8D019C010E94138AEEE8F1E18289A9
:10AAC00093894091281F50E00FEB10E00E9446F25E
:10AAD000F801EA5CF04E02851385080F191F028702
:10AAE000138704EB1AE60E9464BA0E943CA563C176
:10AAF000009198110130D9F524E232E104ED19E614
:10AB00000E94958A24E232E109EE19E60E94138A36
:10AB1000E7EEF9E6008111810F5F1F4F008311837B
:10AB200000EB13E70E9464BA24E232E1C901AEE708
:10AB3000BFE14091281F50E00FEB10E00E9446F269
:10AB4000A00FB11F8D019C010E94138A4091281F04
:10AB500050E00FEB10E00E9446F2F801E458F04E8E
:10AB6000008111810F5F1F4F0083118334C024E2E5
:10AB700032E103EF19E60E94138AE1EFF9E6008162
:10AB800011810F5F1F4F008311830CEA1CE70E94A5
:10AB900064BA24E232E1C901A8E8BFE14091281F6C
:10ABA00050E00FEB10E00E9446F2A00FB11F8D01A4
:10ABB0009C010E94138A4091281F50E00FEB10E087
:10ABC0000E9446F2F801EA57F04E008111810F5FB2
:10ABD0001F4F0083118324EA31E10EEF19E60E9432
:10ABE000138AEEE8F1E106851785ECEFF9E620819E
:10ABF0003181200F311F2083318324EA31E1C901E3
:10AC0000A2E9BFE14091281F50E00FEB10E00E9445
:10AC100046F2A00FB11F8D019C010E94138AEEE83D
:10AC2000F1E1868597854091281F50E00FEB10E0F9
:10AC30000E9446F2F801E057F04E00811181080FA2
:10AC4000191F008311832CEA31E108E01AE60E9403
:10AC5000138AEEE8F1E100891189E6E0FAE6208145
:10AC60003181200F311F208331832CEA31E1C9016A
:10AC7000ACE9BFE14091281F50E00FEB10E00E94CB
:10AC800046F2A00FB11F8D019C010E94138AEEE8CD
:10AC9000F1E1808991894091281F50E00FEB10E08D
:10ACA0000E9446F2F801E656F04E00811181080F2D
:10ACB000191F0083118324E232E10FED19E60E948F
:10ACC000138AEEE8F1E104851585EDEDF9E62081C2
:10ACD0003181200F311F208331836DC024E232E1A6
:10ACE00004ED19E60E94138A24E232E101E41AE637
:10ACF0000E94138AE9E4FAE6008111810F5F1F4F79
:10AD00000083118324E232E1C901AAEBBFE1409143
:10AD1000281F50E00FEB10E00E9446F2A00FB11F79
:10AD20008D019C010E94138A4091281F50E00FEB77
:10AD300010E00E9446F2F801E854F04E00811181C3
:10AD40000F5F1F4F0083118336C024E232E104ED10
:10AD500019E60E94958A24E232E10BE41AE60E9489
:10AD6000138AE3E5FAE6008111810F5F1F4F00832C
:10AD7000118324E232E1C901A4ECBFE14091281F14
:10AD800050E00FEB10E00E9446F2A00FB11F8D01C2
:10AD90009C010E94138A4091281F50E00FEB10E0A5
:10ADA0000E9446F2F801EE53F04E008111810F5FD0
:10ADB0001F4F008311832CEB31E102E11AE60E9460
:10ADC000138AEEE8F1E104891589E0E1FAE62081D1
:10ADD0003181200F311F208331832CEB31E1C901F8
:10ADE000A6EABFE14091281F50E00FEB10E00E945F
:10ADF00046F2A00FB11F8D019C010E94138AEEE85C
:10AE0000F1E1848995894091281F50E00FEB10E013
:10AE10000E9446F2F801EC55F04E00811181080FB6
:10AE2000191F008311834FBEE5E00C9471F30E945B
:10AE300058F3380104E510EAD80183010E9482F139
:10AE4000C80100E010E0EEE7F1E1008311830E9409
:10AE50001767C02ECC2009F457C000E5C01609F0D2
:10AE600053C00E94776710E0EEE7F1E100831183A1
:10AE7000EEE7F1E100811181012B09F047C60E9444
:10AE80009A6110E0EEE7F1E100831183EEE7F1E172
:10AE900000811181012B09F039C60E94C46110E0C4
:10AEA000EEE7F1E100831183EEE7F1E1008111812A
:10AEB000012B09F02BC6009109A00093211F0091DE
:10AEC0000AA00093201FE6E2FFE1008106FF08C010
:10AED0000E94DE6110E0EEE7F1E10083118314C00F
:10AEE00000917A1D002381F401E000937A1DE0E2D5
:10AEF000FFE100811181015010400E94226310E0A7
:10AF0000EEE7F1E100831183EEE7F1E100811181C9
:10AF1000012B09F0FBC54EE250E020E030E004E5F3
:10AF200010EA0E94B3F340E050E025E58D010E9455
:10AF30002CAD9A938A9343EB50E060E08D01005F63
:10AF40001F4F0E944AF422968C01E4E8F0E0FBBF18
:10AF5000F3E70C94FEF2E2EDF9E6008111811A9319
:10AF60000A9348EB50E060E08D010B5E1F4F0E949A
:10AF70004AF422969D01255E3F4F0FE81EE10E9494
:10AF8000D68DA7C5E2E7FAE6008111811A930A93EC
:10AF900048EB50E060E08D010B5E1F4F0E944AF4C9
:10AFA00022969D01255E3F4F0AE61AE60E94D68D45
:10AFB00090C5EDE2FAE6008111811A930A9348EBFD
:10AFC00050E060E08D010B5E1F4F0E944AF4229614
:10AFD0009D01255E3F4F0FE21AE60E94D68D79C58E
:10AFE000EDE7FAE6008111811A930A9348EB50E0ED
:10AFF00060E08D010B5E1F4F0E944AF422969D0176
:10B00000255E3F4F05E71AE60E94D68D62C5EEE544
:10B01000FAE6008111811A930A9348EB50E060E050
:10B020008D010B5E1F4F0E944AF422969D01255E02
:10B030003F4F06E51AE60E94D68D4BC5E8E6FAE6D4
:10B04000008111811A930A9348EB50E060E08D0172
:10B050000B5E1F4F0E944AF422969D01255E3F4FD2
:10B0600000E61AE60E94D68D34C5E7EEF9E60081C7
:10B0700011811A930A9348EB50E060E08D010B5E5A
:10B080001F4F0E944AF422969D01255E3F4F09EE14
:10B0900019E60E94D68D1DC5E1EFF9E60081118108
:10B0A0001A930A9348EB50E060E08D010B5E1F4F4E
:10B0B0000E944AF422969D01255E3F4F03EF19E658
:10B0C0000E94D68D06C5E0E1FAE6008111811A934F
:10B0D0000A9348EB50E060E08D010B5E1F4F0E9429
:10B0E0004AF422969D01255E3F4F02E11AE60E9436
:10B0F000D68DEFC4E9E4FAE6008111811A930A9330
:10B1000048EB50E060E08D010B5E1F4F0E944AF457
:10B1100022969D01255E3F4F01E41AE60E94D68DDE
:10B12000D8C4E3E5FAE6008111811A930A9348EB4B
:10B1300050E060E08D010B5E1F4F0E944AF42296A2
:10B140009D01255E3F4F0BE41AE60E94D68DC1C4D7
:10B150009D01255E3F4F04ED19E60E94D68DB9C4CE
:10B160000091C51D0670043041F49D01255E3F4FDE
:10B1700007E81AE60E94D68DACC49D01255E3F4FBC
:10B180000FE71AE60E94D68DA4C4E2ECFDE100812F
:10B19000118100701370012B39F40AE210E0EEE720
:10B1A000F1E100831183B2C4E1EFF5E80485158570
:10B1B0001A930A9348EB50E060E08D010B5E1F4F3D
:10B1C0000E944AF422969D01255E3F4F07E816E84B
:10B1D0000E94D68D7EC4E2E2FAE6008111811A93C4
:10B1E0000A9348EB50E060E08D010B5E1F4F0E9418
:10B1F0004AF422969D01255E3F4F04E21AE60E9422
:10B20000D68D67C4E7E3FAE6008111811A930A93A9
:10B2100048EB50E060E08D010B5E1F4F0E944AF446
:10B2200022969D01255E3F4F09E31AE60E94D68DC6
:10B2300050C40E9468A500E010E01A930A9348EBFE
:10B2400050E060E08D010B5E1F4F0E944AF4229691
:10B250009D01255E3F4F04EF11E10E94D68D39C458
:10B260000E9468A500E010E01A930A9348EB50E0B2
:10B2700060E08D010B5E1F4F0E944AF422969D01F3
:10B28000255E3F4F0CEF11E10E94D68D22C40E9433
:10B2900068A500E010E01A930A9348EB50E060E0E4
:10B2A0008D010B5E1F4F0E944AF422969D01255E80
:10B2B0003F4F04E012E10E94D68D0BC40E9468A5A6
:10B2C00000E010E01A930A9348EB50E060E08D0133
:10B2D0000B5E1F4F0E944AF422969D01255E3F4F50
:10B2E0000CE012E10E94D68DF4C30E9468A500E034
:10B2F00010E01A930A9348EB50E060E08D010B5E7A
:10B300001F4F0E944AF422969D01255E3F4F04E1A3
:10B3100012E10E94D68DDDC300E010E01A930A937B
:10B3200048EB50E060E08D010B5E1F4F0E944AF435
:10B3300022969D01255E3F4F04EF1FE90E94D68DA6
:10B34000C8C3ECEFF9E6008111811A930A9348EB28
:10B3500050E060E08D010B5E1F4F0E944AF4229680
:10B360009D01255E3F4F0EEF19E60E94D68DB1C3B9
:10B37000E6E0FAE6008111811A930A9348EB50E067
:10B3800060E08D010B5E1F4F0E944AF422969D01E2
:10B39000255E3F4F08E01AE60E94D68D9AC3EDED78
:10B3A000F9E6008111811A930A9348EB50E060E0BE
:10B3B0008D010B5E1F4F0E944AF422969D01255E6F
:10B3C0003F4F0FED19E60E94D68D83C3843600E00F
:10B3D000900764F1883C00E0900744F5AC0107E178
:10B3E00010E00E9446F2F801E854FE490081118104
:10B3F0001A930A9348EB50E060E08D010B5E1F4FFB
:10B400000E944AF422969D01255E3F4F49010EEBB2
:10B4100011E65801AC0107E110E00E9446F2A00ECF
:10B42000B11E850194010E94D68D53C3883C00E073
:10B43000900764F18C3201E0900744F5AC0107E11C
:10B4400010E00E9446F2F801E854FE4900811181A3
:10B450001A930A9348EB50E060E08D010B5E1F4F9A
:10B460000E944AF422969D01255E3F4F49010EEB52
:10B4700011E65801AC0107E110E00E9446F2A00E6F
:10B48000B11E850194010E94D68D23C38C3201E048
:10B49000900764F1803901E0900744F5AC0107E1C1
:10B4A00010E00E9446F2F801E854FE490081118143
:10B4B0001A930A9348EB50E060E08D010B5E1F4F3A
:10B4C0000E944AF422969D01255E3F4F49010EEBF2
:10B4D00011E65801AC0107E110E00E9446F2A00E0F
:10B4E000B11E850194010E94D68DF3C2803901E01E
:10B4F000900784F1843F01E0900764F5FC01E05976
:10B50000F1402F01A2010FEB10E00E9446F2F8017A
:10B51000EA5CF04E008111811A930A9348EB50E0E7
:10B5200060E08D010B5E1F4F0E944AF422969D0140
:10B53000255E3F4F490108E31FE15801A2010FEBCF
:10B5400010E00E9446F2A00EB11E850194010E94F7
:10B55000D68DBFC2843F01E0900784F1883502E0B8
:10B56000900764F5FC01E45FF1402F01A2010FEBAD
:10B5700010E00E9446F2F801EA5CF04E0285138565
:10B580001A930A9348EB50E060E08D010B5E1F4F69
:10B590000E944AF422969D01255E3F4F490102E434
:10B5A0001FE15801A2010FEB10E00E9446F2A00E2D
:10B5B000B11E850194010E94D68D8BC2883502E0B0
:10B5C000900764F18C3B02E0900744F5AC010FEB6F
:10B5D00010E00E9446F2F801E455F04A0081118122
:10B5E0001A930A9348EB50E060E08D010B5E1F4F09
:10B5F0000E944AF422969D01255E3F4F49010EEAC2
:10B600001FE55801AC010FEB10E00E9446F2A00EBE
:10B61000B11E850194010E94D68D5BC28C3B02E075
:10B62000900764F1803203E0900744F5AC010FEB22
:10B6300010E00E9446F2F801E65EFA4E00811181A8
:10B640001A930A9348EB50E060E08D010B5E1F4FA8
:10B650000E944AF422969D01255E3F4F49010CE16C
:10B6600015E15801AC010FEB10E00E9446F2A00E6C
:10B67000B11E850194010E94D68D2BC2803203E059
:10B68000900784F1843803E0900764F5FC01E052F0
:10B69000F3402F01A2010FEB10E00E9446F2F801E7
:10B6A000EA5CF04E02A913A91A930A9348EB50E002
:10B6B00060E08D010B5E1F4F0E944AF422969D01AF
:10B6C000255E3F4F49010AE61FE15801A2010FEB39
:10B6D00010E00E9446F2A00EB11E850194010E9466
:10B6E000D68DF7C1843803E0900764F1883E03E00B
:10B6F000900744F5AC010FEB10E00E9446F2F80110
:10B70000EA50F048008111811A930A9348EB50E007
:10B7100060E08D010B5E1F4F0E944AF422969D014E
:10B72000255E3F4F490108EF1FE75801AC010FEBC1
:10B7300010E00E9446F2A00EB11E850194010E9405
:10B74000D68DC7C1883E03E0900764F18C3404E0D5
:10B75000900744F5AC010FEB10E00E9446F2F801AF
:10B76000EC59FA4C008111811A930A9348EB50E08E
:10B7700060E08D010B5E1F4F0E944AF422969D01EE
:10B78000255E3F4F490106E615E35801AC010FEB7A
:10B7900010E00E9446F2A00EB11E850194010E94A5
:10B7A000D68D97C18C3404E0900784F1803B04E08F
:10B7B000900764F5FC01EC54F4402F01A2010FEB5B
:10B7C00010E00E9446F2F801EA57F04E0081118124
:10B7D0001A930A9348EB50E060E08D010B5E1F4F17
:10B7E0000E944AF422969D01255E3F4F490108E8D8
:10B7F0001FE15801A2010FEB10E00E9446F2A00EDB
:10B80000B11E850194010E94D68D63C1803B04E086
:10B81000900784F1843105E0900764F5FC01E05B5A
:10B82000F4402F01A2010FEB10E00E9446F2F80154
:10B83000EC55F04E008111811A930A9348EB50E0C9
:10B8400060E08D010B5E1F4F0E944AF422969D011D
:10B85000255E3F4F490106EA1FE15801A2010FEBA7
:10B8600010E00E9446F2A00EB11E850194010E94D4
:10B87000D68D2FC1843105E0900764F1883705E04B
:10B88000900744F5AC010FEB10E00E9446F2F8017E
:10B89000E453FA4A008111811A930A9348EB50E06D
:10B8A00060E08D010B5E1F4F0E944AF422969D01BD
:10B8B000255E3F4F49010EEC15E55801AC010FEB39
:10B8C00010E00E9446F2A00EB11E850194010E9474
:10B8D000D68DFFC0883705E0900764F18C3D05E008
:10B8E000900744F5AC010FEB10E00E9446F2F8011E
:10B8F000E65CF44F008111811A930A9348EB50E003
:10B9000060E08D010B5E1F4F0E944AF422969D015C
:10B91000255E3F4F49010CE31BE05801AC010FEBE2
:10B9200010E00E9446F2A00EB11E850194010E9413
:10B93000D68DCFC08C3D05E0900784F1803406E0C1
:10B94000900764F5FC01EC5DF5402F01A2010FEBBF
:10B9500010E00E9446F2F801E255F04E008111819C
:10B960001A930A9348EB50E060E08D010B5E1F4F85
:10B970000E944AF422969D01255E3F4F490100EB4B
:10B980001FE15801A2010FEB10E00E9446F2A00E49
:10B99000B11E850194010E94D68D9BC0803406E0C3
:10B9A000900764F1843A06E0900744F5AC010FEB90
:10B9B00010E00E9446F2F801E657FA480081118132
:10B9C0001A930A9348EB50E060E08D010B5E1F4F25
:10B9D0000E944AF422969D01255E3F4F49010CE8E2
:10B9E00015E75801AC010FEB10E00E9446F2A00EE3
:10B9F000B11E850194010E94D68D6BC0843A06E089
:10BA0000900764F1883007E0900744F5AC010FEB34
:10BA100010E00E9446F2F801EC5CF44D00811181C7
:10BA20001A930A9348EB50E060E08D010B5E1F4FC4
:10BA30000E944AF422969D01255E3F4F490106E38C
:10BA40001BE25801AC010FEB10E00E9446F2A00E81
:10BA5000B11E850194010E94D68D3BC0883007E05D
:10BA6000900784F18C3607E0900764F5FC01E850FC
:10BA7000F7402F01A2010FEB10E00E9446F2F801FF
:10BA8000E656F04E008111811A930A9348EB50E07C
:10BA900060E08D010B5E1F4F0E944AF422969D01CB
:10BAA000255E3F4F49010CE91FE15801A2010FEB50
:10BAB00010E00E9446F2A00EB11E850194010E9482
:10BAC000D68D07C005E110E0EEE7F1E100831183B8
:10BAD0001DC02AE230E08D010F5F1F4F0E941BAD99
:10BAE00010E01A930A934CE950E060E08D01055D87
:10BAF0001F4F0E944AF4229603E0FD0105A740E093
:10BB00002EE230E08D010E9459E507C0EEE7F1E139
:10BB10002081318105E50E9461ADEDE00C9469F36F
:10BB200000E010E0E4E8F1E100831183E2ECFDE1E4
:10BB3000008111810B7F11830083E2ECFDE1008124
:10BB400011811F771183008300E00093811D089508
:10BB500000E010E0E4E8F1E100831183E2ECFDE1B4
:10BB6000008111811F771183008300E00093811D04
:10BB700008950E9461F3D801C901E4E8F1E1008170
:10BB80001181080F191F01322EE41207A8F4AC012D
:10BB90009D0100E51FEAE4E8F1E160817181060F93
:10BBA000171F0E94C071E4E8F1E100811181080FC4
:10BBB000191F0083118306C00FEF1FEFE4E8F1E1C6
:10BBC00000831183E4E00C9472F3E4E8F1E1008176
:10BBD00011810F3F2FEF120769F0E4E8F1E10081D6
:10BBE0001181012B39F0E2ECFDE100811181106837
:10BBF00011830083089500E000937E1DEEE7F1E1DC
:10BC000000811181012B19F400E00093811D08953A
:10BC1000E2ECFDE10081118100701370012B41F411
:10BC2000E2ECFDE1008111810B7F11830083089517
:10BC3000E4E8F1E10081118109332AE4120740F0C0
:10BC4000E2ECFDE10081118104601183008308951D
:10BC5000E2ECFDE1008111810B7F118300830895E7
:10BC6000BA93AA9300E010E0EEE7F1E100831183BC
:10BC7000E2ECFDE10081118100701370012B39F0BD
:10BC80000AE210E0EEE7F1E1008311834BC0E2EC41
:10BC9000FDE100811181012F07FF3EC000E00E94FD
:10BCA0006386EEE7F1E100811181012BD9F5ECE12A
:10BCB000F4E030E0A7ECB1E00E94A5F407EC11E05D
:10BCC0000E94ACF4A80127EC31E0E6E8F1E1008144
:10BCD00011810E94C07101E00E940DA9E4E8F1E128
:10BCE0004081518120E53FEA00E113E10E94C071EB
:10BCF000E4E8F1E100811181E8E8F1E100831183DA
:10BD000000E00E94D3A802E000937F1D0E9465A876
:10BD100000E000937F1D06C00AE210E0EEE7F1E1CB
:10BD200000831183EEE7F1E12081318104E50E9477
:10BD300061ADA991B9910895BA93AA9300E010E07A
:10BD4000EEE7F1E100831183E2ECFDE10081118176
:10BD500000701370012B39F00AE210E0EEE7F1E118
:10BD60000083118357C00091811D002309F44CC04A
:10BD700000E00E946386EEE7F1E100811181012B72
:10BD800009F048C00091821D002351F006E210E046
:10BD9000E5EFF3E030E0A7ECB1E00E94A5F308C0C6
:10BDA00046E250E020E030E007EC11E00E94B3F3FF
:10BDB00046E250E027EC31E0E6E8F1E10081118154
:10BDC0000E94C07101E00E940DA9E4E8F1E1408108
:10BDD000518120E53FEA00E113E10E94C071E4E8EF
:10BDE000F1E100811181E8E8F1E10083118300E0D5
:10BDF0000E94D3A802E000937F1D0E9465A8FBDE8D
:10BE000000E000937F1D06C00AE210E0EEE7F1E1DA
:10BE100000831183EEE7F1E12081318104E50E9486
:10BE200061ADA991B991089545E150E020E030E07D
:10BE30000FE91AE60E94B3F3E8E8FEE10081118100
:10BE400022813381EFE9FAE6078310872187328761
:10BE5000E7EDFDE100811181EFE9FAE60387148740
:10BE60000FEF00939F6A08950E945DF3102E1A0150
:10BE7000888599850FEF00939F6AE3EDFDE10081CE
:10BE80001181EFE9FAE601831283E5EDFDE100811E
:10BE90001181EFE9FAE603831483EFE9FAE685837B
:10BEA0009683F9014080518062807380EFE9FAE661
:10BEB0004782508661867286F10100811181EFE927
:10BEC000FAE603871487ACEABAE68D01FB0148E085
:10BED00050E00E943FF310929F6AEAE00C946EF3E8
:10BEE0000E9462F3A02F04E510EAC80149E450E083
:10BEF00020E030E004E510EA0E94B3F340E050E0B7
:10BF00002A2F8C010E942CAD0091281F10E01A935B
:10BF10000A9349EA50E060E08C01005F1F4F0E94E5
:10BF20004AF42296EFE9FAE6018112811A930A9304
:10BF300048EB50E060E08C010D5E1F4F0E944AF418
:10BF4000229626EA3AE68C01075E1F4F0E9462A005
:10BF50002AEA3AE68C010E5D1F4F0E947FA00091F5
:10BF60009F6A10E01A930A934CE950E060E08C015C
:10BF7000095D1F4F0E944AF422969C01265D3F4FA7
:10BF80000CEA1AE60E94D68DEFE9FAE603811481E5
:10BF90001A930A9348EB50E060E08C01065C1F4F57
:10BFA0000E944AF4229600919F6A043021F0009189
:10BFB0009F6A053079F4EFE9FAE6058116811A9354
:10BFC0000A9348EB50E060E08C01005C1F4F0E9438
:10BFD0004AF4229625E430E08C010F5F1F4F0E9447
:10BFE0001BAD10E01A930A934CE950E060E08C011D
:10BFF0000A5B1F4F0E944AF4229603E0FC01E85BB3
:10C00000FF4F008340E029E430E08C010E9459E5B5
:10C01000E3E00C9473F39A938A9304E510EAC80161
:10C0200049E450E020E030E004E510EA0E94B3F378
:10C0300040E050E023E58C010E942CAD0091281FC8
:10C0400010E01A930A9349EA50E060E08C01005F27
:10C050001F4F0E944AF42296E1EFF5E8068117810E
:10C060001A930A9348EB50E060E08C010D5E1F4F7D
:10C070000E944AF4229621EF35E88C01075E1F4F9B
:10C080000E9462A025EF35E88C010E5D1F4F0E94D3
:10C090007FA00091FB8510E01A930A934CE950E0D1
:10C0A00060E08C01095D1F4F0E944AF422969C01BA
:10C0B000265D3F4F07E816E80E94D68DE1EFF5E8D0
:10C0C000008511851A930A9348EB50E060E08C01DB
:10C0D000065C1F4F0E944AF4229625E430E08C0152
:10C0E0000F5F1F4F0E941BAD10E01A930A934CE99B
:10C0F00050E060E08C010A5B1F4F0E944AF42296D8
:10C1000003E0FC01E85BFF4F008341E029E430E0FD
:10C110008C010E9459E589919991089500E000935E
:10C12000751D00E010E0E2E8F1E10083118308955D
:10C13000E2ECFDE10081118100701370012BF1F43C
:10C14000E1ECF1E000811181003A2AE01207B8F435
:10C15000E1ECF1E04081518124E530EA08E61BEE94
:10C160000E9497F3E1ECF1E000811181E2E8F1E156
:10C170000083118301E00093751D0895CFDF0895BA
:10C18000E2E8F1E100811181013A2AE0120708F0AA
:10C19000C5DFE2ECFDE10081118100701370012B1D
:10C1A000F9F40091751D0023A9F0E2E8F1E1408166
:10C1B000518128E63BEE04E510EA0E9497F3E2E89D
:10C1C000F1E100811181E1ECF1E0008311830E9433
:10C1D00031BB089525E230E00FE40E9461AD08957F
:10C1E0009DDF2AE230E00FE40E9461AD08950E94D5
:10C1F000E4A2013139F40AE210E0EEE7F1E1008354
:10C20000118309C011E006E20E94DE7010E0EEE743
:10C21000F1E100831183EEE7F1E12081318100E655
:10C220000E9461AD08950E94E4A2013151F002E044
:10C2300000930BA002E000930CA013E002E00E9428
:10C24000DE7008950E94E4A2013139F40AE210E0A0
:10C25000EEE7F1E1008311834EC0E2ECFDE10081E5
:10C26000118100FF07C002E010E0EEE7F1E100837A
:10C27000118341C0DCD510E0EEE7F1E100831183CA
:10C28000EEE7F1E100811181012B01F1EEE7F1E12F
:10C29000008111810A3420E01207C1F0EEE7F1E1DC
:10C2A000008111810F3420E0120781F0EEE7F1E107
:10C2B00000811181023320E0120741F0EEE7F1E145
:10C2C00000811181003520E0120731F400E010E018
:10C2D000EEE7F1E100831183EEE7F1E100811181E6
:10C2E000012B49F411E00AE00E94DE7010E0EEE755
:10C2F000F1E100831183EEE7F1E1208131810AE56C
:10C300000E9461AD08958A9380E00E94E4A2013109
:10C3100029F011E006E00E94DE70802F082F89913D
:10C3200008958A9311E004E10E94DE70802F082FA7
:10C33000899108958A93299701E000930BA012E058
:10C3400007E00E94DE70802F8823D1F444E023E1CF
:10C3500030EA8E010E9491908E010E94C7F1E2E2C4
:10C36000FFE1008311832283338345E027E130EA34
:10C370000DEF1FE90E94919000911CA00093261FD1
:10C38000082F2996899108958A9302E000930BA0C3
:10C3900012E007E00E94DE70802F813361F411E02B
:10C3A00009E30E94DE7002E000930BA012E007E0B8
:10C3B0000E94DE70802F082F899108950E9461F3FA
:10C3C0006F9780E0E2ECFDE10081118104FFADC0D8
:10C3D000DBDF802F882309F0A8C0009109A000931B
:10C3E000211F00910AA00093201FE0E2FFE10081DD
:10C3F0001181E8E8FEE1A481B58111960A171B07B7
:10C4000009F092C02BE030EA8E01005F1F4F0E94BE
:10C41000C0909E01205F3F4F8E010E94118E27E148
:10C4200030EA8E01005F1F4F0E94C0909E01205F86
:10C430003F4F8E01085F1F4F0E94118E2FE83EE193
:10C440008E010E943D89023071F42FED39E68E0194
:10C45000085F1F4F0E943D89023029F400917C1D26
:10C46000002309F462C00E94FB5104ED19E60E940A
:10C47000B7882FE83EE1BE018901FB0148E050E0AA
:10C480000E943FF32FED39E6BE01685F7F4F8901BF
:10C49000FB0148E050E00E943FF300917C1D002327
:10C4A000F9F40FE71AE60E94B78807E81AE60E9437
:10C4B000B7880E94B0752FE83AE66FE77AE68901FF
:10C4C000FB0148E050E00E943FF327E93AE667E8C5
:10C4D0007AE68901FB0148E050E00E943FF314C076
:10C4E0002FE73AE66FE87AE68901FB0148E050E081
:10C4F0000E943FF327E83AE667E97AE68901FB0103
:10C5000048E050E00E943FF32FE83EE10FE71AE6D3
:10C510000E94138A2FE83EE107E81AE60E94138A78
:10C5200001E000937C1D01C080E5082F6F96E4E0D8
:10C530000C9472F30E945DF3C80148E150E020E0E2
:10C5400030E008E01FE10E94B3F38C01012F00935B
:10C550000BA0082F00930CA013E003E20E94DE70F2
:10C56000602E662009F066C07724662009F062C05C
:10C57000772009F05FC0F9D5602E6620B1F70091F1
:10C5800009A00950C1F1055081F70AE010EA28011D
:10C59000F201008110E0E8E0FFE106831783E8E0A4
:10C5A000FFE10681102F00E0E8E0FFE1068317833A
:10C5B000F201018110E0E8E0FFE126813781202BC4
:10C5C000312B26833783F20102810E944F9010E0C5
:10C5D0000053184FE8E0FFE100831183F20103816B
:10C5E0000E944F9000930B1FF20104810E944F9014
:10C5F00000930A1FBACF0AE010EAD8019D0107ECA8
:10C6000011E00E94C09027EC31E000E11FE10E94A0
:10C61000118E9D01265F3F4F07EC11E00E94C090F4
:10C6200027EC31E008E11FE10E94118E6CDE7724D7
:10C6300073949BCF08E3601609F46624062DE8E0A6
:10C640000C946EF30E9461F3D80180E0E2ECFDE10E
:10C650000081118104FFA9C08D016CDF802F882328
:10C6600009F0A3C02FE83EE100E11FE10E943D89EF
:10C67000023001F52FED39E608E11FE10E943D8906
:10C680000230C1F428E83EE108E01FE10E9496A0D4
:10C69000023081F4E8E0FFE106811781E8E8FEE17D
:10C6A000248135810217130729F400917C1D002392
:10C6B00009F47BC00E94FB5104ED19E60E94B78883
:10C6C00040E450E020E030E008E81EE10E94B3F3CF
:10C6D000E8E0FFE10081118122813381E8E8FEE199
:10C6E0000083118322833383E8E0FFE10681178111
:10C6F000E8E8FEE1048315830FEF00938E1E2FE818
:10C700003EE160E17FE18901FB0148E050E00E94E9
:10C710003FF32FED39E668E17FE18901FB0148E055
:10C7200050E00E943FF300917C1D0023D9F40FE7F5
:10C730001AE60E94B7880E94B0752FE83AE66FE7C4
:10C740007AE68901FB0148E050E00E943FF327E9C7
:10C750003AE667E87AE68901FB0148E050E00E948A
:10C760003FF314C02FE73AE66FE87AE68901FB0150
:10C7700048E050E00E943FF327E83AE667E97AE6AE
:10C780008901FB0148E050E00E943FF32FE83EE1C1
:10C790000FE71AE60E94138A2FE83EE107E81AE63F
:10C7A0000E94138A01E000937C1D082FE4E00C94A2
:10C7B00072F30E945AF3A897480100919811005013
:10C7C00029F00A9531F00B5021F005C000E1A02EB0
:10C7D00002C002E1A02EA5DD902F992319F545E0B6
:10C7E00029E030EA8E010C5E1F4F0E94919048E2D2
:10C7F00050E020E230E084010E94B3F3E1EBF8E086
:10C8000030E0DE010E94A5F49E012C5E3F4F8E01B8
:10C810000E9472F48E010E94ACF4A8019E01840172
:10C820000E9497F3992309F093C080E0843608F0C2
:10C830008FC0992309F08CC0AAE4B2E1482F50E0E0
:10C8400007E110E00E9446F2A00FB11F8D010E9487
:10C85000F288002361F0482F50E007E110E00E94C9
:10C8600046F2F801E45CFD4E068900FF6FC080933C
:10C870000BA0482F50E007E110E00E9446F2F801BB
:10C88000E45CFD4E0281138124813581012B022B52
:10C89000032BF9F4482F50E007E110E00E9446F224
:10C8A000F801E45CFD4E068901FD13C008EE13E0BB
:10C8B00020E030E028013901482F50E007E110E086
:10C8C0000E9446F2F801E45CFD4E4282538264828B
:10C8D000758228E030E0D901482F50E007E110E0F0
:10C8E0000E9446F2F801E45CFD4E4281538164816E
:10C8F00075819D010CE010EA0E94119126E130EA59
:10C90000D9010AE4402E02E1502E482F50E007E101
:10C9100010E00E9446F2400E511E82019D010E94CD
:10C920008E8D4AE050E026E130EA06E210EA0E94ED
:10C93000F5904AE050E026E230EA00E110EA0E9479
:10C9400058901BE00A2D0E94DE70902F83956ECFC9
:10C95000992309F504EA11E10E94F2880023D9F431
:10C9600026E130EA04EA11E10E948E8D4AE050E0AF
:10C9700026E130EA06E210EA0E94F5904AE050E033
:10C9800026E230EA0BE010EA0E94589016E006E139
:10C990000E94DE70902F992309F50CEA11E10E94A4
:10C9A000F2880023D9F426E130EA0CEA11E10E9472
:10C9B0008E8D4AE050E026E130EA06E210EA0E945D
:10C9C000F5904AE050E026E230EA0BE010EA0E94DF
:10C9D000589016E007E10E94DE70902F092FA8966C
:10C9E000EBE00C946BF30E9460F3A897C801EEE8AB
:10C9F000F1E10081005D0E943C9000930BA000914A
:10CA000091110E943C9000930CA0009190110E9403
:10CA10003C9000930DA0009193110E943C900093D4
:10CA20000EA0009192110E943C9000930FA00091E3
:10CA3000281F009310A017E009E10E94DE70402E2D
:10CA400001E3401619F004E3401669F511E009E32B
:10CA50000E94DE70EEE8F1E10081005D0E943C90F2
:10CA600000930BA0009191110E943C9000930CA0A8
:10CA7000009190110E943C9000930DA000919311A1
:10CA80000E943C9000930EA0009192110E943C9055
:10CA900000930FA00091281F009310A017E009E158
:10CAA0000E94DE70402E4420B9F544E029E030EACF
:10CAB0008E010C5E1F4F0E9491909E012C5E3F4F95
:10CAC0008E010E949AF4E7EBF8E030E0DE010E946C
:10CAD00084F443E02DE030EA8E010C5E1F4F0E948B
:10CAE00091909E012C5E3F4F8E010E9472F48E0148
:10CAF0000E94ACF49E01119501951040AC01400FCD
:10CB0000511F485D5F4F8A010E949AF4E5E3F1E00E
:10CB100030E0DC010E9484F4042DA896E5E00C943A
:10CB200071F30E9459F3C80144240E94E4A2013128
:10CB300009F4AFC08C013DDE402E4420D9F0E3DB88
:10CB4000402E442011F0042D00C1F4DB402E44207F
:10CB500011F0042DFAC0E6E2FFE1008105FF02C0FA
:10CB600003E3F3C08C0125DE402E442019F0CBDB1B
:10CB7000042DEBC0442011F0042DE7C0E2E2FFE1F8
:10CB80000081118122813381480159018C012BDF01
:10CB9000402E442009F4D8C000E3401621F002E3FF
:10CBA000401609F074C05524442081F004E6501664
:10CBB00068F40BE919E521E0015010402040E1F74D
:10CBC00000C00000B7DB402E5394EECF442011F09C
:10CBD000042DBBC0E6E2FFE1008105FF0AC08C0125
:10CBE00002DF402E442019F08EDB03E3AEC0042D9B
:10CBF000ACC0E2E2FFE10081118122813381801625
:10CC00009106A206B30609F440C048E250E020E2D3
:10CC100030E08C010E94B3F301EB18E020E00E94A9
:10CC2000B6F4E1EBF8E030E0DC010E94A5F30DEF93
:10CC30001FE90E94ACF4D80101EB18E020E00E944B
:10CC4000B6F4B801AD012DEF3FE98C01060F171FB7
:10CC50000E9497F3E2E2FFE100811181228133819A
:10CC60003A932A931A930A9343EC50E060E08C01C4
:10CC7000085E1F4F0E944AF42496E5E3F1E030E09D
:10CC8000DC010E9484F400E060C003E35EC0042D78
:10CC90005CC048E250E020E230E08C010E94B3F337
:10CCA00001EB18E020E00E94B6F4E1EBF8E030E0A0
:10CCB000DC010E94A5F345E02EE231E10DEF1FE912
:10CCC0000E9491900DEF1FE90E94ACF4D80101EB96
:10CCD00018E020E00E94B6F4B801AD012DEF3FE965
:10CCE0008C01060F171F0E9497F30E94EC4D20E065
:10CCF00030E048015901E2E2FFE100811181228127
:10CD00003381A801B9014F5F5F4F6F4F7F4FE2E260
:10CD1000FFE14083518362837383BA92AA929A920D
:10CD20008A923A932A931A930A934AEB58E060E066
:10CD30008C01085E1F4F0E944AF42896E5E3F1E05B
:10CD400030E0DC010E9484F4042DECE00C946AF3E2
:10CD50008A9380E0E2ECFDE10081118104FF64C070
:10CD600011E009E30E94DE70802F882349F5E8E096
:10CD7000FFE10081005D0E943C9000930BA00091B8
:10CD80000B1F0E943C9000930CA000910A1F0E9470
:10CD90003C9000930DA000910D1F0E943C900093C9
:10CDA0000EA000910C1F0E943C9000930FA00091D8
:10CDB000281F009310A017E009E00E94DE70802F6A
:10CDC000882391F1B7DA802F882371F5E6E2FFE13D
:10CDD000008106FF29C0E8E0FFE10081005D0E94BC
:10CDE0003C9000930BA000910B1F0E943C9000937D
:10CDF0000CA000910A1F0E943C9000930DA000918E
:10CE00000D1F0E943C9000930EA000910C1F0E94E9
:10CE10003C9000930FA00091281F009310A017E0F2
:10CE200009E00E94DE70802F082F899108950E94EA
:10CE300061F380E00E94E4A2013109F454C07ADA7F
:10CE4000802F882309F04FC0E2ECFDE100811181C1
:10CE500004FF19C0E6E2FFE1008103FD02C08AE49D
:10CE60000BC045E050E027E130EA0EE211E10E94FC
:10CE70007FF3012B09F089E4E6E2FFE1008102FD86
:10CE800007C08FE405C0E6E2FFE1008103FD8DE409
:10CE9000E6E2FFE1008107FD8BE4E6E2FFE10081CD
:10CEA00005FD82E38823F9F4E2ECFDE100811181C4
:10CEB00004FF19C069DA802F8823A9F4009109A022
:10CEC0000093211F00910AA00093201FE0E2FFE1E0
:10CED00000811181E8E8FEE1A481B58111960A176D
:10CEE0001B0709F080E5082FE4E00C9472F3BC0105
:10CEF000E8E8FEE1248135812F5F3F4FE0E2FFE16A
:10CF00004081518124173507A0F4E0E2FFE1208140
:10CF10003181E8E8FEE144815581241B350B215025
:10CF20003040213010E0310711F400E011C000E57D
:10CF30000FC0E0E2FFE120813181E8E8FEE1848179
:10CF4000958101962817390711F400E001C000E52A
:10CF5000CB0108958A9380E00E94E4A2013141F060
:10CF600001E000930BA012E008E00E94DE70802F29
:10CF7000082F899108950E9455F3C8012901FC01E9
:10CF80000081005D0E943C9000930BA0FC01038196
:10CF90000E943C9000930CA0FC0102810E943C90F6
:10CFA00000930DA0F20101810E943C9000930EA01D
:10CFB000F20100810E943C9000930FA047E050E0F6
:10CFC00023E031E107EC11E00E9404724CE050E0F4
:10CFD000980100E110EA0E94F5904CE050E02BE14E
:10CFE00031E107EC11E00E94047298014CE050E03E
:10CFF0000CE110EA0E94589048E050E023E131E152
:10D0000007EC11E00E9404724CE050E0980102E24B
:10D0100010EA0E945890E8E8FEE11581012F009384
:10D0200028A0E8E8FEE10481009329A008E200932B
:10D030002AA048E250E020E230E00BE210EA0E9431
:10D04000B3F30DEF16E020E00E94B6F4EDEFF6E04A
:10D0500030E0A801ABE2B0EA8A010E94A5F31BE42C
:10D0600001E00E94DE70602E662009F07AC059D976
:10D07000602E662009F075C001E1802EFC01008160
:10D08000118122813381EAE2F1E10083118322835D
:10D09000338345E050E029E030EA0EE211E10E94DE
:10D0A00097F3E2ECFDE10081118104FF09C0E8E89B
:10D0B000FEE104811581EAE2F1E10687178706C0E7
:10D0C00000E010E0EAE2F1E10687178740E0282D52
:10D0D00030E0215030400AE211E10E94834D00937C
:10D0E0003A11EBE8F1E1008103950083482D50E00F
:10D0F00060E070E000918B1110E001501040212F92
:10D10000220F220B322F0E948CF2065511412D4F17
:10D110003F4F68017901A601B7012AE231E1082DEC
:10D1200010E00E949572002361F44BE050E863E048
:10D1300070E02BE831E101E010E00E9495720023DD
:10D1400029F00FE0602E01E00093791D662049F47C
:10D150000E949945012B29F00FE0602E01E0009319
:10D16000791D062DE0E10C9466F38A9311E005E049
:10D170000E94DE70802F082F8991089511E004EA43
:10D180000E94DE7010E0EEE7F1E100831183EEE72C
:10D19000F1E100811181012B09F05CC048E250E00F
:10D1A00020E230E007EC11E00E94B3F348E250E0E7
:10D1B00029E030EA07EC11E00E9497F300E00093C9
:10D1C000EF010E9474ACEEE7F1E100811181012BC7
:10D1D00011F5CBDF10E0EEE7F1E100831183EEE71C
:10D1E000F1E100811181012B71F748E250E020E26A
:10D1F00030E007EC11E00E94B3F348E250E029E090
:10D2000030EA07EC11E00E9497F300E00093EF0191
:10D210000E9474ACD8CFEEE7F1E1008111810833B0
:10D2200020E0120731F400E010E0EEE7F1E10083C6
:10D230001183EEE7F1E100811181012B59F400E047
:10D240000E94D3A802E000937F1D0E9465A800E021
:10D2500000937F1D58D808950E9461F3C801A22F42
:10D26000B32F8C01012F00930BA0082F00930CA06B
:10D2700013E00A2F0E94DE7010E0EEE7F1E1008378
:10D280001183EEE7F1E100811181012B09F06CC0FF
:10D29000E7E2FFE1008107FF09C0A33A39F441E06A
:10D2A00031E007E019E020E00E94A7AB48E250E03F
:10D2B00020E230E007EC11E00E94B3F348E250E0D6
:10D2C00029E030EA07EC11E00E9497F300E00093B8
:10D2D000EF010E9474ACEEE7F1E100811181012BB6
:10D2E00011F543DF10E0EEE7F1E100831183EEE793
:10D2F000F1E100811181012B71F748E250E020E259
:10D3000030E007EC11E00E94B3F348E250E029E07E
:10D3100030EA07EC11E00E9497F300E00093EF0180
:10D320000E9474ACD8CFEEE7F1E10081118108339F
:10D3300020E0120731F400E010E0EEE7F1E10083B5
:10D340001183EEE7F1E100811181012B69F4BB2328
:10D3500059F000E00E94D3A802E000937F1D0E94D4
:10D3600065A800E000937F1D0E948361E4E00C94B7
:10D3700072F39A938A93C80148E050E09C010BE055
:10D3800010EA0E94589015E001EA0E94DE7010E059
:10D39000EEE7F1E100831183EEE7F1E10081118115
:10D3A000012B09F05CC048E250E020E230E007ECDD
:10D3B00011E00E94B3F348E250E029E030EA07ECC4
:10D3C00011E00E9497F300E00093EF010E9474AC1B
:10D3D000EEE7F1E100811181012B11F5C6DE10E0CD
:10D3E000EEE7F1E100831183EEE7F1E100811181C5
:10D3F000012B71F748E250E020E230E007EC11E049
:10D400000E94B3F348E250E029E030EA07EC11E073
:10D410000E9497F300E00093EF010E9474ACD8CF14
:10D42000EEE7F1E100811181083320E0120731F4C9
:10D4300000E010E0EEE7F1E100831183EEE7F1E1B7
:10D4400000811181012B59F400E00E94D3A802E071
:10D4500000937F1D0E9465A800E000937F1D0E943D
:10D4600083618991999108950E9460F3402EC901CA
:10D47000DA0140920BA08C01012F00930CA0082F21
:10D4800000930DA08D01012F00930EA00A2F009391
:10D490000FA016E002EA0E94DE7010E0EEE7F1E174
:10D4A00000831183EEE7F1E100811181012B09F086
:10D4B0005CC048E250E020E230E007EC11E00E945E
:10D4C000B3F348E250E029E030EA07EC11E00E94B3
:10D4D00097F300E00093EF010E9474ACEEE7F1E1F6
:10D4E00000811181012B11F540DE10E0EEE7F1E142
:10D4F00000831183EEE7F1E100811181012B71F7C7
:10D5000048E250E020E230E007EC11E00E94B3F383
:10D5100048E250E029E030EA07EC11E00E9497F37E
:10D5200000E00093EF010E9474ACD8CFEEE7F1E188
:10D5300000811181083320E0120731F400E010E08F
:10D54000EEE7F1E100831183EEE7F1E10081118163
:10D55000012B59F400E00E94D3A802E000937F1D44
:10D560000E9465A800E000937F1D0E948361E5E0B2
:10D570000C9471F30E9460F3402ED901CA014092CD
:10D580000BA00D911197005D0E943C9000930CA0A0
:10D59000FD0103810E943C9000930DA0FD010281DA
:10D5A0000E943C9000930EA0FC010081005D0E944F
:10D5B0003C9000930FA0FC0103810E943C900093DB
:10D5C00010A0FC0102810E943C90009311A018E081
:10D5D00002EA0E94DE7010E0EEE7F1E100831183C1
:10D5E000EEE7F1E100811181012B09F05CC048E216
:10D5F00050E020E230E007EC11E00E94B3F348E293
:10D6000050E029E030EA07EC11E00E9497F300E0D7
:10D610000093EF010E9474ACEEE7F1E1008111810B
:10D62000012B11F5A2DD10E0EEE7F1E1008311839B
:10D63000EEE7F1E100811181012B71F748E250E042
:10D6400020E230E007EC11E00E94B3F348E250E042
:10D6500029E030EA07EC11E00E9497F300E0009324
:10D66000EF010E9474ACD8CFEEE7F1E100811181A7
:10D67000083320E0120731F400E010E0EEE7F1E1BA
:10D6800000831183EEE7F1E100811181012B59F450
:10D6900000E00E94D3A802E000937F1D0E9465A8CD
:10D6A00000E000937F1D0E948361E5E00C9471F31C
:10D6B000269700E010E0EEE7F1E1008311830E947D
:10D6C000E4A2013139F40AE210E0EEE7F1E100836F
:10D6D0001183C6C00091771D002339F001E110E0ED
:10D6E000EEE7F1E100831183BBC00091781D0023B8
:10D6F00039F009E010E0EEE7F1E100831183B0C0FA
:10D700000091791D002339F001E010E0EEE7F1E12E
:10D7100000831183A5C0E2ECFDE10081118104FDCD
:10D7200007C004E110E0EEE7F1E10083118398C047
:10D73000E2ECFDE10081118100FF07C002E010E092
:10D74000EEE7F1E1008311838BC000918B1104316E
:10D7500038F00CE410E0EEE7F1E10083118380C0C3
:10D760000E949A6110E0EEE7F1E100831183EEE799
:10D77000F1E100811181012B09F072C0E2ECFDE1C1
:10D780000081118104FF0CC0E8E0F0EA048903FF86
:10D7900007C00DE410E0EEE7F1E10083118360C003
:10D7A0009E018E010E5F1F4F0E947EB9EEE7F1E1F0
:10D7B00000831183EEE7F1E100811181012B09F073
:10D7C0004FC00A811B81003D27E0120730F00A811B
:10D7D0001B81033028E0120738F007E010E0EEE785
:10D7E000F1E1008311833CC021E08E010E5F1F4FE9
:10D7F0000E94F3E9EEE7F1E100831183EEE7F1E146
:10D8000000811181012B61F500E00E946386EEE743
:10D81000F1E100811181012B19F59E018E010E5F4E
:10D820001F4FA9DB10E0EEE7F1E100831183EEE783
:10D83000F1E100811181012B99F401E00E940DA911
:10D84000E2ECFDE10081118101FF05C010E000E183
:10D850000E9421A904C010E000E00E9421A98EDCF2
:10D86000EEE7F1E12081318108E50E9461AD269665
:10D8700008950E945FF30AE510EAD80100E010E085
:10D88000EEE7F1E1008311830E94E4A2013139F453
:10D890000AE210E0EEE7F1E10083118354C1009148
:10D8A000771D002339F001E110E0EEE7F1E100839C
:10D8B000118349C10091781D002339F009E010E07F
:10D8C000EEE7F1E1008311833EC1B1DA10E0EEE74B
:10D8D000F1E100831183EEE7F1E100811181012B79
:10D8E00001F1EEE7F1E1008111810A3420E0120735
:10D8F000C1F0EEE7F1E1008111810F3420E0120761
:10D9000081F0EEE7F1E100811181023320E012079E
:10D9100041F0EEE7F1E100811181003520E01207CE
:10D9200031F400E010E0EEE7F1E100831183EEE76F
:10D93000F1E100811181012B09F005C147E350E0BD
:10D9400020E330E00C9110E00E94D3EAEEE7F1E131
:10D9500000831183EEE7F1E100811181012B09F0D1
:10D96000F2C000E00E946386EEE7F1E100811181E0
:10D97000012B09F0E8C00AE510EAD80101E00E9495
:10D980000DA9E2ECFDE10081118101FF05C010E06D
:10D9900000E10E9421A904C010E000E00E9421A93A
:10D9A0000C91E4EDF0E0FBBFF3E70C94FAF2E6DB58
:10D9B000CAC08D010E5F1F4F0E9482F1C80148EB63
:10D9C0005BE021E030E08C010E94D3EAEEE7F1E178
:10D9D00000831183EEE7F1E100811181012B09F051
:10D9E000B2C031E023EA8C0137DCADC08D010E5F9F
:10D9F0001F4F0E9482F1C80148EB5BE021E030E05C
:10DA00008C010E94D3EAEEE7F1E100831183EEE797
:10DA1000F1E100811181012B09F095C08D01055FB5
:10DA20001F4F0E9482F1280148EB5BE021E030E0CB
:10DA300082010E94D3EAEEE7F1E100831183EEE771
:10DA4000F1E100811181012B09F07DC048165906D2
:10DA50003CF405E010E0EEE7F1E10083118373C0D0
:10DA60000C91023329F4A2019C0106E0FDDC6BC09D
:10DA7000A2019C0107E0F8DC66C021E93DE18D01CF
:10DA80000E5F1F4F0E9426A0EEE7F1E10083118395
:10DA9000EEE7F1E100811181012B09F054C025E985
:10DAA0003DE18D01055F1F4F0E9426A0EEE7F1E1E9
:10DAB00000831183EEE7F1E100811181012B09F070
:10DAC00042C00C91043339F445E95DE121E93DE1BF
:10DAD00004E050DD38C045E95DE121E93DE105E0C4
:10DAE00049DD31C028E030E08D010E5F1F4F0E94FC
:10DAF000FAEAEEE7F1E100831183EEE7F1E100815C
:10DB00001181012B01F58D010E5F1F4F32DC1BC00F
:10DB10008D010E5F1F4F0E9482F1C80148EB5BE050
:10DB200021E030E08C010E94D3EAEEE7F1E10083CE
:10DB30001183EEE7F1E100811181012B21F431E045
:10DB400020EA8C0189DBEEE7F1E12081318109E5F2
:10DB50000E9461ADE6E00C9470F30E9460F3A89718
:10DB6000C80110E000E00E94DE70402E442009F061
:10DB700063C044E029E030EA8E010E9491909E014A
:10DB80008E010C5E1F4F0E949AF4E7EBF8E030E044
:10DB9000DE0154960E9484F443E02DE030EA8E01C9
:10DBA0000E9491909E018E010C5E1F4F0E9472F4A4
:10DBB0009E012C5E3F4F8C010E949AF40E9491615D
:10DBC000402E4420C9F545E029E030EA8E010E944C
:10DBD0009190E1EBF8E030E0DE0154960E94A5F46C
:10DBE0009E018E010C5E1F4F0E9472F49C018E01FB
:10DBF0000E949AF448E250E020E230E08C010E945A
:10DC0000B3F38E010C5E1F4F0E94ACF4A8019E017D
:10DC10002C5E3F4F8C010E9497F38E010E94ACF462
:10DC2000A8019E015195419550408C01040F151F8C
:10DC3000085D1F4F0E949AF4042DA896E5E00C940D
:10DC400071F30E9461F30091861D002309F06EC0FC
:10DC50000E945EA8E3EDFDE1008111811A930A9311
:10DC60004AEF51E060E00DE012E00E944AF4229693
:10DC7000E2ECFDE10081118101FF07C031E121E10A
:10DC80000DE012E00E9410AC06C031E021E00DE092
:10DC900012E00E9410AC2AE13AE604E21AE60E9481
:10DCA000138AE2E2FAE6008111810F5F1F4F0083C1
:10DCB00011832AE13AE6C901A0EBBFE14091281F98
:10DCC00050E00FEB10E00E9446F2A00FB11F8D0153
:10DCD0009C010E94138A4091281F50E00FEB10E036
:10DCE0000E9446F2F801E255F04E008111810F5F6B
:10DCF0001F4F0083118300E010E0E3EDFDE100839E
:10DD00001183E1EDFDE1008111810F5F1F4F008361
:10DD10001183E5EDFDE1008111810F5F1F4F00834D
:10DD20001183ECEDFDE100810F700083E4E00C94C1
:10DD300072F30E945DF3239700917F1D023029F05A
:10DD400000917F1D033009F007C101E00093B90184
:10DD500000917F1D023009F0C8C0E9E3F1E00491B1
:10DD6000009354A0EAE3F1E00491009355A0E2ECA3
:10DD7000FDE10081118101FF04C001E8009356A07C
:10DD800003C000E8009356A0EFE7F4E030E0A7E519
:10DD9000B0EA0E94A5F403E412E020E00E9459AB2F
:10DDA00027EC31E007E510EA0E9472F40DED1DE169
:10DDB0000E94ACF4012BC9F0ECEDFDE1008100FD07
:10DDC00014C0E4ECFDE1008100FF05C00DED1DE194
:10DDD0000E947FAB04C00DED1DE10E9435AB27EC26
:10DDE00031E007E510EA0E9472F406E01EE10E94AD
:10DDF000ACF4012BC9F0ECEDFDE1008101FD14C094
:10DE0000E4ECFDE1008100FF05C006E01EE10E9498
:10DE10007FAB04C006E01EE10E9435AB27EC31E089
:10DE200007E510EA0E9472F40FE21EE10E94ACF4D2
:10DE3000012BC9F0ECEDFDE1008102FD14C0E4EC22
:10DE4000FDE1008100FF05C00FE21EE10E947FABF3
:10DE500004C00FE21EE10E9435AB27EC31E007E57C
:10DE600010EA0E9472F408E51EE10E94ACF4012B56
:10DE7000C9F0ECEDFDE1008103FD14C0E4ECFDE12F
:10DE8000008100FF05C008E51EE10E947FAB04C0D1
:10DE900008E51EE10E9435AB27EC31E007E510EA0A
:10DEA0000E9472F424E530EA07EC11E00E949AF433
:10DEB000E7E3F1E030E0A7ECB1E00E9484F407EC86
:10DEC00011E00E94ACF4A80127EC31E000E71DEF5F
:10DED0000E94C07100E71DEF0E94A1A80E94B4A695
:10DEE00003E000937F1D0E945EA800917F1D033018
:10DEF00079F5E4ECFDE1008102FD27C0E1E8FEE1F7
:10DF000000811181012BE1F0E9E3F1E00491088344
:10DF1000EAE3F1E004910983E2ECFDE10081118183
:10DF200001FF03C000E90A8302C000E80A8343E05E
:10DF300050E09E01E1E8FEE1008111810E94D17173
:10DF400000E00E940DA90E94B4A600E000937F1D8E
:10DF500000E00093B90127C1E3EDFDE100811181EB
:10DF6000012B49F4E2ECFDE1008111810070137096
:10DF7000012B09F418C101E00093B901E2ECFDE1C5
:10DF80000081118101FF05C010E001E10E9421A97B
:10DF900004C010E001E00E9421A9EFE7F4E030E0C6
:10DFA000A7ECB1E00E94A5F4E7E3F1E030E0A7ECD4
:10DFB000B1E00E9484F407EC11E00E94ACF4A801E7
:10DFC00027EC31E000E71DEF0E94C07100E71DEF74
:10DFD0000E94A1A8E2ECFDE10081118104FFCBC009
:10DFE000E2ECFDE10081118100701370012B09F456
:10DFF000C0C00E94E4A2013109F4B9C0E2E2FFE12D
:10E000000081118122813381280139010DE012E064
:10E01000A4DD002309F0A9C00E941767002309F0BE
:10E02000A2C0E2E2FFE1008111812281338140162A
:10E0300051066206730609F494C00E94E15200E0A2
:10E0400010E01A930A9364E272E142E951E12EE88A
:10E0500031E1009198110E94345FE1EDFDE1008112
:10E0600011810F5F1F4F00831183E5EDFDE10081FA
:10E0700011810F5F1F4F0083118300E010E0E3ED7B
:10E08000FDE100831183E2ECFDE10081118100607C
:10E090001C6700831183E2ECFDE1008111810F7F99
:10E0A0001C7F0083118300919811002381F406E204
:10E0B00010E0E5EFF3E030E0A7ECB1E00E94A5F35B
:10E0C00040E026E230E007EC11E00E94EFA700916B
:10E0D0009811002341F000919811013021F0009136
:10E0E00098110C3031F5E2ECFDE10081118101FF66
:10E0F00005C011E001E10E9421A904C011E001E086
:10E100000E9421A92DE032E007EC11E00E949AF470
:10E110000E9474ACE2ECFDE10081118101FF05C0B9
:10E1200011E000E10E9421A904C011E000E00E947A
:10E1300021A900E00E94D3A802E000937F1D0E9465
:10E14000B4A600E000937F1D0E945EA8E4ECFDE110
:10E15000008102FD11C000E00E940DA90E94B4A63A
:10E160000BC06FDD09C06DDD07C06BDD05C069DD6B
:10E1700003C067DD01C065DD01E00E940DA90E94BA
:10E1800082A8E4ECFDE1008102FD05C000E00E94F0
:10E190000DA90E9465A800E000937F1D0E945EA863
:10E1A00000E00093B9012396E8E00C946EF300E0E0
:10E1B0000093261F00E00093271F08950E9461F33B
:10E1C00021971883902F80E00881002309F445C02F
:10E1D000A0E0A430B0F40E945C7310E004E00E9460
:10E1E0007273802F882369F00E94677307E110E83B
:10E1F0002DE0015010402040E1F700C00000A39541
:10E20000E8CF882339F502E0009308A00881009345
:10E2100009A090930AA00881802F08810E5F0883CF
:10E22000A2E00881A01740F4B0E0FD01E85FFF45DF
:10E2300000818027A395F5CF088110E0F801E85F01
:10E24000FF45808328E030EA088103950E94F97336
:10E25000802F01C080E30E946773882309F083C088
:10E26000A0E0A430B0F40E945C7311E004E00E94CE
:10E270007273802F882369F00E94677307E110E8AA
:10E280002DE0015010402040E1F700C00000A395B0
:10E29000E8CF882309F063C040E09E0101E010E070
:10E2A0000E94B7730881023011F086E459C040E043
:10E2B0009E0101E010E00E94B7730881002319F06D
:10E2C00008810D3410F087E44BC008810395088362
:10E2D00041E028E030EA088110E00E94B77300E0D6
:10E2E000288130E0F901E85FFF45008308810A9545
:10E2F00008830881802FA0E00881A01740F4B0E0D7
:10E30000FD01E85FFF4500818027A395F5CF0881D7
:10E3100010E0F801E85FFF450081801711F088E404
:10E3200001C080E08823E1F4009108A00F7700236A
:10E3300029F0009108A00F77005D802FE8E0F0EA57
:10E34000008107FF06C0E7E2FFE10081006800836B
:10E3500007C0E7E2FFE100810F77008301C080E39F
:10E360000E94677301C080E300E010E90150104093
:10E37000E9F700C00000082F2196E4E00C9472F346
:10E380000E945FF32801D901CA010E94C73FAC0176
:10E390009D0182010E9497F30E94C93FE6E00C9420
:10E3A00070F30E945DF3D801C9012A016624772425
:10E3B0006414750468F4FC01E60DF71D20818D01DD
:10E3C000060D171D08D001E0600E00E0701EF0CFB2
:10E3D000E8E00C946EF30E9461F3D801822F0E9452
:10E3E000C73F8C930E94C93FE4E00C9472F30E94F3
:10E3F00061F3D8010E94C73F0C91802F0E94C93F52
:10E40000082FE4E00C9472F30E945FF32801D90115
:10E41000CA01AC019D0182010E9497F300E0F20164
:10E42000E80FF91F00838201E6E00C9470F30C0101
:10E43000B80180E08531A0F490E0A901480F591F90
:10E440000E9428F290E0FB01E80FF91F008390E0A2
:10E45000FB01E80FF91F0081002311F08395EACF3B
:10E4600000E090E0FB01E80FF91F0083C001089570
:10E470000E9461F31801DA01962F20E02531D0F4D3
:10E48000022F10E0FD01392FE00FF11F3BBF069175
:10E4900030E0A101420F531F0E9434F2022F10E01E
:10E4A000FD01392FE00FF11F3BBF0691002311F052
:10E4B0002395E4CFE4E00C9472F3392E782FC80151
:10E4C0000A01262E60E020E02531B0F430E0AC01F6
:10E4D000420F531F0E9428F2602F022F10E0F0011C
:10E4E000322DE00FF11F3BBF0691601721F4662328
:10E4F00019F02395E9CF61E0062F872F932D08951A
:10E500000E945CF338012901CA01DB01BA93AA9386
:10E510009A938A9313E0A201930100EA0E94117476
:10E52000802E082DE9E00C946DF30E9455F324979A
:10E53000488359836A837B837801C901AA240881AF
:10E5400019812A813B8128013901A0E0B0E08701CF
:10E55000980145E089010E9454F268018701980101
:10E5600040E250E089010E9460F24A010C2D0D2921
:10E57000E1F0AA20D1F403E00A93A201B3019C01C7
:10E580002A0F3B1F10E200EA0E945674A02E9096BC
:10E5900000E2400E00E0501E00E0601E00E0701E31
:10E5A0000FEFC00E0FEFD01EE1CF082D092971F03B
:10E5B000AA2061F403E00A93A201B3019C012A0F8F
:10E5C0003B1F182D00EA0E945674A02E0A2D249697
:10E5D000E0E10C9466F306EC00C00A95E9F70895B3
:10E5E00005EA0A95F1F708950EE60A95F1F7089500
:10E5F00005E50A95F1F7089501E40A95F1F7089504
:10E6000007E30A95F1F7089502E30A95F1F70895F3
:10E6100008E20A95F1F7089503E20A95F1F70895E3
:10E620000EE10A95F1F708950EE10A95F1F70895C4
:10E6300009E10A95F1F7089509E10A95F1F70895BE
:10E6400009E10A95F1F7089504E10A95F1F70895B3
:10E6500004E10A95F1F7089504E10A95F1F70895A8
:10E6600004E10A95F1F7089504E10A95F1F7089598
:10E670000FE00A95F1F70895EAE8FAE00091D01D5D
:10E6800010E0000F111FE00FF11F05911491F80128
:10E690000995089501B30C7F01BB02B30C7F02BB47
:10E6A0000E94E4A2003121F00E94E4A2013019F49A
:10E6B00000E00093D01D08958998DEDF8898809B44
:10E6C000FECFDADF899AD8DF889AD6DF0895889A54
:10E6D000D3DF899AD1DF8898809BFECFCDDF8998E0
:10E6E000CBDF08950E9461F3B02FA12F80E8889AB4
:10E6F000BA2B90E09830A0F4082F10E0492F0E9428
:10E700005AF20B23002311F0899801C0899AB4DFD3
:10E710008898809BFECFB0DF889AAEDF9395EACFD2
:10E720008998AADF8898809BFECFA6DF00B302708D
:10E73000902F889AA1DF092FE4E00C9472F30E94D5
:10E7400061F3902F81E0A0E0B0E0A83B0BE0B007C0
:10E7500050F4882341F0B0DF10E0092FC3DF802F91
:10E76000B6DF1196F2CF082FE4E00C9472F30E940A
:10E770005BF32801C901842EA0E8889A7DDF89987F
:10E780007BDF662477246414750480F59924B0E057
:10E79000B83080F48898809BFECF6EDF819B06C0E6
:10E7A0000A2F10E04B2F0E945AF2902A889A64DFB9
:10E7B000B395EECFF20131976E167F0621F48820D3
:10E7C00011F0899801C0899A57DF8898809BFECF05
:10E7D00053DF889A51DF89984FDFFC01E60DF71D62
:10E7E000908201E0600E00E0701ECDCFEAE00C9454
:10E7F0006CF30E945FF3402EC9015524A0E0A415DC
:10E8000060F4552051F410E0B0E0FC01EA0FFB1F6A
:10E81000008168DF502EA395F2CF052DE6E00C9421
:10E8200070F30E9459F3602E59012A01912E8C85B4
:10E830009D85AE85BF85062D82DF802E882091F5CF
:10E840003BDF10E0062D4EDF802E882059F503E0D7
:10E85000901691F49D01022F702E689472F810E0CA
:10E86000072D40DF802E882039F48C01012F702E77
:10E8700010E0072D37DF802E8820A1F48C01702E48
:10E8800010E0072D2FDF802E882061F415DF11E0C6
:10E89000062D28DF802E882029F441E09201850191
:10E8A00066DF15DF082DE0E10C946AF30E945AF34D
:10E8B000A02E412E4901CA01DB015B840A2D3FDFF6
:10E8C000702E7720A1F5F8DE10E00A2D0BDF702EF8
:10E8D000772069F503E05016D9F49D01022F302FFF
:10E8E000042D10E00150104043E00E944EF2032B33
:10E8F000602EE89462F810E0062DF4DE702E77208A
:10E9000039F48C01012F602E10E0062DEBDE702E05
:10E91000772069F48C01602E10E0062DE3DE702E66
:10E92000772029F49401042D64DF702ED0DE072DAA
:10E93000ECE00C946BF30E9461F304E510EAC8016B
:10E9400048E750E020E030E004E510EA0E94B3F32D
:10E9500040E050E025E48C010E942CAD47E050E0FF
:10E9600023E031E18C01005F1F4F0E9404724DEFE4
:10E9700056E060E08C01085E1F4F0E944AF44BE2B3
:10E9800051E060E08C01095C1F4F0E944AF4EBE00B
:10E99000F7E030E0DC01D7960E9484F44AE157E0CA
:10E9A00060E08C010A5A1F4F0E944AF424E730E0CD
:10E9B0008C010F5F1F4F0E941BAD10E01A930A934A
:10E9C0004CE950E060E08C010B581F4F0E944AF464
:10E9D000229603E0FC01E958FF4F008340E028E75E
:10E9E00030E08C010E9459E5E4E00C9472F3BA9394
:10E9F000AA9304E510EAD8014CE350E020E030E0AF
:10EA000004E510EA0E94B3F340E050E024E48D01F5
:10EA10000E942CAD05E010E020918A1130E0021B2D
:10EA2000130B1A930A9343EB50E060E08D01005FF3
:10EA30001F4F0E944AF4229608EB1BE0ECE8F1E13C
:10EA400020813181021B130B1A930A9343EB50E090
:10EA500060E08D010B5E1F4F0E944AF42296ECE7A6
:10EA6000F1E1008111811A930A9348EB50E060E0D4
:10EA70008D01065E1F4F0E944AF42296E8E8FEE1EF
:10EA8000048115811A930A9348EB50E060E08D01F0
:10EA9000005E1F4F0E944AF42296E2ECFDE10081E5
:10EAA000118100FF0EC028E83EE18D010A5D1F4F75
:10EAB0000E9462A027ED3DE18D01015D1F4F0E9484
:10EAC0007FA004E110E020918B1130E0021B130BBA
:10EAD0001A930A9343EB50E060E08D010C5C1F4FEA
:10EAE0000E944AF4229628E330E08D010F5F1F4F09
:10EAF0000E941BAD10E01A930A934CE950E060E0CD
:10EB00008D01075C1F4F0E944AF4229603E0FD012D
:10EB100003AF40E02CE330E08D010E9459E5A9915C
:10EB2000B9910895219740E050E060E070E09E01C7
:10EB300001E010E00E9480720881002341F4E2ECC1
:10EB4000FDE10081118100611183008307C0E2ECC7
:10EB5000FDE1008111810F7E1183008321960895CC
:10EB60000E9459F3A0E0B0E080E490E0E2ECFDE127
:10EB70000081118104FF6EC002EB1DE10E94B78885
:10EB80000AEB1DE10E94B78844245524ECE8F1E12A
:10EB9000008111814016510608F04DC00A2F0B2B41
:10EBA00009F049C040E0959D9001849D8001949DAD
:10EBB000100D211D341F589E100D211D341F0655A8
:10EBC0001F4F2F4F3F4F48015901A401B5012BE3BF
:10EBD00031E18C010E948072002319F0A6E1B0E0BF
:10EBE00025C040917A119C01215030400BE311E186
:10EBF0000E94834D0023C1F422E431E102EB1DE1C8
:10EC00000E94138AEAE0F1E1058D168DEBE3F1E154
:10EC1000248135810217130748F422E431E10AEB1D
:10EC20001DE10E94138A02C0A1E0B0E001E0400EA5
:10EC300000E0501EABCF0A2F0B2B61F422EB3DE11D
:10EC40000FE71AE60E94DD882AEB3DE107E81AE6A5
:10EC50000E94DD88ECE00C946AF30E945DF3249737
:10EC6000602E512E80E0442490E000E010E0E1E8C6
:10EC7000FEE1008311830DED1DE10E94ACF4012B38
:10EC800029F0ECEDFDE1008100FF43940DED1DE165
:10EC90000E94ACF4012B29F0ECEDFDE1008101FFB5
:10ECA00043940DED1DE10E94ACF4012B29F0ECED35
:10ECB000FDE1008102FF43940DED1DE10E94ACF4E3
:10ECC000012B29F0ECEDFDE1008103FF4394062DBB
:10ECD0000419702E01E00E940DA90E944F4DE2EC34
:10ECE000FDE10081118101FF05C010E000E90E94F3
:10ECF00021A904C010E000E80E9421A9E4ECFDE194
:10ED0000008101FF02C0552071F0871560F40BEA05
:10ED100011E00E94ACF440E098010BEA11E00E947F
:10ED2000EFA78395F2CFE4ECFDE1008101FF02C083
:10ED30005520F9F0082F10E0E62DF0E031970E177E
:10ED40001F07BCF09923A9F40E949AA8E1E8FEE10C
:10ED500000831183EEE4F1E030E0DE010E94A5F4CF
:10ED60008E010E94ACF4980140E08E010E94EFA752
:10ED700091E00DED1DE10E94ACF4012B09F448C0B7
:10ED8000ECEDFDE1008100FD3DC0E4ECFDE1008122
:10ED900000FF05C00DED1DE10E9486AC06C030E00D
:10EDA00020E80DED1DE10E9410ACECEDFDE10081CD
:10EDB000006100838395E4ECFDE1008101FF02C066
:10EDC000552059F1082F10E0E62DF0E031970E178D
:10EDD0001F071CF1992309F50E949AA8E1E8FEE1BA
:10EDE00000831183EEE4F1E030E0DE010E94A5F43F
:10EDF0008E010E94ACF440E098018E010E94EFA7C2
:10EE000091E00BC0ECEDFDE100810F7E008305C0B9
:10EE1000ECEDFDE100810F7E008306E01EE10E9423
:10EE2000ACF4012B09F448C0ECEDFDE1008101FDDB
:10EE30003DC0E4ECFDE1008100FF05C006E01EE1FD
:10EE40000E9486AC06C030E020E806E01EE10E9489
:10EE500010ACECEDFDE10081006200838395E4ECF1
:10EE6000FDE1008101FF02C0552059F1082F10E09B
:10EE7000E62DF0E031970E171F071CF1992309F5D5
:10EE80000E949AA8E1E8FEE100831183EEE4F1E03C
:10EE900030E0DE010E94A5F48E010E94ACF440E057
:10EEA00098018E010E94EFA791E00BC0ECEDFDE10F
:10EEB00000810F7D008305C0ECEDFDE100810F7D39
:10EEC00000830FE21EE10E94ACF4012B09F448C05C
:10EED000ECEDFDE1008102FD3DC0E4ECFDE10081CF
:10EEE00000FF05C00FE21EE10E9486AC06C030E0C4
:10EEF00020E80FE21EE10E9410ACECEDFDE1008184
:10EF0000006400838395E4ECFDE1008101FF02C011
:10EF1000552059F1082F10E0E62DF0E031970E173B
:10EF20001F071CF1992309F50E949AA8E1E8FEE168
:10EF300000831183EEE4F1E030E0DE010E94A5F4ED
:10EF40008E010E94ACF440E098018E010E94EFA770
:10EF500091E00BC0ECEDFDE100810F7B008305C06B
:10EF6000ECEDFDE100810F7B008308E51EE10E94CE
:10EF7000ACF4012B09F447C0ECEDFDE1008103FD89
:10EF80003CC0E4ECFDE1008100FF05C008E51EE1A6
:10EF90000E9486AC06C030E020E808E51EE10E9431
:10EFA00010ACECEDFDE10081006800838395E4EC9A
:10EFB000FDE1008101FF02C0552051F1082F10E052
:10EFC000E62DF0E031970E171F0714F1992301F594
:10EFD0000E949AA8E1E8FEE100831183EEE4F1E0EB
:10EFE00030E0DE010E94A5F48E010E94ACF440E006
:10EFF00098018E010E94EFA70BC0ECEDFDE10081AE
:10F000000F77008305C0ECEDFDE100810F770083F1
:10F010002496E8E00C946EF301E00E940DA90E9492
:10F020004F4DE2ECFDE10081118101FF05C010E0D0
:10F0300000E90E9421A904C010E000E80E9421A973
:10F040000DED1DE10E94ACF4012BD1F00091DC1D0F
:10F050000F700F3029F00091DC1D0171002381F445
:10F06000E4ECFDE1008100FF05C00DED1DE10E9413
:10F0700086AC06C030E020E80DED1DE10E9410AC2A
:10F0800006E01EE10E94ACF4012BD1F00091DC1DE2
:10F090000F700F3029F00091DC1D0272002381F403
:10F0A000E4ECFDE1008100FF05C006E01EE10E94E6
:10F0B00086AC06C030E020E806E01EE10E9410ACFD
:10F0C0000FE21EE10E94ACF4012BD1F00091DC1D97
:10F0D0000F700F3029F00091DC1D0474002381F4BF
:10F0E000E4ECFDE1008100FF05C00FE21EE10E949B
:10F0F00086AC06C030E020E80FE21EE10E9410ACB2
:10F1000008E51EE10E94ACF4012BD1F00091DC1D5A
:10F110000F700F3029F00091DC1D0878002381F476
:10F12000E4ECFDE1008100FF05C008E51EE10E945E
:10F1300086AC06C030E020E808E51EE10E9410AC75
:10F14000E2ECFDE10081118101FF05C010E001E961
:10F150000E9421A904C010E001E80E9421A920E03A
:10F1600030E007EC11E00E94177247E050E023E026
:10F1700031E10DE012E00E9404722DE032E007EC74
:10F1800011E00E9472F40E9474ACE2ECFDE1008197
:10F19000118104FF15C02BE331E007EC11E00E9460
:10F1A00017724CE050E02BE131E10DE012E00E94DB
:10F1B00004722DE032E007EC11E00E9472F407C007
:10F1C0004DE954E060E007EC11E00E944AF40E942F
:10F1D00074ACE2ECFDE10081118101FF05C010E09B
:10F1E00001E10E9421A904C010E001E00E9421A9D0
:10F1F00025E130E007EC11E00E941772E3EDFDE13C
:10F20000008111811A930A9348EB50E060E00DE011
:10F2100012E00E944AF422962DE032E007EC11E061
:10F220000E9472F40E9474AC08959A938A93C80164
:10F23000E2ECFDE10081118104FF2DC02AE230E003
:10F2400007EC11E00E94177248E050E09C01275F34
:10F250003F4F0DE012E00E9404722DE032E007EC17
:10F2600011E00E9472F40E9474AC2BE331E007ECD1
:10F2700011E00E9417724CE050E09C012F5E3F4F5E
:10F280000DE012E00E9404722DE032E007EC11E084
:10F290000E9472F407C04DE954E060E007EC11E011
:10F2A0000E944AF40E9474AC8991999108950E9439
:10F2B00060F3D801C901442EAFDE442009F444C0F4
:10F2C000FC01008110E01A930A93FC01018110E017
:10F2D0001A930A930D911C9111971A930A93FD01A9
:10F2E000038110E01A930A93FD01028110E01A9342
:10F2F0000A934FED50E060E00DE012E00E944AF406
:10F300002A960DE012E00E941EAB2FE330E00DE0E4
:10F3100012E00E941772E5EDFDE1008111811A9360
:10F320000A9348EB50E060E003E512E00E944AF4E3
:10F33000229623E532E00DE012E00E9472F40DE027
:10F3400012E00E940AAB21C0FC01008110E01A9378
:10F350000A93FC01018110E01A930A930D911C910C
:10F3600011971A930A93FD01038110E01A930A93EF
:10F37000FD01028110E01A930A934FED50E060E026
:10F3800007EC11E00E944AF42A960E9474ACE5E072
:10F390000C9471F30E945DF3A097A02F812FAA23F4
:10F3A00049F441E0382F31600DEA16E020E00E9478
:10F3B000A7AB12C0B0E0BA93AA9344E752E060E072
:10F3C0000DE012E00E944AF4229631E0282F2160DD
:10F3D0000DE012E00E9410AC4A2F50E060E070E0B7
:10F3E00000E210E020E030E00E948CF2065F1F4F48
:10F3F0002F4F3F4F28013901A201B3019E0100E2C6
:10F4000010E00E948072088119811A930A930D817D
:10F4100010E01A930A930E8110E01A930A9346E7BC
:10F4200051E060E007EC11E00E944AF426960E9449
:10F4300074AC8E01FADEAA2371F00D8D1E8D1A9325
:10F440000A9349E852E060E007EC11E00E944AF4B8
:10F4500022960E9474ACA096E8E00C946EF39A9306
:10F460008A93902F80E000917B11081780F0192F6C
:10F47000082F90DF00917B11801738F440E021E0E5
:10F4800030E00BEA11E00E94EFA78395ECCF899161
:10F49000999108950E945DF36197802FE82FF0E025
:10F4A0003196FA93EA934DEB59E060E00DE012E0FB
:10F4B0000E944AF4229631E021E00DE012E00E9421
:10F4C00010AC482F50E060E070E001E110E020E077
:10F4D00030E00E948CF2065511412D4F3F4F28011C
:10F4E0003901A201B3019E0101E110E00E94807286
:10F4F000002331F006E110E0EEE7F1E10083118333
:10F50000088119811A930A930D8110E01A930A93C6
:10F510000E8110E01A930A9346E751E060E007EC91
:10F5200011E00E944AF426960E9474AC45E09E01C8
:10F530002C5F3F4F0DE012E00E949190E1EBF8E06C
:10F5400030E0A7ECB1E00E94A5F42DE032E007EC3A
:10F5500011E00E9472F40E9474AC0E851F851A930C
:10F560000A9349E852E060E007EC11E00E944AF497
:10F5700022960E9474AC6196E8E00C946EF38A9334
:10F5800080E000918B11801720F4082F83DF839592
:10F59000F8CF899108950E9460F3402EC9010AE7CF
:10F5A0001CE1D801082F092B29F09C01042D0E9491
:10F5B00061AD36C045E150E020E030E08D010E94B1
:10F5C000B3F3AC01242D8D010E942CAD00917B1171
:10F5D00010E01A930A9346EA50E060E08D01005F64
:10F5E0001F4F0E944AF4229621E130E08D010F5F07
:10F5F0001F4F0E941BAD10E01A930A934CE950E094
:10F6000060E08D010E5E1F4F0E944AF4229603E0D7
:10F61000FD01048B41E025E130E08D010E9459E5B8
:10F62000E5E00C9471F30E9459F32B97772407ECD3
:10F6300011E0C8010AE510EA280100E010E0EEE759
:10F64000F1E1008311830E94E4A2002339F00AE271
:10F6500010E0EEE7F1E1008311836EC20091781DA6
:10F66000002339F009E010E0EEE7F1E100831183B7
:10F6700063C200918B11043138F00CE410E0EEE726
:10F68000F1E10083118358C20E949A6110E0EEE715
:10F69000F1E100831183EEE7F1E100811181012B9B
:10F6A00009F04AC2E8E0F0EA048903FF07C00DE46C
:10F6B00010E0EEE7F1E1008311833EC2E2ECFDE1F0
:10F6C0000081118100FF07C002E010E0EEE7F1E1E8
:10F6D0000083118331C282010E948DE9EEE7F1E1DE
:10F6E00000831183EEE7F1E100811181012B09F024
:10F6F00023C29E01295F3F4F8201045E1F4F0E947B
:10F7000026A0EEE7F1E100831183EEE7F1E100814D
:10F710001181012B09F010C29E012B5F3F4F8E011A
:10F720000F5F1F4F0E947EB9EEE7F1E10083118366
:10F73000EEE7F1E100811181012B09F0FDC10981A2
:10F740001A81003D27E0120730F009811A81033049
:10F7500028E0120738F007E010E0EEE7F1E100835F
:10F760001183EAC19E012F5F3F4F8E01095F1F4F3A
:10F770000E9496A0023039F007E010E0EEE7F1E1D8
:10F7800000831183D9C121E08E010F5F1F4F0E94BA
:10F79000F3E9EEE7F1E100831183EEE7F1E10081A7
:10F7A0001181012B09F0C8C128E030E082010A5F15
:10F7B0001F4F0E94FAEAEEE7F1E100831183EEE7C2
:10F7C000F1E100811181012B09F0B6C12CE030E09C
:10F7D0008201015F1F4F0E94FAEAEEE7F1E1008328
:10F7E0001183EEE7F1E100811181012B09F0A4C141
:10F7F00000917B11602EE2ECFDE10081118104FF9C
:10F8000024C02AE031E18E01095F1F4F0E9496A0BB
:10F81000033039F409E010E0EEE7F1E100831183F1
:10F820008BC100918A11053038F003E110E0EEE75A
:10F83000F1E10083118380C1E8E8FEE104811581D4
:10F84000FC01058F168F63940BC000E010E0FC01F3
:10F85000058F168F00E010E0E8E8FEE104831583D1
:10F860000E944F4D00E00E946386EEE7F1E10081C7
:10F870001181012B09F060C10AE510EA280145E079
:10F8800050E092012B5D3F4F8C010C5F1F4F0E9497
:10F8900097F309811A812B813C81FC01008311833C
:10F8A0002283338348E050E092012A5F3F4F8C016E
:10F8B000075F1F4F0E9497F34CE050E09201215FD9
:10F8C0003F4F8C010F5E1F4F0E9497F340E02FE1E6
:10F8D00030E08C010E94834DFC01078FF894462D87
:10F8E00050E060E070E000E210E020E030E00E94D4
:10F8F0008CF2065F1F4F2F4F3F4F48015901A40163
:10F90000B5019C0100E210E00E949572002359F0BD
:10F91000789401E00093791D01E010E0EEE7F1E159
:10F920000083118309C178942AE031E18901FC0147
:10F9300040E250E00E943FF360927B1100E00883B8
:10F94000E2ECFDE100811181006111830083EAE8AE
:10F95000F1E1008103950083F89440E050E060E01D
:10F9600070E09E0101E010E00E9495720023C1F456
:10F9700045E050E863E070E02BE731E101E010E0A2
:10F980000E949572002361F448E050E863E070E063
:10F990002AE831E101E010E00E949572002359F05D
:10F9A000789401E00093791D01E010E0EEE7F1E1C9
:10F9B00000831183C1C078940E942B45012B51F024
:10F9C00001E00093791D01E010E0EEE7F1E1008332
:10F9D0001183B2C0E1EDFDE100811181E3EDFDE1B4
:10F9E0000083118319DB00E23ADD41E031E005EFED
:10F9F00016E020E00E94A7AB00917B110023D1F517
:10FA00000FE71AE60E94B788ECE9F2E030E0ADE0DB
:10FA1000B2E00E94A5F40DE012E00E941EABE8E8FF
:10FA2000FEE1048115811A930A9343EB50E060E0F4
:10FA30000DE012E00E944AF422960DE012E00E94CE
:10FA40000AAB0E9474ACEFEBF2E030E0ADE0B2E064
:10FA50000E94A5F40DE012E00E941EAB2DE032E002
:10FA60000FE71AE60E94D68D0DE012E00E940AAB65
:10FA70000E9474AC07E81AE60E94B78804ED19E604
:10FA80000E94B788EEEAF2E030E0ADE0B2E00E941A
:10FA9000A5F40DE012E00E941EAB2DE032E004ED73
:10FAA00019E60E94D68D0DE012E00E940AAB0E947A
:10FAB00074AC00917B11002351F441E050E060E010
:10FAC00070E020E031E101E010E00E9495727724BF
:10FAD00073949E012B5F3F4F8E010F5F1F4F0E945B
:10FAE000BB6710E0EEE7F1E100831183EEE7F1E19F
:10FAF00000811181012B01F542DD00917B11002372
:10FB000041F441E031E00EEB16E020E00E94A7ABAB
:10FB100007C041E031E00AED16E020E00E94A7AB0B
:10FB20000E9461A9E1EDFDE1008111810F5F1F4F8E
:10FB3000008311830E94BE6800E010E0E3EDFDE168
:10FB40000083118320E0172D00E00E94B586EEE7C8
:10FB5000F1E12081318101E41EDD2B96ECE00C9473
:10FB60006AF30E9461F3C80100E010E0EEE7F1E102
:10FB7000008311830091771D002339F001E110E02B
:10FB8000EEE7F1E100831183F3C00091781D0023BB
:10FB900039F009E010E0EEE7F1E100831183E8C0FD
:10FBA000E2ECFDE10081118100FF07C002E010E0FE
:10FBB000EEE7F1E100831183DBC00E94E4A2003193
:10FBC00039F00AE210E0EEE7F1E100831183D0C0E2
:10FBD0008C010C5F1F4F0E94ACF4D8010A2F0B2B35
:10FBE00039F408E110E0EEE7F1E100831183C0C0D1
:10FBF00027E030E08C010C5F1F4F0E94FAEAEEE72D
:10FC0000F1E100831183EEE7F1E100811181012B25
:10FC100009F0AEC042E050E060E070E023E031E186
:10FC200007E010E00E948072002339F006E110E046
:10FC3000EEE7F1E10083118318C047E050E02FEFB9
:10FC400030E007EC11E00E94B3F347E050E023E01E
:10FC500031E107EC11E00E947FF3012B31F00CE25F
:10FC600010E0EEE7F1E100831183EEE7F1E10081BE
:10FC70001181012B09F07CC042E350E020E030E02C
:10FC800007EC11E00E94B3F340E050E863E070E05D
:10FC900027EC31E002E310E00E949572002339F076
:10FCA0000FE010E0EEE7F1E10083118323C040E0B4
:10FCB00050E863E070E029EF31E002E310E00E94D9
:10FCC0008072002339F006E110E0EEE7F1E10083F5
:10FCD000118310C042E350E029EF31E007EC11E05E
:10FCE0000E947FF3012B31F00FE010E0EEE7F1E12D
:10FCF00000831183EEE7F1E100811181012BC1F551
:10FD000042E050E060E070E09C012C5F3F4F07E074
:10FD100010E00E949572002339F00FE010E0EEE74A
:10FD2000F1E10083118324C042E050E060E070E024
:10FD300023E031E107E010E00E948072002339F0F7
:10FD400006E110E0EEE7F1E10083118311C047E026
:10FD500050E023E031E18C010C5F1F4F0E947FF3E4
:10FD6000012B31F00FE010E0EEE7F1E100831183A9
:10FD7000EEE7F1E1208131810DE50E9461ADE4E023
:10FD80000C9472F38A93802F41E031E007E217E090
:10FD900020E00E94A7AB082F015019F00A9581F0CE
:10FDA00016C041E031E00DE317E020E00E94A7AB70
:10FDB00041E031E009E517E020E00E94A7AB07C071
:10FDC00041E031E00FE717E020E00E94A7AB41E0FF
:10FDD00031E00FED17E020E00E94A7ABEDE8FDE178
:10FDE000008111811A930A930091901D10E01A93DB
:10FDF0000A9300918F1D10E01A930A93E9E8FDE140
:10FE0000008111811A930A9300918C1D10E01A93BE
:10FE10000A9300918B1D10E01A930A934DE951E06B
:10FE200060E004E510EA0E944AF42C9631E021E0FB
:10FE300004E510EA0E9410AC41E031E007EF17E062
:10FE400020E00E94A7ABE7EAFDE1008111811A934F
:10FE50000A93E5EAFDE1008111811A930A934AE8C9
:10FE600051E060E004E510EA0E944AF4249631E093
:10FE700021E004E510EA0E9410AC89910895BA933C
:10FE8000AA93EBE3F1E1008111811A930A930091A7
:10FE90003E1110E01A930A9300913D1110E01A935D
:10FEA0000A9346E751E060E007EC11E00E944AF453
:10FEB00026960E9474ACEBE3F1E1048115811A935C
:10FEC0000A9340EC51E060E007EC11E00E944AF434
:10FED00022960E9474ACE1EFF2E030E0ADE0B2E0D7
:10FEE0000E94A5F40DE012E00E941EAB2DE032E06E
:10FEF00002E411E10E94D68D0DE012E00E940AABEF
:10FF00000E9474AC40E021E030E00BEA11E00E9476
:10FF1000EFA7A991B9910895EEE7F1E10081118170
:10FF2000012B81F44EE458E060E007EC11E00E9400
:10FF30004AF40E9474AC40E021E030E00BEA11E0AA
:10FF40000E94EFA70895BA93AA9341E031E00FE32E
:10FF500018E020E00E94A7ABE1EFF2E030E0ADE076
:10FF6000B2E00E94A5F40DE012E00E941EAB2DE06D
:10FF700032E002EB1DE10E94D68D0DE012E00E94FE
:10FF80000AAB0E9474ACA991B99108950E9459F3EB
:10FF9000602EA0E0B0E080E490E002E0601609F09E
:10FFA00072C04424552408EB40160BE0500608F0BC
:10FFB0006AC0ECE8F1E1008111814016510608F0B9
:10FFC00062C00A2F0B2B09F05EC040E0959D9001A6
:10FFD000849D8001949D100D211D341F589E100D8D
:10FFE000211D341F06551F4F2F4F3F4F4801590108
:10FFF000A401B5012BE331E18C010E948072002342
:020000021000EC
:1000000019F0A6E1B0E03AC040917A119C0121506C
:1000100030400BE311E10E94834D002371F5EBE3C7
:10002000F1E104811581E9EAFDE1208131810217C6
:10003000130760F0EBEAFDE100811181EBE3F1E1F0
:10004000248135810217130708F019DFEBEAFDE17F
:1000500000811181EBE3F1E124813581021713075F
:1000600090F0E7EAFDE100811181EBE3F1E1248109
:1000700035810217130710F406C04EDF01E0400E71
:1000800000E0501E90CF0A2F0B2B11F541E031E01C
:1000900000E118E020E00E94A7ABEFEAFDE100815B
:1000A00011811A930A93EDEAFDE1008111811A93FF
:1000B0000A934AE851E060E00DE012E00E944AF441
:1000C000249631E021E00DE012E00E9410AC3BDF0D
:1000D0008D01ECE00C946AF30E9459F3602EA0E0CD
:1000E000B0E080E490E0662009F069C04424552423
:1000F00008EB40160BE0500608F061C0ECE8F1E1B7
:10010000008111814016510608F059C00A2F0B2BAF
:1001100009F055C040E0959D9001849D8001949D1B
:10012000100D211D341F589E100D211D341F065522
:100130001F4F2F4F3F4F48015901A401B5012BE339
:1001400031E18C010E948072002319F0A6E1B0E039
:1001500031C040917A119C01215030400BE311E1F4
:100160000E94834D002329F521E93DE10BE311E1D4
:100170000E9496A0033048F425E93DE10BE311E12C
:100180000E9496A0023008F07ADE25E93DE10BE3FB
:1001900011E10E9496A0013091F0E7EAFDE10081B3
:1001A0001181EBE3F1E1248135810217130710F48B
:1001B00006C0B2DE01E0400E00E0501E99CF0A2FCB
:1001C0000B2BB1F541E031E008E218E020E00E949D
:1001D000A7ABEDE9FDE1008111811A930A9300912B
:1001E000A01D10E01A930A9300919F1D10E01A932E
:1001F0000A93E9E9FDE1008111811A930A930091C4
:100200009C1D10E01A930A9300919B1D10E01A9315
:100210000A934DE951E060E00DE012E00E944AF4DB
:100220002C9631E021E00DE012E00E9410AC8BDE54
:100230008D01ECE00C946AF3F8012081205019F054
:100240002A9571F10895EBE3F1E1408151816281DA
:100250007381E9E9FDE14083518362837383EBE3BA
:10026000F1E14081518162817381EDE9FDE14083DB
:10027000518362837383EBE3F1E124813581EDEAFD
:10028000FDE120833183EBE3F1E124813581EFEA65
:10029000FDE120833183F801208123952083089597
:1002A000EBE3F1E14081518162817381EDE9FDE190
:1002B0004083518362837383EBE3F1E124813581D1
:1002C000EFEAFDE120833183089502EB1DE10E94F6
:1002D000B788089522E431E102EB1DE10E94138A00
:1002E000002319F007E110E0089500E010E0089500
:1002F0000E9459F32197A0E0B0E080E490E000E094
:100300000883E3DF4424552408EB40160BE0500635
:1003100008F06EC0ECE8F1E1008111814016510651
:1003200008F066C00A2F0B2B09F062C040E0959DD3
:100330009001849D8001949D100D211D341F589EB5
:10034000100D211D341F06551F4F2F4F3F4F4801E1
:100350005901A401B5012BE331E18C010E948072A7
:10036000002319F0A6E1B0E03EC040917A119C0153
:10037000215030400BE311E10E94834D002399F599
:10038000EBE3F1E104811581E9EAFDE120813181AE
:100390000217130790F0EBEAFDE100811181EBE316
:1003A000F1E1248135810217130738F093DFD8017A
:1003B0000A2F0B2BE9F48E013FDFEBEAFDE1008110
:1003C0001181EBE3F1E1248135810217130780F0FD
:1003D000E7EAFDE100811181EBE3F1E12481358160
:1003E0000217130728F001E0400E00E0501E8CCFEA
:1003F0008D012196ECE00C946AF30E9459F3219749
:10040000A0E0B0E080E490E000E008835EDF4424F8
:10041000552408EB40160BE0500608F068C0ECE8E5
:10042000F1E1008111814016510608F060C00A2FE9
:100430000B2B09F05CC040E0959D9001849D8001EC
:10044000949D100D211D341F589E100D211D341F29
:1004500006551F4F2F4F3F4F48015901A401B501C9
:100460002BE331E18C010E948072002319F0A6E198
:10047000B0E038C040917A119C01215030400BE32C
:1004800011E10E94834D002369F521E93DE10BE371
:1004900011E10E9496A0033090F425E93DE10BE3C1
:1004A00011E10E9496A0023050F001E00093B11DCE
:1004B00011DFD8010A2F0B2BD1F48E01BDDE25E907
:1004C0003DE10BE311E10E9496A0013081F0E7EAE3
:1004D000FDE100811181EBE3F1E124813581021717
:1004E000130728F001E0400E00E0501E92CF8D016E
:1004F0002196ECE00C946AF30E945FF32801D90185
:10050000842F952F40E09D0182010E945779ECE7EE
:10051000F1E1008111810F5F1F4F1A930A9343E4A9
:1005200053E060E004E510EA0E944AF4229631E0CC
:1005300021E004E510EA0E9410AC843041F441E06F
:1005400031E002EC17E020E00E94A7AB55C08230FA
:1005500011F08330E1F441E031E00FE917E020E0F1
:100560000E94A7ABEBEAFDE1008111811A930A9387
:10057000E9EAFDE1008111811A930A934AE851E00A
:1005800060E004E510EA0E944AF424962FC041E09E
:1005900031E001EB17E020E00E94A7ABE5E9FDE1C7
:1005A000008111811A930A930091981D10E01A930B
:1005B0000A930091971D10E01A930A93E1E9FDE177
:1005C000008111811A930A930091941D10E01A93EF
:1005D0000A930091931D10E01A930A934DE951E09C
:1005E00060E004E510EA0E944AF42C9631E021E034
:1005F00004E510EA0E9410AC40E021E030E00BEA94
:1006000011E00E94EFA700E20E942F7A0E94BF7AB9
:1006100040E021E030E00BEA11E00E94EFA79923CF
:1006200019F0092FAFDB1CC0843031F402E0AEDCDE
:10063000EEE7F1E100831183882311F0813031F47A
:10064000082F4ADDEEE7F1E100831183823011F0DB
:10065000833031F4082F9ADCEEE7F1E10083118357
:10066000EEE7F1E100811181012B51F40E9461A9B3
:1006700000E00E94D3A800E000937F1D0E9465A8BF
:10068000EEE7F1E100811181012BE1F4E1EDFDE103
:10069000008111810F5F1F4F00831183ECE7F1E1AF
:1006A000008111810F5F1F4F00831183F89446E092
:1006B00050E863E070E02CE731E102E010E00E94D6
:1006C00095727894E6E00C9470F30E945CF3802EAF
:1006D000D9013A012B0104E510EAC80145E151E0D6
:1006E00020E030E004E510EA0E94B3F30A2F0B2B60
:1006F00029F09D01082D0E9461ADADC0AD01282DEE
:100700008C010E942CAD47E050E023E031E18C01E8
:10071000005F1F4F0E94047248E050E023E131E186
:100720008C01085E1F4F0E9404724CE050E02BE1E8
:1007300031E18C010F5D1F4F0E9404722DED3DE1F0
:100740008C01025D1F4F0E949AF426E03EE18C016D
:10075000095A1F4F0E949AF42FE23EE18C01005883
:100760001F4F0E949AF428E53EE18C0107551F4F68
:100770000E949AF4ECE7F1E1008111811A930A9347
:1007800048EB50E060E08C0100521F4F0E944AF499
:10079000229693018C010E521F4F0E9462A092017B
:1007A0008C0105521F4F0E947FA029E93DE18C0179
:1007B0000A511F4F0E9462A02DE93DE18C010151B9
:1007C0001F4F0E9462A0EDEAFDE1008111811A93A2
:1007D0000A9343EB50E060E08C0108501F4F0E94E9
:1007E0004AF42296EFEAFDE1008111811A930A93FF
:1007F00043EB50E060E08C0103501F4F0E944AF42D
:1008000022969C012E5F3E4F02EB1DE10E94D68D89
:1008100000E0FC01EF52FF4F008321E131E08C0149
:100820000F5F1F4F0E941BAD10E01A930A934CE913
:1008300050E060E08C010E5E1E4F0E944AF422964A
:1008400003E0FC01EC5EFE4F008340E025E131E077
:100850008C010E9459E5E9E00C946DF30E945DF370
:1008600080E090E0A0E4B0E04AEA50E060E070E0B0
:100870002BE331E18D010E948072002319F086E1A3
:1008800090E014C0EBE3F1E100811181228133811A
:10089000E9E8FDE10083118322833383EBE3F1E197
:1008A00004811581E5EAFDE100831183ECE8F1E1C3
:1008B000408151814150504060E0B59F9001A49F1C
:1008C0008001B49F100D211D361F5A9F100D211D50
:1008D000361F06551F4F2F4F3F4F28013901A201E8
:1008E000B3012BE331E18D010E948072002319F0E6
:1008F00086E190E014C0EBE3F1E1008111812281F7
:100900003381EDE8FDE10083118322833383EBE340
:10091000F1E104811581E7EAFDE1008311838C0197
:10092000E8E00C946EF30E9461F326970AE510EA62
:10093000D80100E010E0EEE7F1E1008311830091BF
:10094000781D002339F009E010E0EEE7F1E10083C3
:10095000118396C1E2ECFDE10081118100FF07C027
:1009600002E010E0EEE7F1E10083118389C1E2ECDF
:10097000FDE10081118104FD07C004E110E0EEE714
:10098000F1E1008311837CC1ECE8F1E10081118188
:10099000012B39F40FE110E0EEE7F1E10083118360
:1009A0006FC18D010E948DE9EEE7F1E100831183B3
:1009B000EEE7F1E100811181012B09F061C19E0197
:1009C0008E010E5F1F4F0E947EB9EEE7F1E10083BA
:1009D0001183EEE7F1E100811181012B09F050C193
:1009E000FD0106810E941C90802F44E050E020E031
:1009F00030E0082F10E00E94D3EAEEE7F1E1008337
:100A00001183EEE7F1E100811181012B09F038C17A
:100A100025DFEEE7F1E100831183EEE7F1E10081EC
:100A20001181012B09F02CC10E944F4D00E00E9462
:100A30006386EEE7F1E100811181012B09F020C10D
:100A40000AE510EAD801E1EDFDE100811181E3ED55
:100A5000FDE10083118300E00093B11D0091791D39
:100A6000002311F48430E9F484E0E5EAFDE100813B
:100A70001181E9EAFDE100831183E7EAFDE10081EC
:100A80001181EBEAFDE10083118332DCEEE7F1E155
:100A900000831183EEE7F1E100811181012B09F060
:100AA000EFC0882319F0813009F075C021E93DE1DC
:100AB0008D01085F1F4F0E9426A0EEE7F1E1008341
:100AC0001183EEE7F1E100811181012B09F0D8C01B
:100AD00025E93DE18D010F5E1F4F0E9426A0EEE744
:100AE000F1E100831183EEE7F1E100811181012B37
:100AF00009F0C6C025E93DE101E91DE10E9496A08B
:100B0000013031F405E010E0EEE7F1E100831183FC
:100B1000EEE7F1E100811181012B09F0B1C029E874
:100B20003DE105E91DE10E9496A0033041F02DE86A
:100B30003DE101E91DE10E9496A0013071F451E010
:100B4000482F9E018E010E5F1F4FD6DC05E110E09D
:100B5000EEE7F1E10083118393C04FDCEEE7F1E1B2
:100B600000831183EEE7F1E100811181012B09F08F
:100B700087C00091B11D002371F452E0482F9E01FF
:100B80008E010E5F1F4FB8DC05E110E0EEE7F1E1EA
:100B90000083118375C0823019F0833009F069C079
:100BA0008D01085F1F4F0E9482F1E9EAFDE1008399
:100BB00011838D010F5E1F4F0E9482F1EBEAFDE170
:100BC00000831183EBEAFDE100811181E9EAFDE197
:100BD000208131810217130738F405E010E0EEE7B9
:100BE000F1E1008311834CC0E7EAFDE1008111814E
:100BF000E9EAFDE1208131810217130758F4E7EAA1
:100C0000FDE100811181EBEAFDE1208131810217D4
:100C10001307B0F0E9EAFDE100811181E5EAFDE1A9
:100C20002081318102171307C8F4EBEAFDE100814E
:100C30001181E5EAFDE1208131810217130770F48B
:100C400051E0482F9E018E010E5F1F4F55DC05E1DC
:100C500010E0EEE7F1E10083118312C049DBEEE71B
:100C6000F1E100831183EEE7F1E100811181012BB5
:100C700039F450E0482F9E018E010E5F1F4F3CDC7F
:100C800000E010E0E3EDFDE10083118320E010E0DF
:100C900000E00E94B586BE01AE014E5F5F4FEEE7F9
:100CA000F1E12081318102E410DD2696E4E00C942C
:100CB00072F300E00093861D00E010E0E1E8FEE141
:100CC0000083118308958A93802F0E944F4D809353
:100CD000B9010091861D002309F442C0EEE7F1E15D
:100CE00000811181012B69F50091861D015029F0C9
:100CF0000A9581F00A95A1F024C0ECEDFDE1008198
:100D00000F70008301E00E940DA90E94B4A60E940A
:100D1000B8A817C000E00E940DA90E94B4A611C097
:100D2000ECEDFDE100810F70008301E00E940DA950
:100D30000E94B4A60E94B8A800E00E940DA90E94DB
:100D4000B4A6EEE7F1E100811181012B49F400E046
:100D500010E0E8E8F1E10083118300E00093861DD4
:100D600000E00093B901899108950E945DF32397F3
:100D7000802F412E922F0E944F4D0091861D0023FF
:100D800009F0EDC1EEE7F1E1008111810A3020E0C8
:100D9000120749F0EEE7F1E100811181013220E014
:100DA000120709F0A4C1ECEDFDE100810F70008392
:100DB0000E945EA841E031E006E614E020E00E94D7
:100DC000A7AB442009F4F7C0EFE9FAE601811281EC
:100DD0001A930A9349E152E060E00DE012E00E94AC
:100DE0004AF4229631E021E00DE012E00E9410ACBE
:100DF000E9E3F2E030E0A3E5B2E00E94A5F400915F
:100E00009F6A005089F00A9561F10A9509F463C060
:100E10000A9509F47DC00A9509F497C00A9509F46A
:100E2000AFC00750D9F133C129E630E007EC11E03B
:100E30000E94177227EC31E003E512E00E9472F481
:100E40002DE032E00CEA1AE60E94D68D03E512E0AE
:100E50000E941EAB0DE012E00E940AAB0E9474AC2F
:100E600016C122ED30E007EC11E00E94177227EC6A
:100E700031E003E512E00E9472F42DE032E00CEA6A
:100E80001AE60E94D68D03E512E00E941EAB0DE02B
:100E900012E00E940AAB0E9474ACF9C027ED34E066
:100EA00007EC11E00E94177227EC31E003E512E035
:100EB0000E9472F42DE032E00CEA1AE60E94D68D10
:100EC00003E512E00E941EAB0DE012E00E940AABA7
:100ED0000E9474ACDCC027EE30E007EC11E00E9409
:100EE000177227EC31E003E512E00E9472F42DE066
:100EF00032E00CEA1AE60E94D68D03E512E00E9469
:100F00001EAB0DE012E00E940AAB0E9474ACBFC0A1
:100F10002CEF30E007EC11E00E94177227EC31E073
:100F200003E512E00E9472F42DE032E00CEA1AE6CA
:100F30000E94D68D03E512E00E941EAB0DE012E088
:100F40000E940AAB0E9474ACA2C0EFE9FAE60581E8
:100F500016811A930A934BE053E060E007EC11E02E
:100F60000E944AF4229627EC31E003E512E00E9449
:100F700072F431E021E003E512E00E9410AC87C07A
:100F8000EFE9FAE6058116811A930A934EEF52E0D3
:100F900060E007EC11E00E944AF4229627EC31E071
:100FA00003E512E00E9472F431E021E003E512E073
:100FB0000E9410AC6CC0E1EDFDE1008111811A933B
:100FC0000A934AEF51E060E00DE012E00E944AF41B
:100FD000229631E021E00DE012E00E9410ACE2EC3C
:100FE000FDE10081118100FF32C02AE13AE604E20E
:100FF0001AE60E94138AE2E2FAE6008111810F5F8D
:101000001F4F008311832AE13AE6D90100EB602EDD
:101010000FE1702E4091281F50E00FEB10E00E946E
:1010200046F2600E711E83019D010E94138A409159
:10103000281F50E00FEB10E00E9446F2F801E25545
:10104000F04E008111810F5F1F4F00831183E2EC8E
:10105000FDE10081118100601C6700831183E2ECD7
:10106000FDE1008111810F7F1C7F00831183E5ED7D
:10107000FDE1008111810F5F1F4F00831183E1EDBE
:10108000FDE1008111810F5F1F4F00831183E2ECAE
:10109000FDE10081118101FF05C010E000E10E9427
:1010A00021A904C010E000E00E9421A947E351E01B
:1010B00060E007EC11E00E944AF40E9474ACE4EC9A
:1010C000FDE1008102FF04C001E00093861D0FC016
:1010D000E2ECFDE10081118100FD02C0882321F0D6
:1010E00003E00093861D03C001E00093861DEEE738
:1010F000F1E100811181012B91F5E4ECFDE100812A
:1011000002FD2DC0E2ECFDE10081118100FD02C075
:10111000882329F1E1E8FEE100811181012BE1F052
:10112000E9E3F1E004910883EAE3F1E00491098343
:10113000E2ECFDE10081118101FF03C000E90A83B7
:1011400002C000E80A8343E050E09E01E1E8FEE1CE
:10115000008111810E94D17102E00093861D9923C4
:1011600011F000E0B0DD2396E8E00C946EF340E06F
:1011700050E060E070E0F801448355836683778334
:1011800040E050E060E070E0F8014083518362830A
:10119000738308950E9461F3F80140835183628351
:1011A000738380E090E0A0E0B0E0F8018483958351
:1011B000A683B783E4E00C9472F3F9014081518176
:1011C00062817381F8014083518362837383F901E3
:1011D0004481558166817781F80144835583668314
:1011E00077830895F8014481558166817781F801FC
:1011F0000081118122813381042B152B262B372B63
:10120000012B022B032B11F401E0089500E0089557
:10121000F8014481558166817781F9010480158048
:1012200026803780401551056205730599F4F90150
:101230004081518162817381F80100811181228195
:101240003381401751076207730710F401E00895D6
:1012500000E00895F9014481558166817781F801A4
:101260000481158126813781401751076207730772
:1012700010F401E0089500E008950E9461F3D801A0
:10128000C9019C018D01C4DF002311F001E020C0E1
:10129000FD010481158126813781FC01448155813E
:1012A00066817781041715072607370781F40D91AA
:1012B0001D912D913C91FC0140815181628173818E
:1012C000041715072607370711F402E001C003E0F1
:1012D000E4E00C9472F30E9459F3D80119012A0139
:1012E0003B0160E08D01F10148E050E00E943FF3D6
:1012F0000D911D912D913C91040D151D261D371D3D
:101300003C932E931E930E930D911D912D913C9124
:101310001397F10180809180A280B3800815190590
:101320002A053B0568F4FD0104811581268137817A
:101330000F5F1F4F2F4F3F4F048315832683378343
:10134000FD010481158126813781F101848095801A
:10135000A680B780081519052A053B0508F461E049
:10136000062FECE00C946AF30E945DF31801DA0199
:1013700080E08101F90148E050E00E943FF34D9187
:101380005D916D917C911397F10140805180628055
:101390007380440E551E661E771E40825182628203
:1013A0007382FD014481558166817781F10144801A
:1013B000558066807780440E551E661E771E4482D7
:1013C000558266827782F101408151816281738109
:1013D000F90140805180628073804415550566058F
:1013E000770568F4F10144815581668177814F5F0B
:1013F0005F4F6F4F7F4F4483558366837783F1013F
:101400004481558166817781F901448055806680E9
:101410007780441555056605770508F481E0082FA7
:10142000E8E00C946EF30E9460F36097C801D90164
:101430009E018901FC0148E050E00E943FF3AD01AC
:101440009E018E01085F1F4F8FDF402E442049F41C
:101450009E01285F3F4F8C01F90148E050E00E9457
:101460003FF3042D6096E5E00C9471F30E945DF368
:101470001801DA0180E08101F90148E050E00E94A2
:101480003FF34D915D916D917C911397F1014080F7
:10149000518062807380441A550A660A770A408236
:1014A000518262827382FD01448155816681778118
:1014B000F1014480558066807780441A550A660A97
:1014C000770A4482558266827782F9014081518190
:1014D00062817381F1014080518062807380441584
:1014E00055056605770568F4F101448155816681EB
:1014F00077814150504060407040448355836683FB
:101500007783F9014481558166817781F1014480B7
:10151000558066807780441555056605770508F483
:1015200081E0082FE8E00C946EF30E9460F360976E
:10153000C801D9019E018901FC0148E050E00E94E8
:101540003FF3AD019E018E01085F1F4F8FDF402EDC
:10155000442049F49E01285F3F4F8C01F90148E087
:1015600050E00E943FF3042D6096E5E00C9471F387
:101570000E9456F3289718016901CA019101F601EA
:101580008C0146805780D8016D907C90A0E0579CDC
:10159000B001469CA001569C500D611D7A1F749CA1
:1015A000500D611D7A1F4C835D836E837F83448061
:1015B0005580D80112966D907C904C815D816E8132
:1015C0007F81EE24579C600D711D469C400D511D7E
:1015D0006E1D7E1D569C500D611D7E1D749C500D10
:1015E000611D7E1D4C835D836E837F8342805380AB
:1015F000D80114966D907C904C815D816E817F81C5
:10160000EE24579C600D711D469C400D511D6E1DB2
:101610007E1D569C500D611D7E1D749C500D611DDC
:101620007E1D4C835D836E837F8340805180D80113
:1016300016966D907C904C815D816E817F81EE2449
:10164000579C600D711D469C400D511D6E1D7E1DE9
:10165000569C500D611D7E1D749C500D611D7E1D9C
:101660004C835D836E837F8344805580D8016D9069
:101670007C90A0E0579CB001469CA001569C500D68
:10168000611D7A1F749C500D611D7A1FD101149643
:101690004D935D936D937C9342805380D801129655
:1016A0006D907C90D10114964D915D916D917C91DE
:1016B000EE24579C600D711D469C400D511D6E1D02
:1016C0007E1D569C500D611D7E1D749C500D611D2C
:1016D0007E1D7C936E935E934E9340805180D80123
:1016E00014966D907C90D10114964D915D916D9101
:1016F0007C91EE24579C600D711D469C400D511D40
:101700006E1D7E1D569C500D611D7E1D749C500DDE
:10171000611D7E1D7C936E935E934E934280538039
:10172000D8016D907C90A0E0579CB001469CA00130
:10173000569C500D611D7A1F749C500D611D7A1FBF
:10174000488359836A837B8340805180D8011296F5
:101750006D907C90A0E0579CB001469CA001569CE7
:10176000500D611D7A1F749C500D611D7A1F4A0136
:101770005B01488159816A817B81480D591D6A1D31
:101780007B1D488359836A837B83488159816A81A1
:101790007B81481559056A057B0560F44C815D81A4
:1017A0006E817F814F5F5F4F6F4F7F4F4C835D83B3
:1017B0006E837F8340805180D8016D907C90A0E043
:1017C000579CB001469CA001569C500D611D7A1F8C
:1017D000749C500D611D7A1FD1014D935D936D93E3
:1017E0007C93D90112964D915C9160E070E04A01C2
:1017F0005B01488159816A817B81480D591D6A1DB1
:101800007B1D488359836A837B83488159816A8120
:101810007B81481559056A057B0560F44C815D8123
:101820006E817F814F5F5F4F6F4F7F4F4C835D8332
:101830006E837F834A815B8160E070E0D101149602
:101840004D905D906D907C90440E551E661E771EE7
:101850007C926E925E924E924C815D81D901169679
:101860006D917C91640F751F7C936E9348815981B3
:10187000D90112964D935C932896EFE00C9467F390
:101880000E9456F32897D801C9012A018C010C5FE8
:101890001F4F68018D010C5F1F4F3801042D052972
:1018A00011F401E069C0FC010481158126813781B2
:1018B000A20160E070E00E94ACF2FD010483158398
:1018C00026833783FC0184809580A680B780FD0144
:1018D0004481558166817781820120E030E00E9459
:1018E0008CF2801A910AA20AB30A88829982AA828B
:1018F000BB82EE2402E0E016C8F50EEFC00E0FEF3B
:10190000D01E0EEF600E0FEF701E088119810A8342
:101910001B83F601008111810883198308811981D5
:101920002A813B81A20160E070E00E94ACF20C834E
:101930001D832E833F830C811D81F301008311835E
:10194000F3014081518182010E9446F220E030E0A3
:10195000488159816A817B81401B510B620B730B5B
:10196000488359836A837B83E394C4CF08811981B8
:10197000FD010087118700E02896EFE00C9467F3E3
:101980000E945DF36097280166242EE230E0820118
:101990000E948FF4C801082F092B89F18C010F5F79
:1019A0001F4F0E94ACF4702E01E0701619F400E392
:1019B000FC01028303E07016F0F0FC0103810533A3
:1019C000D0F000E0FC01038392018E01085F1F4FFD
:1019D00028D141E050E060E070E09E01285F3F4F79
:1019E0008E0179DC002321F492018E01DFD00DC03D
:1019F000662463940AC000E0FC01038306C0E2EBA6
:101A0000FAE030E0D2010E9484F4062D6096E8E00E
:101A10000C946EF30E9461F3D8018D010E94ACF426
:101A2000802F833028F100E090E0FD01E80FF91FDE
:101A3000018390E0FD01E80FF91F3197008190E0EC
:101A4000FD01E80FF91F008390E0FD01E80FF91F89
:101A50003297008190E0FD01E80FF91F3197008374
:101A60000EE290E0FD01E80FF91F3297008318C0E5
:101A7000823041F40C91FD010283FD010181FD01E1
:101A8000038306C000E3FD0102830C91FD01038383
:101A900000E30C930EE2FD01018300E0FD010483ED
:101AA000E4E00C9472F30E9460F36097C801D901DE
:101AB0004AE050E060E070E08E01085F1F4F6ADB93
:101AC0008E0155DB0C91402E1196442019F1AE0188
:101AD000485F5F4F9E018C014BDD9E018901FC0137
:101AE00048E050E00E943FF3442D50E04053504006
:101AF000652F660F660B762F9E018C01ECDB9E0135
:101B00008901FC0148E050E00E943FF30C91402E17
:101B10001196DBCF6096E5E00C9471F30E945CF3C4
:101B20006497380129019E018901F30148E050E0E2
:101B30000E943FF3C201DC014AE050E09E018E01A9
:101B4000065F1F4F9DDE9E01BE01665F7F4F8901CC
:101B5000FB014AE050E00E943FF3088519850A30F6
:101B6000104030F00885095AFC010083019605C039
:101B70000885005DFC01008301968E0133DB0023A4
:101B8000D9F200E0FC0100830197FC010081802E66
:101B90000C91FC0100838C9201971196A817B9074C
:101BA000A0F382016496E9E00C946DF30E9461F366
:101BB000D801C9019C018D01B1DF8C012BDF8C01A3
:101BC000E4E00C9472F30E945DF3D80129012EE247
:101BD00030E082010E948FF4C801082F092BA1F088
:101BE0008C01041915093801762C66248C010F5FCD
:101BF0001F4F0E94ACF4602A712A9C012F5F3F4F57
